:020000040001F9
:20000000FFCFFECFFDCFFCCFFBCFFACFF9CFF8CFF7CFF6CFF5CFF4CFF3CFF2CFF1CFF0CF78
:20002000EFCFEECFEDCFECCFEBCFEACFE9CFE8CFE7CFE6CFE5CFE4CFE3CFE2CFE1CFE0CF58
:20004000DFCFDECFDDCFDCCFDBCFDACFD9CFD8CFD7CFD6CFD5CFD4CFD3CFD2CFD1CFD0CF38
:20006000CFCFCECFCDCFCCCFCBCFCACFC9CFC8CFC7CFC6CFC5CFC4CFC3CFC2CFC1CFC0CF18
:20008000BFCFBECFBDCFBCCFBBCFBACFB9CFB8CFB7CFB6CFB5CFB4CFB3CFB2CFB1CFB0CFF8
:2000A000AFCFAECFADCFACCFABCFAACFA9CFA8CFA7CFA6CFA5CFA4CFA3CFA2CFA1CFA0CFD8
:2000C0009FCF9ECF9DCF9CCF9BCF9ACF99CF98CF97CF96CF95CF94CF93CF92CF91CF90CFB8
:2000E0008FCF8ECF8DCF8CCF8BCF8ACF89CF88CF87CF86CF85CF84CF83CF82CF81CF80CF98
:200100007FCF7ECF7DCF7CCF7BCF7ACF79CF78CF77CF76CF75CF74CF73CF72CF71CF70CF77
:200120006FCF6ECF6DCF6CCF6BCF6ACF69CF68CF67CF66CF65CF64CF63CF62CF61CF60CF57
:200140005FCF5ECF5DCF5CCF5BCF5ACF59CF58CF57CF56CF55CF54CF53CF52CF51CF50CF37
:200160004FCF4ECF4DCF4CCF4BCF4ACF49CF48CF47CF46CF45CF44CF43CF42CF41CF40CF17
:200180003FCF3ECF3DCF3CCF3BCF3ACF39CF38CF37CF36CF35CF34CF33CF32CF31CF30CFF7
:2001A0002FCF2ECF2DCF2CCF2BCF2ACF29CF28CF27CF26CF25CF24CF23CF22CF21CF20CFD7
:2001C0001FCF1ECF1DCF1CCF1BCF1ACF19CF18CF17CF16CF15CF14CF13CF12CF11CF10CFB7
:2001E0000FCF0ECF0DCF0CCF0BCF0ACF09CF08CF07CF06CF05CF04CF03CF02CF01CF00CF97
:20020000FFCFFECFFDCFFCCFFBCFFACFF9CFF8CFF7CFF6CFF5CFF4CFF3CFF2CFF1CFF0CF76
:20022000EFCFEECFEDCFECCFEBCFEACFE9CFE8CFE7CFE6CFE5CFE4CFE3CFE2CFE1CFE0CF56
:20024000DFCFDECFDDCFDCCFDBCFDACFD9CFD8CFD7CFD6CFD5CFD4CFD3CFD2CFD1CFD0CF36
:20026000CFCFCECFCDCFCCCFCBCFCACFC9CFC8CFC7CFC6CFC5CFC4CFC3CFC2CFC1CFC0CF16
:20028000BFCFBECFBDCFBCCFBBCFBACFB9CFB8CFB7CFB6CFB5CFB4CFB3CFB2CFB1CFB0CFF6
:2002A000AFCFAECFADCFACCFABCFAACFA9CFA8CFA7CFA6CFA5CFA4CFA3CFA2CFA1CFA0CFD6
:2002C0009FCF9ECF9DCF9CCF9BCF9ACF99CF98CF97CF96CF95CF94CF93CF92CF91CF90CFB6
:2002E0008FCF8ECF8DCF8CCF8BCF8ACF89CF88CF87CF86CF85CF84CF83CF82CF81CF80CF96
:200300007FCF7ECF7DCF7CCF7BCF7ACF79CF78CF77CF76CF75CF74CF73CF72CF71CF70CF75
:200320006FCF6ECF6DCF6CCF6BCF6ACF69CF68CF67CF66CF65CF64CF63CF62CF61CF60CF55
:200340005FCF5ECF5DCF5CCF5BCF5ACF59CF58CF57CF56CF55CF54CF53CF52CF51CF50CF35
:200360004FCF4ECF4DCF4CCF4BCF4ACF49CF48CF47CF46CF45CF44CF43CF42CF41CF40CF15
:200380003FCF3ECF3DCF3CCF3BCF3ACF39CF38CF37CF36CF35CF34CF33CF32CF31CF30CFF5
:2003A0002FCF2ECF2DCF2CCF2BCF2ACF29CF28CF27CF26CF25CF24CF23CF22CF21CF20CFD5
:2003C0001FCF1ECF1DCF1CCF1BCF1ACF19CF18CF17CF16CF15CF14CF13CF12CF11CF10CFB5
:2003E0000FCF0ECF0DCF0CCF0BCF0ACF09CF08CF07CF06CF05CF04CF03CF02CF01CF00CF95
:20040000FFCFFECFFDCFFCCFFBCFFACFF9CFF8CFF7CFF6CFF5CFF4CFF3CFF2CFF1CFF0CF74
:20042000EFCFEECFEDCFECCFEBCFEACFE9CFE8CFE7CFE6CFE5CFE4CFE3CFE2CFE1CFE0CF54
:20044000DFCFDECFDDCFDCCFDBCFDACFD9CFD8CFD7CFD6CFD5CFD4CFD3CFD2CFD1CFD0CF34
:20046000CFCFCECFCDCFCCCFCBCFCACFC9CFC8CFC7CFC6CFC5CFC4CFC3CFC2CFC1CFC0CF14
:20048000BFCFBECFBDCFBCCFBBCFBACFB9CFB8CFB7CFB6CFB5CFB4CFB3CFB2CFB1CFB0CFF4
:2004A000AFCFAECFADCFACCFABCFAACFA9CFA8CFA7CFA6CFA5CFA4CFA3CFA2CFA1CFA0CFD4
:2004C0009FCF9ECF9DCF9CCF9BCF9ACF99CF98CF97CF96CF95CF94CF93CF92CF91CF90CFB4
:2004E0008FCF8ECF8DCF8CCF8BCF8ACF89CF88CF87CF86CF85CF84CF83CF82CF81CF80CF94
:200500007FCF7ECF7DCF7CCF7BCF7ACF79CF78CF77CF76CF75CF74CF73CF72CF71CF70CF73
:200520006FCF6ECF6DCF6CCF6BCF6ACF69CF68CF67CF66CF65CF64CF63CF62CF61CF60CF53
:200540005FCF5ECF5DCF5CCF5BCF5ACF59CF58CF57CF56CF55CF54CF53CF52CF51CF50CF33
:200560004FCF4ECF4DCF4CCF4BCF4ACF49CF48CF47CF46CF45CF44CF43CF42CF41CF40CF13
:200580003FCF3ECF3DCF3CCF3BCF3ACF39CF38CF37CF36CF35CF34CF33CF32CF31CF30CFF3
:2005A0002FCF2ECF2DCF2CCF2BCF2ACF29CF28CF27CF26CF25CF24CF23CF22CF21CF20CFD3
:2005C0001FCF1ECF1DCF1CCF1BCF1ACF19CF18CF17CF16CF15CF14CF13CF12CF11CF10CFB3
:2005E0000FCF0ECF0DCF0CCF0BCF0ACF09CF08CF07CF06CF05CF04CF03CF02CF01CF00CF93
:20060000FFCFFECFFDCFFCCFFBCFFACFF9CFF8CFF7CFF6CFF5CFF4CFF3CFF2CFF1CFF0CF72
:20062000EFCFEECFEDCFECCFEBCFEACFE9CFE8CFE7CFE6CFE5CFE4CFE3CFE2CFE1CFE0CF52
:20064000DFCFDECFDDCFDCCFDBCFDACFD9CFD8CFD7CFD6CFD5CFD4CFD3CFD2CFD1CFD0CF32
:20066000CFCFCECFCDCFCCCFCBCFCACFC9CFC8CFC7CFC6CFC5CFC4CFC3CFC2CFC1CFC0CF12
:20068000BFCFBECFBDCFBCCFBBCFBACFB9CFB8CFB7CFB6CFB5CFB4CFB3CFB2CFB1CFB0CFF2
:2006A000AFCFAECFADCFACCFABCFAACFA9CFA8CFA7CFA6CFA5CFA4CFA3CFA2CFA1CFA0CFD2
:2006C0009FCF9ECF9DCF9CCF9BCF9ACF99CF98CF97CF96CF95CF94CF93CF92CF91CF90CFB2
:2006E0008FCF8ECF8DCF8CCF8BCF8ACF89CF88CF87CF86CF85CF84CF83CF82CF81CF80CF92
:200700007FCF7ECF7DCF7CCF7BCF7ACF79CF78CF77CF76CF75CF74CF73CF72CF71CF70CF71
:200720006FCF6ECF6DCF6CCF6BCF6ACF69CF68CF67CF66CF65CF64CF63CF62CF61CF60CF51
:200740005FCF5ECF5DCF5CCF5BCF5ACF59CF58CF57CF56CF55CF54CF53CF52CF51CF50CF31
:200760004FCF4ECF4DCF4CCF4BCF4ACF49CF48CF47CF46CF45CF44CF43CF42CF41CF40CF11
:200780003FCF3ECF3DCF3CCF3BCF3ACF39CF38CF37CF36CF35CF34CF33CF32CF31CF30CFF1
:2007A0002FCF2ECF2DCF2CCF2BCF2ACF29CF28CF27CF26CF25CF24CF23CF22CF21CF20CFD1
:2007C0001FCF1ECF1DCF1CCF1BCF1ACF19CF18CF17CF16CF15CF14CF13CF12CF11CF10CFB1
:2007E0000FCF0ECF0DCF0CCF0BCF0ACF09CF08CF07CF06CF05CF04CF03CF02CF01CF00CF91
:20080000FFCFFECFFDCFFCCFFBCFFACFF9CFF8CFF7CFF6CFF5CFF4CFF3CFF2CFF1CFF0CF70
:20082000EFCFEECFEDCFECCFEBCFEACFE9CFE8CFE7CFE6CFE5CFE4CFE3CFE2CFE1CFE0CF50
:20084000DFCFDECFDDCFDCCFDBCFDACFD9CFD8CFD7CFD6CFD5CFD4CFD3CFD2CFD1CFD0CF30
:20086000CFCFCECFCDCFCCCFCBCFCACFC9CFC8CFC7CFC6CFC5CFC4CFC3CFC2CFC1CFC0CF10
:20088000BFCFBECFBDCFBCCFBBCFBACFB9CFB8CFB7CFB6CFB5CFB4CFB3CFB2CFB1CFB0CFF0
:2008A000AFCFAECFADCFACCFABCFAACFA9CFA8CFA7CFA6CFA5CFA4CFA3CFA2CFA1CFA0CFD0
:2008C0009FCF9ECF9DCF9CCF9BCF9ACF99CF98CF97CF96CF95CF94CF93CF92CF91CF90CFB0
:2008E0008FCF8ECF8DCF8CCF8BCF8ACF89CF88CF87CF86CF85CF84CF83CF82CF81CF80CF90
:200900007FCF7ECF7DCF7CCF7BCF7ACF79CF78CF77CF76CF75CF74CF73CF72CF71CF70CF6F
:200920006FCF6ECF6DCF6CCF6BCF6ACF69CF68CF67CF66CF65CF64CF63CF62CF61CF60CF4F
:200940005FCF5ECF5DCF5CCF5BCF5ACF59CF58CF57CF56CF55CF54CF53CF52CF51CF50CF2F
:200960004FCF4ECF4DCF4CCF4BCF4ACF49CF48CF47CF46CF45CF44CF43CF42CF41CF40CF0F
:200980003FCF3ECF3DCF3CCF3BCF3ACF39CF38CF37CF36CF35CF34CF33CF32CF31CF30CFEF
:2009A0002FCF2ECF2DCF2CCF2BCF2ACF29CF28CF27CF26CF25CF24CF23CF22CF21CF20CFCF
:2009C0001FCF1ECF1DCF1CCF1BCF1ACF19CF18CF17CF16CF15CF14CF13CF12CF11CF10CFAF
:2009E0000FCF0ECF0DCF0CCF0BCF0ACF09CF08CF07CF06CF05CF04CF03CF02CF01CF00CF8F
:200A0000FFCFFECFFDCFFCCFFBCFFACFF9CFF8CFF7CFF6CFF5CFF4CFF3CFF2CFF1CFF0CF6E
:200A2000EFCFEECFEDCFECCFEBCFEACFE9CFE8CFE7CFE6CFE5CFE4CFE3CFE2CFE1CFE0CF4E
:200A4000DFCFDECFDDCFDCCFDBCFDACFD9CFD8CFD7CFD6CFD5CFD4CFD3CFD2CFD1CFD0CF2E
:200A6000CFCFCECFCDCFCCCFCBCFCACFC9CFC8CFC7CFC6CFC5CFC4CFC3CFC2CFC1CFC0CF0E
:200A8000BFCFBECFBDCFBCCFBBCFBACFB9CFB8CFB7CFB6CFB5CFB4CFB3CFB2CFB1CFB0CFEE
:200AA000AFCFAECFADCFACCFABCFAACFA9CFA8CFA7CFA6CFA5CFA4CFA3CFA2CFA1CFA0CFCE
:200AC0009FCF9ECF9DCF9CCF9BCF9ACF99CF98CF97CF96CF95CF94CF93CF92CF91CF90CFAE
:200AE0008FCF8ECF8DCF8CCF8BCF8ACF89CF88CF87CF86CF85CF84CF83CF82CF81CF80CF8E
:200B00007FCF7ECF7DCF7CCF7BCF7ACF79CF78CF77CF76CF75CF74CF73CF72CF71CF70CF6D
:200B20006FCF6ECF6DCF6CCF6BCF6ACF69CF68CF67CF66CF65CF64CF63CF62CF61CF60CF4D
:200B40005FCF5ECF5DCF5CCF5BCF5ACF59CF58CF57CF56CF55CF54CF53CF52CF51CF50CF2D
:200B60004FCF4ECF4DCF4CCF4BCF4ACF49CF48CF47CF46CF45CF44CF43CF42CF41CF40CF0D
:200B80003FCF3ECF3DCF3CCF3BCF3ACF39CF38CF37CF36CF35CF34CF33CF32CF31CF30CFED
:200BA0002FCF2ECF2DCF2CCF2BCF2ACF29CF28CF27CF26CF25CF24CF23CF22CF21CF20CFCD
:200BC0001FCF1ECF1DCF1CCF1BCF1ACF19CF18CF17CF16CF15CF14CF13CF12CF11CF10CFAD
:200BE0000FCF0ECF0DCF0CCF0BCF0ACF09CF08CF07CF06CF05CF04CF03CF02CF01CF00CF8D
:200C0000FFCFFECFFDCFFCCFFBCFFACFF9CFF8CFF7CFF6CFF5CFF4CFF3CFF2CFF1CFF0CF6C
:200C2000EFCFEECFEDCFECCFEBCFEACFE9CFE8CFE7CFE6CFE5CFE4CFE3CFE2CFE1CFE0CF4C
:200C4000DFCFDECFDDCFDCCFDBCFDACFD9CFD8CFD7CFD6CFD5CFD4CFD3CFD2CFD1CFD0CF2C
:200C6000CFCFCECFCDCFCCCFCBCFCACFC9CFC8CFC7CFC6CFC5CFC4CFC3CFC2CFC1CFC0CF0C
:200C8000BFCFBECFBDCFBCCFBBCFBACFB9CFB8CFB7CFB6CFB5CFB4CFB3CFB2CFB1CFB0CFEC
:200CA000AFCFAECFADCFACCFABCFAACFA9CFA8CFA7CFA6CFA5CFA4CFA3CFA2CFA1CFA0CFCC
:200CC0009FCF9ECF9DCF9CCF9BCF9ACF99CF98CF97CF96CF95CF94CF93CF92CF91CF90CFAC
:200CE0008FCF8ECF8DCF8CCF8BCF8ACF89CF88CF87CF86CF85CF84CF83CF82CF81CF80CF8C
:200D00007FCF7ECF7DCF7CCF7BCF7ACF79CF78CF77CF76CF75CF74CF73CF72CF71CF70CF6B
:200D20006FCF6ECF6DCF6CCF6BCF6ACF69CF68CF67CF66CF65CF64CF63CF62CF61CF60CF4B
:200D40005FCF5ECF5DCF5CCF5BCF5ACF59CF58CF57CF56CF55CF54CF53CF52CF51CF50CF2B
:200D60004FCF4ECF4DCF4CCF4BCF4ACF49CF48CF47CF46CF45CF44CF43CF42CF41CF40CF0B
:200D80003FCF3ECF3DCF3CCF3BCF3ACF39CF38CF37CF36CF35CF34CF33CF32CF31CF30CFEB
:200DA0002FCF2ECF2DCF2CCF2BCF2ACF29CF28CF27CF26CF25CF24CF23CF22CF21CF20CFCB
:200DC0001FCF1ECF1DCF1CCF1BCF1ACF19CF18CF17CF16CF15CF14CF13CF12CF11CF10CFAB
:200DE0000FCF0ECF0DCF0CCF0BCF0ACF09CF08CF07CF06CF05CF04CF03CF02CF01CF00CF8B
:200E0000FFCFFECFFDCFFCCFFBCFFACFF9CFF8CFF7CFF6CFF5CFF4CFF3CFF2CFF1CFF0CF6A
:200E2000EFCFEECFEDCFECCFEBCFEACFE9CFE8CFE7CFE6CFE5CFE4CFE3CFE2CFE1CFE0CF4A
:200E4000DFCFDECFDDCFDCCFDBCFDACFD9CFD8CFD7CFD6CFD5CFD4CFD3CFD2CFD1CFD0CF2A
:200E6000CFCFCECFCDCFCCCFCBCFCACFC9CFC8CFC7CFC6CFC5CFC4CFC3CFC2CFC1CFC0CF0A
:200E8000BFCFBECFBDCFBCCFBBCFBACFB9CFB8CFB7CFB6CFB5CFB4CFB3CFB2CFB1CFB0CFEA
:200EA000AFCFAECFADCFACCFABCFAACFA9CFA8CFA7CFA6CFA5CFA4CFA3CFA2CFA1CFA0CFCA
:200EC0009FCF9ECF9DCF9CCF9BCF9ACF99CF98CF97CF96CF95CF94CF93CF92CF91CF90CFAA
:200EE0008FCF8ECF8DCF8CCF8BCF8ACF89CF88CF87CF86CF85CF84CF83CF82CF81CF80CF8A
:200F00007FCF7ECF7DCF7CCF7BCF7ACF79CF78CF77CF76CF75CF74CF73CF72CF71CF70CF69
:200F20006FCF6ECF6DCF6CCF6BCF6ACF69CF68CF67CF66CF65CF64CF63CF62CF61CF60CF49
:200F40005FCF5ECF5DCF5CCF5BCF5ACF59CF58CF57CF56CF55CF54CF53CF52CF51CF50CF29
:200F60004FCF4ECF4DCF4CCF4BCF4ACF49CF48CF47CF46CF45CF44CF43CF42CF41CF40CF09
:200F80003FCF3ECF3DCF3CCF3BCF3ACF39CF38CF37CF36CF35CF34CF33CF32CF31CF30CFE9
:200FA0002FCF2ECF2DCF2CCF2BCF2ACF29CF28CF27CF26CF25CF24CF23CF22CF21CF20CFC9
:200FC0001FCF1ECF1DCF1CCF1BCF1ACF19CF18CF17CF16CF15CF14CF13CF12CF11CF10CFA9
:200FE0000FCF0ECF0DCF0CCF0BCF0ACF09CF08CF07CF06CF05CF04CF03CF02CF01CF00CF89
:20100000FFCFFECFFDCFFCCFFBCFFACFF9CFF8CFF7CFF6CFF5CFF4CFF3CFF2CFF1CFF0CF68
:20102000EFCFEECFEDCFECCFEBCFEACFE9CFE8CFE7CFE6CFE5CFE4CFE3CFE2CFE1CFE0CF48
:20104000DFCFDECFDDCFDCCFDBCFDACFD9CFD8CFD7CFD6CFD5CFD4CFD3CFD2CFD1CFD0CF28
:20106000CFCFCECFCDCFCCCFCBCFCACFC9CFC8CFC7CFC6CFC5CFC4CFC3CFC2CFC1CFC0CF08
:20108000BFCFBECFBDCFBCCFBBCFBACFB9CFB8CFB7CFB6CFB5CFB4CFB3CFB2CFB1CFB0CFE8
:2010A000AFCFAECFADCFACCFABCFAACFA9CFA8CFA7CFA6CFA5CFA4CFA3CFA2CFA1CFA0CFC8
:2010C0009FCF9ECF9DCF9CCF9BCF9ACF99CF98CF97CF96CF95CF94CF93CF92CF91CF90CFA8
:2010E0008FCF8ECF8DCF8CCF8BCF8ACF89CF88CF87CF86CF85CF84CF83CF82CF81CF80CF88
:201100007FCF7ECF7DCF7CCF7BCF7ACF79CF78CF77CF76CF75CF74CF73CF72CF71CF70CF67
:201120006FCF6ECF6DCF6CCF6BCF6ACF69CF68CF67CF66CF65CF64CF63CF62CF61CF60CF47
:201140005FCF5ECF5DCF5CCF5BCF5ACF59CF58CF57CF56CF55CF54CF53CF52CF51CF50CF27
:201160004FCF4ECF4DCF4CCF4BCF4ACF49CF48CF47CF46CF45CF44CF43CF42CF41CF40CF07
:201180003FCF3ECF3DCF3CCF3BCF3ACF39CF38CF37CF36CF35CF34CF33CF32CF31CF30CFE7
:2011A0002FCF2ECF2DCF2CCF2BCF2ACF29CF28CF27CF26CF25CF24CF23CF22CF21CF20CFC7
:2011C0001FCF1ECF1DCF1CCF1BCF1ACF19CF18CF17CF16CF15CF14CF13CF12CF11CF10CFA7
:2011E0000FCF0ECF0DCF0CCF0BCF0ACF09CF08CF07CF06CF05CF04CF03CF02CF01CF00CF87
:20120000FFCFFECFFDCFFCCFFBCFFACFF9CFF8CFF7CFF6CFF5CFF4CFF3CFF2CFF1CFF0CF66
:20122000EFCFEECFEDCFECCFEBCFEACFE9CFE8CFE7CFE6CFE5CFE4CFE3CFE2CFE1CFE0CF46
:20124000DFCFDECFDDCFDCCFDBCFDACFD9CFD8CFD7CFD6CFD5CFD4CFD3CFD2CFD1CFD0CF26
:20126000CFCFCECFCDCFCCCFCBCFCACFC9CFC8CFC7CFC6CFC5CFC4CFC3CFC2CFC1CFC0CF06
:20128000BFCFBECFBDCFBCCFBBCFBACFB9CFB8CFB7CFB6CFB5CFB4CFB3CFB2CFB1CFB0CFE6
:2012A000AFCFAECFADCFACCFABCFAACFA9CFA8CFA7CFA6CFA5CFA4CFA3CFA2CFA1CFA0CFC6
:2012C0009FCF9ECF9DCF9CCF9BCF9ACF99CF98CF97CF96CF95CF94CF93CF92CF91CF90CFA6
:2012E0008FCF8ECF8DCF8CCF8BCF8ACF89CF88CF87CF86CF85CF84CF83CF82CF81CF80CF86
:201300007FCF7ECF7DCF7CCF7BCF7ACF79CF78CF77CF76CF75CF74CF73CF72CF71CF70CF65
:201320006FCF6ECF6DCF6CCF6BCF6ACF69CF68CF67CF66CF65CF64CF63CF62CF61CF60CF45
:201340005FCF5ECF5DCF5CCF5BCF5ACF59CF58CF57CF56CF55CF54CF53CF52CF51CF50CF25
:201360004FCF4ECF4DCF4CCF4BCF4ACF49CF48CF47CF46CF45CF44CF43CF42CF41CF40CF05
:201380003FCF3ECF3DCF3CCF3BCF3ACF39CF38CF37CF36CF35CF34CF33CF32CF31CF30CFE5
:2013A0002FCF2ECF2DCF2CCF2BCF2ACF29CF28CF27CF26CF25CF24CF23CF22CF21CF20CFC5
:2013C0001FCF1ECF1DCF1CCF1BCF1ACF19CF18CF17CF16CF15CF14CF13CF12CF11CF10CFA5
:2013E0000FCF0ECF0DCF0CCF0BCF0ACF09CF08CF07CF06CF05CF04CF03CF02CF01CF00CF85
:20140000FFCFFECFFDCFFCCFFBCFFACFF9CFF8CFF7CFF6CFF5CFF4CFF3CFF2CFF1CFF0CF64
:20142000EFCFEECFEDCFECCFEBCFEACFE9CFE8CFE7CFE6CFE5CFE4CFE3CFE2CFE1CFE0CF44
:20144000DFCFDECFDDCFDCCFDBCFDACFD9CFD8CFD7CFD6CFD5CFD4CFD3CFD2CFD1CFD0CF24
:20146000CFCFCECFCDCFCCCFCBCFCACFC9CFC8CFC7CFC6CFC5CFC4CFC3CFC2CFC1CFC0CF04
:20148000BFCFBECFBDCFBCCFBBCFBACFB9CFB8CFB7CFB6CFB5CFB4CFB3CFB2CFB1CFB0CFE4
:2014A000AFCFAECFADCFACCFABCFAACFA9CFA8CFA7CFA6CFA5CFA4CFA3CFA2CFA1CFA0CFC4
:2014C0009FCF9ECF9DCF9CCF9BCF9ACF99CF98CF97CF96CF95CF94CF93CF92CF91CF90CFA4
:2014E0008FCF8ECF8DCF8CCF8BCF8ACF89CF88CF87CF86CF85CF84CF83CF82CF81CF80CF84
:201500007FCF7ECF7DCF7CCF7BCF7ACF79CF78CF77CF76CF75CF74CF73CF72CF71CF70CF63
:201520006FCF6ECF6DCF6CCF6BCF6ACF69CF68CF67CF66CF65CF64CF63CF62CF61CF60CF43
:201540005FCF5ECF5DCF5CCF5BCF5ACF59CF58CF57CF56CF55CF54CF53CF52CF51CF50CF23
:201560004FCF4ECF4DCF4CCF4BCF4ACF49CF48CF47CF46CF45CF44CF43CF42CF41CF40CF03
:201580003FCF3ECF3DCF3CCF3BCF3ACF39CF38CF37CF36CF35CF34CF33CF32CF31CF30CFE3
:2015A0002FCF2ECF2DCF2CCF2BCF2ACF29CF28CF27CF26CF25CF24CF23CF22CF21CF20CFC3
:2015C0001FCF1ECF1DCF1CCF1BCF1ACF19CF18CF17CF16CF15CF14CF13CF12CF11CF10CFA3
:2015E0000FCF0ECF0DCF0CCF0BCF0ACF09CF08CF07CF06CF05CF04CF03CF02CF01CF00CF83
:20160000FFCFFECFFDCFFCCFFBCFFACFF9CFF8CFF7CFF6CFF5CFF4CFF3CFF2CFF1CFF0CF62
:20162000EFCFEECFEDCFECCFEBCFEACFE9CFE8CFE7CFE6CFE5CFE4CFE3CFE2CFE1CFE0CF42
:20164000DFCFDECFDDCFDCCFDBCFDACFD9CFD8CFD7CFD6CFD5CFD4CFD3CFD2CFD1CFD0CF22
:20166000CFCFCECFCDCFCCCFCBCFCACFC9CFC8CFC7CFC6CFC5CFC4CFC3CFC2CFC1CFC0CF02
:20168000BFCFBECFBDCFBCCFBBCFBACFB9CFB8CFB7CFB6CFB5CFB4CFB3CFB2CFB1CFB0CFE2
:2016A000AFCFAECFADCFACCFABCFAACFA9CFA8CFA7CFA6CFA5CFA4CFA3CFA2CFA1CFA0CFC2
:2016C0009FCF9ECF9DCF9CCF9BCF9ACF99CF98CF97CF96CF95CF94CF93CF92CF91CF90CFA2
:2016E0008FCF8ECF8DCF8CCF8BCF8ACF89CF88CF87CF86CF85CF84CF83CF82CF81CF80CF82
:201700007FCF7ECF7DCF7CCF7BCF7ACF79CF78CF77CF76CF75CF74CF73CF72CF71CF70CF61
:201720006FCF6ECF6DCF6CCF6BCF6ACF69CF68CF67CF66CF65CF64CF63CF62CF61CF60CF41
:201740005FCF5ECF5DCF5CCF5BCF5ACF59CF58CF57CF56CF55CF54CF53CF52CF51CF50CF21
:201760004FCF4ECF4DCF4CCF4BCF4ACF49CF48CF47CF46CF45CF44CF43CF42CF41CF40CF01
:201780003FCF3ECF3DCF3CCF3BCF3ACF39CF38CF37CF36CF35CF34CF33CF32CF31CF30CFE1
:2017A0002FCF2ECF2DCF2CCF2BCF2ACF29CF28CF27CF26CF25CF24CF23CF22CF21CF20CFC1
:2017C0001FCF1ECF1DCF1CCF1BCF1ACF19CF18CF17CF16CF15CF14CF13CF12CF11CF10CFA1
:2017E0000FCF0ECF0DCF0CCF0BCF0ACF09CF08CF07CF06CF05CF04CF03CF02CF01CF00CF81
:20180000FFCFFECFFDCFFCCFFBCFFACFF9CFF8CFF7CFF6CFF5CFF4CFF3CFF2CFF1CFF0CF60
:20182000EFCFEECFEDCFECCFEBCFEACFE9CFE8CFE7CFE6CFE5CFE4CFE3CFE2CFE1CFE0CF40
:20184000DFCFDECFDDCFDCCFDBCFDACFD9CFD8CFD7CFD6CFD5CFD4CFD3CFD2CFD1CFD0CF20
:20186000CFCFCECFCDCFCCCFCBCFCACFC9CFC8CFC7CFC6CFC5CFC4CFC3CFC2CFC1CFC0CF00
:20188000BFCFBECFBDCFBCCFBBCFBACFB9CFB8CFB7CFB6CFB5CFB4CFB3CFB2CFB1CFB0CFE0
:2018A000AFCFAECFADCFACCFABCFAACFA9CFA8CFA7CFA6CFA5CFA4CFA3CFA2CFA1CFA0CFC0
:2018C0009FCF9ECF9DCF9CCF9BCF9ACF99CF98CF97CF96CF95CF94CF93CF92CF91CF90CFA0
:2018E0008FCF8ECF8DCF8CCF8BCF8ACF89CF88CF87CF86CF85CF84CF83CF82CF81CF80CF80
:201900007FCF7ECF7DCF7CCF7BCF7ACF79CF78CF77CF76CF75CF74CF73CF72CF71CF70CF5F
:201920006FCF6ECF6DCF6CCF6BCF6ACF69CF68CF67CF66CF65CF64CF63CF62CF61CF60CF3F
:201940005FCF5ECF5DCF5CCF5BCF5ACF59CF58CF57CF56CF55CF54CF53CF52CF51CF50CF1F
:201960004FCF4ECF4DCF4CCF4BCF4ACF49CF48CF47CF46CF45CF44CF43CF42CF41CF40CFFF
:201980003FCF3ECF3DCF3CCF3BCF3ACF39CF38CF37CF36CF35CF34CF33CF32CF31CF30CFDF
:2019A0002FCF2ECF2DCF2CCF2BCF2ACF29CF28CF27CF26CF25CF24CF23CF22CF21CF20CFBF
:2019C0001FCF1ECF1DCF1CCF1BCF1ACF19CF18CF17CF16CF15CF14CF13CF12CF11CF10CF9F
:2019E0000FCF0ECF0DCF0CCF0BCF0ACF09CF08CF07CF06CF05CF04CF03CF02CF01CF00CF7F
:201A0000FFCFFECFFDCFFCCFFBCFFACFF9CFF8CFF7CFF6CFF5CFF4CFF3CFF2CFF1CFF0CF5E
:201A2000EFCFEECFEDCFECCFEBCFEACFE9CFE8CFE7CFE6CFE5CFE4CFE3CFE2CFE1CFE0CF3E
:201A4000DFCFDECFDDCFDCCFDBCFDACFD9CFD8CFD7CFD6CFD5CFD4CFD3CFD2CFD1CFD0CF1E
:201A6000CFCFCECFCDCFCCCFCBCFCACFC9CFC8CFC7CFC6CFC5CFC4CFC3CFC2CFC1CFC0CFFE
:201A8000BFCFBECFBDCFBCCFBBCFBACFB9CFB8CFB7CFB6CFB5CFB4CFB3CFB2CFB1CFB0CFDE
:201AA000AFCFAECFADCFACCFABCFAACFA9CFA8CFA7CFA6CFA5CFA4CFA3CFA2CFA1CFA0CFBE
:201AC0009FCF9ECF9DCF9CCF9BCF9ACF99CF98CF97CF96CF95CF94CF93CF92CF91CF90CF9E
:201AE0008FCF8ECF8DCF8CCF8BCF8ACF89CF88CF87CF86CF85CF84CF83CF82CF81CF80CF7E
:201B00007FCF7ECF7DCF7CCF7BCF7ACF79CF78CF77CF76CF75CF74CF73CF72CF71CF70CF5D
:201B20006FCF6ECF6DCF6CCF6BCF6ACF69CF68CF67CF66CF65CF64CF63CF62CF61CF60CF3D
:201B40005FCF5ECF5DCF5CCF5BCF5ACF59CF58CF57CF56CF55CF54CF53CF52CF51CF50CF1D
:201B60004FCF4ECF4DCF4CCF4BCF4ACF49CF48CF47CF46CF45CF44CF43CF42CF41CF40CFFD
:201B80003FCF3ECF3DCF3CCF3BCF3ACF39CF38CF37CF36CF35CF34CF33CF32CF31CF30CFDD
:201BA0002FCF2ECF2DCF2CCF2BCF2ACF29CF28CF27CF26CF25CF24CF23CF22CF21CF20CFBD
:201BC0001FCF1ECF1DCF1CCF1BCF1ACF19CF18CF17CF16CF15CF14CF13CF12CF11CF10CF9D
:201BE0000FCF0ECF0DCF0CCF0BCF0ACF09CF08CF07CF06CF05CF04CF03CF02CF01CF00CF7D
:201C0000FFCFFECFFDCFFCCFFBCFFACFF9CFF8CFF7CFF6CFF5CFF4CFF3CFF2CFF1CFF0CF5C
:201C2000EFCFEECFEDCFECCFEBCFEACFE9CFE8CFE7CFE6CFE5CFE4CFE3CFE2CFE1CFE0CF3C
:201C4000DFCFDECFDDCFDCCFDBCFDACFD9CFD8CFD7CFD6CFD5CFD4CFD3CFD2CFD1CFD0CF1C
:201C6000CFCFCECFCDCFCCCFCBCFCACFC9CFC8CFC7CFC6CFC5CFC4CFC3CFC2CFC1CFC0CFFC
:201C8000BFCFBECFBDCFBCCFBBCFBACFB9CFB8CFB7CFB6CFB5CFB4CFB3CFB2CFB1CFB0CFDC
:201CA000AFCFAECFADCFACCFABCFAACFA9CFA8CFA7CFA6CFA5CFA4CFA3CFA2CFA1CFA0CFBC
:201CC0009FCF9ECF9DCF9CCF9BCF9ACF99CF98CF97CF96CF95CF94CF93CF92CF91CF90CF9C
:201CE0008FCF8ECF8DCF8CCF8BCF8ACF89CF88CF87CF86CF85CF84CF83CF82CF81CF80CF7C
:201D00007FCF7ECF7DCF7CCF7BCF7ACF79CF78CF77CF76CF75CF74CF73CF72CF71CF70CF5B
:201D20006FCF6ECF6DCF6CCF6BCF6ACF69CF68CF67CF66CF65CF64CF63CF62CF61CF60CF3B
:201D40005FCF5ECF5DCF5CCF5BCF5ACF59CF58CF57CF56CF55CF54CF53CF52CF51CF50CF1B
:201D60004FCF4ECF4DCF4CCF4BCF4ACF49CF48CF47CF46CF45CF44CF43CF42CF41CF40CFFB
:201D80003FCF3ECF3DCF3CCF3BCF3ACF39CF38CF37CF36CF35CF34CF33CF32CF31CF30CFDB
:201DA0002FCF2ECF2DCF2CCF2BCF2ACF29CF28CF27CF26CF25CF24CF23CF22CF21CF20CFBB
:201DC0001FCF1ECF1DCF1CCF1BCF1ACF19CF18CF17CF16CF15CF14CF13CF12CF11CF10CF9B
:201DE0000FCF0ECF0DCF0CCF0BCF0ACF09CF08CF07CF06CF05CF04CF03CF02CF01CF00CF7B
:201E0000FFCFFECFFDCFFCCFFBCFFACFF9CFF8CFF7CFF6CFF5CFF4CFF3CFF2CFF1CFF0CF5A
:201E2000EFCFEECFEDCFECCFEBCFEACFE9CFE8CFE7CFE6CFE5CFE4CFE3CFE2CFE1CFE0CF3A
:201E4000DFCFDECFDDCFDCCFDBCFDACFD9CFD8CFD7CFD6CFD5CFD4CFD3CFD2CFD1CFD0CF1A
:201E6000CFCFCECFCDCFCCCFCBCFCACFC9CFC8CFC7CFC6CFC5CFC4CFC3CFC2CFC1CFC0CFFA
:201E8000BFCFBECFBDCFBCCFBBCFBACFB9CFB8CFB7CFB6CFB5CFB4CFB3CFB2CFB1CFB0CFDA
:201EA000AFCFAECFADCFACCFABCFAACFA9CFA8CFA7CFA6CFA5CFA4CFA3CFA2CFA1CFA0CFBA
:201EC0009FCF9ECF9DCF9CCF9BCF9ACF99CF98CF97CF96CF95CF94CF93CF92CF91CF90CF9A
:201EE0008FCF8ECF8DCF8CCF8BCF8ACF89CF88CF87CF86CF85CF84CF83CF82CF81CF80CF7A
:201F00007FCF7ECF7DCF7CCF7BCF7ACF79CF78CF77CF76CF75CF74CF73CF72CF71CF70CF59
:201F20006FCF6ECF6DCF6CCF6BCF6ACF69CF68CF67CF66CF65CF64CF63CF62CF61CF60CF39
:201F40005FCF5ECF5DCF5CCF5BCF5ACF59CF58CF57CF56CF55CF54CF53CF52CF51CF50CF19
:201F60004FCF4ECF4DCF4CCF4BCF4ACF49CF48CF47CF46CF45CF44CF43CF42CF41CF40CFF9
:201F80003FCF3ECF3DCF3CCF3BCF3ACF39CF38CF37CF36CF35CF34CF33CF32CF31CF30CFD9
:201FA0002FCF2ECF2DCF2CCF2BCF2ACF29CF28CF27CF26CF25CF24CF23CF22CF21CF20CFB9
:201FC0001FCF1ECF1DCF1CCF1BCF1ACF19CF18CF17CF16CF15CF14CF13CF12CF11CF10CF99
:201FE0000FCF0ECF0DCF0CCF0BCF0ACF09CF08CF07CF06CF05CF04CF03CF02CF01CF00CF79
:20200000FFCFFECFFDCFFCCFFBCFFACFF9CFF8CFF7CFF6CFF5CFF4CFF3CFF2CFF1CFF0CF58
:20202000EFCFEECFEDCFECCFEBCFEACFE9CFE8CFE7CFE6CFE5CFE4CFE3CFE2CFE1CFE0CF38
:20204000DFCFDECFDDCFDCCFDBCFDACFD9CFD8CFD7CFD6CFD5CFD4CFD3CFD2CFD1CFD0CF18
:20206000CFCFCECFCDCFCCCFCBCFCACFC9CFC8CFC7CFC6CFC5CFC4CFC3CFC2CFC1CFC0CFF8
:20208000BFCFBECFBDCFBCCFBBCFBACFB9CFB8CFB7CFB6CFB5CFB4CFB3CFB2CFB1CFB0CFD8
:2020A000AFCFAECFADCFACCFABCFAACFA9CFA8CFA7CFA6CFA5CFA4CFA3CFA2CFA1CFA0CFB8
:2020C0009FCF9ECF9DCF9CCF9BCF9ACF99CF98CF97CF96CF95CF94CF93CF92CF91CF90CF98
:2020E0008FCF8ECF8DCF8CCF8BCF8ACF89CF88CF87CF86CF85CF84CF83CF82CF81CF80CF78
:202100007FCF7ECF7DCF7CCF7BCF7ACF79CF78CF77CF76CF75CF74CF73CF72CF71CF70CF57
:202120006FCF6ECF6DCF6CCF6BCF6ACF69CF68CF67CF66CF65CF64CF63CF62CF61CF60CF37
:202140005FCF5ECF5DCF5CCF5BCF5ACF59CF58CF57CF56CF55CF54CF53CF52CF51CF50CF17
:202160004FCF4ECF4DCF4CCF4BCF4ACF49CF48CF47CF46CF45CF44CF43CF42CF41CF40CFF7
:202180003FCF3ECF3DCF3CCF3BCF3ACF39CF38CF37CF36CF35CF34CF33CF32CF31CF30CFD7
:2021A0002FCF2ECF2DCF2CCF2BCF2ACF29CF28CF27CF26CF25CF24CF23CF22CF21CF20CFB7
:2021C0001FCF1ECF1DCF1CCF1BCF1ACF19CF18CF17CF16CF15CF14CF13CF12CF11CF10CF97
:2021E0000FCF0ECF0DCF0CCF0BCF0ACF09CF08CF07CF06CF05CF04CF03CF02CF01CF00CF77
:20220000FFCFFECFFDCFFCCFFBCFFACFF9CFF8CFF7CFF6CFF5CFF4CFF3CFF2CFF1CFF0CF56
:20222000EFCFEECFEDCFECCFEBCFEACFE9CFE8CFE7CFE6CFE5CFE4CFE3CFE2CFE1CFE0CF36
:20224000DFCFDECFDDCFDCCFDBCFDACFD9CFD8CFD7CFD6CFD5CFD4CFD3CFD2CFD1CFD0CF16
:20226000CFCFCECFCDCFCCCFCBCFCACFC9CFC8CFC7CFC6CFC5CFC4CFC3CFC2CFC1CFC0CFF6
:20228000BFCFBECFBDCFBCCFBBCFBACFB9CFB8CFB7CFB6CFB5CFB4CFB3CFB2CFB1CFB0CFD6
:2022A000AFCFAECFADCFACCFABCFAACFA9CFA8CFA7CFA6CFA5CFA4CFA3CFA2CFA1CFA0CFB6
:2022C0009FCF9ECF9DCF9CCF9BCF9ACF99CF98CF97CF96CF95CF94CF93CF92CF91CF90CF96
:2022E0008FCF8ECF8DCF8CCF8BCF8ACF89CF88CF87CF86CF85CF84CF83CF82CF81CF80CF76
:202300007FCF7ECF7DCF7CCF7BCF7ACF79CF78CF77CF76CF75CF74CF73CF72CF71CF70CF55
:202320006FCF6ECF6DCF6CCF6BCF6ACF69CF68CF67CF66CF65CF64CF63CF62CF61CF60CF35
:202340005FCF5ECF5DCF5CCF5BCF5ACF59CF58CF57CF56CF55CF54CF53CF52CF51CF50CF15
:202360004FCF4ECF4DCF4CCF4BCF4ACF49CF48CF47CF46CF45CF44CF43CF42CF41CF40CFF5
:202380003FCF3ECF3DCF3CCF3BCF3ACF39CF38CF37CF36CF35CF34CF33CF32CF31CF30CFD5
:2023A0002FCF2ECF2DCF2CCF2BCF2ACF29CF28CF27CF26CF25CF24CF23CF22CF21CF20CFB5
:2023C0001FCF1ECF1DCF1CCF1BCF1ACF19CF18CF17CF16CF15CF14CF13CF12CF11CF10CF95
:2023E0000FCF0ECF0DCF0CCF0BCF0ACF09CF08CF07CF06CF05CF04CF03CF02CF01CF00CF75
:20240000FFCFFECFFDCFFCCFFBCFFACFF9CFF8CFF7CFF6CFF5CFF4CFF3CFF2CFF1CFF0CF54
:20242000EFCFEECFEDCFECCFEBCFEACFE9CFE8CFE7CFE6CFE5CFE4CFE3CFE2CFE1CFE0CF34
:20244000DFCFDECFDDCFDCCFDBCFDACFD9CFD8CFD7CFD6CFD5CFD4CFD3CFD2CFD1CFD0CF14
:20246000CFCFCECFCDCFCCCFCBCFCACFC9CFC8CFC7CFC6CFC5CFC4CFC3CFC2CFC1CFC0CFF4
:20248000BFCFBECFBDCFBCCFBBCFBACFB9CFB8CFB7CFB6CFB5CFB4CFB3CFB2CFB1CFB0CFD4
:2024A000AFCFAECFADCFACCFABCFAACFA9CFA8CFA7CFA6CFA5CFA4CFA3CFA2CFA1CFA0CFB4
:2024C0009FCF9ECF9DCF9CCF9BCF9ACF99CF98CF97CF96CF95CF94CF93CF92CF91CF90CF94
:2024E0008FCF8ECF8DCF8CCF8BCF8ACF89CF88CF87CF86CF85CF84CF83CF82CF81CF80CF74
:202500007FCF7ECF7DCF7CCF7BCF7ACF79CF78CF77CF76CF75CF74CF73CF72CF71CF70CF53
:202520006FCF6ECF6DCF6CCF6BCF6ACF69CF68CF67CF66CF65CF64CF63CF62CF61CF60CF33
:202540005FCF5ECF5DCF5CCF5BCF5ACF59CF58CF57CF56CF55CF54CF53CF52CF51CF50CF13
:202560004FCF4ECF4DCF4CCF4BCF4ACF49CF48CF47CF46CF45CF44CF43CF42CF41CF40CFF3
:202580003FCF3ECF3DCF3CCF3BCF3ACF39CF38CF37CF36CF35CF34CF33CF32CF31CF30CFD3
:2025A0002FCF2ECF2DCF2CCF2BCF2ACF29CF28CF27CF26CF25CF24CF23CF22CF21CF20CFB3
:2025C0001FCF1ECF1DCF1CCF1BCF1ACF19CF18CF17CF16CF15CF14CF13CF12CF11CF10CF93
:2025E0000FCF0ECF0DCF0CCF0BCF0ACF09CF08CF07CF06CF05CF04CF03CF02CF01CF00CF73
:20260000FFCFFECFFDCFFCCFFBCFFACFF9CFF8CFF7CFF6CFF5CFF4CFF3CFF2CFF1CFF0CF52
:20262000EFCFEECFEDCFECCFEBCFEACFE9CFE8CFE7CFE6CFE5CFE4CFE3CFE2CFE1CFE0CF32
:20264000DFCFDECFDDCFDCCFDBCFDACFD9CFD8CFD7CFD6CFD5CFD4CFD3CFD2CFD1CFD0CF12
:20266000CFCFCECFCDCFCCCFCBCFCACFC9CFC8CFC7CFC6CFC5CFC4CFC3CFC2CFC1CFC0CFF2
:20268000BFCFBECFBDCFBCCFBBCFBACFB9CFB8CFB7CFB6CFB5CFB4CFB3CFB2CFB1CFB0CFD2
:2026A000AFCFAECFADCFACCFABCFAACFA9CFA8CFA7CFA6CFA5CFA4CFA3CFA2CFA1CFA0CFB2
:2026C0009FCF9ECF9DCF9CCF9BCF9ACF99CF98CF97CF96CF95CF94CF93CF92CF91CF90CF92
:2026E0008FCF8ECF8DCF8CCF8BCF8ACF89CF88CF87CF86CF85CF84CF83CF82CF81CF80CF72
:202700007FCF7ECF7DCF7CCF7BCF7ACF79CF78CF77CF76CF75CF74CF73CF72CF71CF70CF51
:202720006FCF6ECF6DCF6CCF6BCF6ACF69CF68CF67CF66CF65CF64CF63CF62CF61CF60CF31
:202740005FCF5ECF5DCF5CCF5BCF5ACF59CF58CF57CF56CF55CF54CF53CF52CF51CF50CF11
:202760004FCF4ECF4DCF4CCF4BCF4ACF49CF48CF47CF46CF45CF44CF43CF42CF41CF40CFF1
:202780003FCF3ECF3DCF3CCF3BCF3ACF39CF38CF37CF36CF35CF34CF33CF32CF31CF30CFD1
:2027A0002FCF2ECF2DCF2CCF2BCF2ACF29CF28CF27CF26CF25CF24CF23CF22CF21CF20CFB1
:2027C0001FCF1ECF1DCF1CCF1BCF1ACF19CF18CF17CF16CF15CF14CF13CF12CF11CF10CF91
:2027E0000FCF0ECF0DCF0CCF0BCF0ACF09CF08CF07CF06CF05CF04CF03CF02CF01CF00CF71
:20280000FFCFFECFFDCFFCCFFBCFFACFF9CFF8CFF7CFF6CFF5CFF4CFF3CFF2CFF1CFF0CF50
:20282000EFCFEECFEDCFECCFEBCFEACFE9CFE8CFE7CFE6CFE5CFE4CFE3CFE2CFE1CFE0CF30
:20284000DFCFDECFDDCFDCCFDBCFDACFD9CFD8CFD7CFD6CFD5CFD4CFD3CFD2CFD1CFD0CF10
:20286000CFCFCECFCDCFCCCFCBCFCACFC9CFC8CFC7CFC6CFC5CFC4CFC3CFC2CFC1CFC0CFF0
:20288000BFCFBECFBDCFBCCFBBCFBACFB9CFB8CFB7CFB6CFB5CFB4CFB3CFB2CFB1CFB0CFD0
:2028A000AFCFAECFADCFACCFABCFAACFA9CFA8CFA7CFA6CFA5CFA4CFA3CFA2CFA1CFA0CFB0
:2028C0009FCF9ECF9DCF9CCF9BCF9ACF99CF98CF97CF96CF95CF94CF93CF92CF91CF90CF90
:2028E0008FCF8ECF8DCF8CCF8BCF8ACF89CF88CF87CF86CF85CF84CF83CF82CF81CF80CF70
:202900007FCF7ECF7DCF7CCF7BCF7ACF79CF78CF77CF76CF75CF74CF73CF72CF71CF70CF4F
:202920006FCF6ECF6DCF6CCF6BCF6ACF69CF68CF67CF66CF65CF64CF63CF62CF61CF60CF2F
:202940005FCF5ECF5DCF5CCF5BCF5ACF59CF58CF57CF56CF55CF54CF53CF52CF51CF50CF0F
:202960004FCF4ECF4DCF4CCF4BCF4ACF49CF48CF47CF46CF45CF44CF43CF42CF41CF40CFEF
:202980003FCF3ECF3DCF3CCF3BCF3ACF39CF38CF37CF36CF35CF34CF33CF32CF31CF30CFCF
:2029A0002FCF2ECF2DCF2CCF2BCF2ACF29CF28CF27CF26CF25CF24CF23CF22CF21CF20CFAF
:2029C0001FCF1ECF1DCF1CCF1BCF1ACF19CF18CF17CF16CF15CF14CF13CF12CF11CF10CF8F
:2029E0000FCF0ECF0DCF0CCF0BCF0ACF09CF08CF07CF06CF05CF04CF03CF02CF01CF00CF6F
:202A0000FFCFFECFFDCFFCCFFBCFFACFF9CFF8CFF7CFF6CFF5CFF4CFF3CFF2CFF1CFF0CF4E
:202A2000EFCFEECFEDCFECCFEBCFEACFE9CFE8CFE7CFE6CFE5CFE4CFE3CFE2CFE1CFE0CF2E
:202A4000DFCFDECFDDCFDCCFDBCFDACFD9CFD8CFD7CFD6CFD5CFD4CFD3CFD2CFD1CFD0CF0E
:202A6000CFCFCECFCDCFCCCFCBCFCACFC9CFC8CFC7CFC6CFC5CFC4CFC3CFC2CFC1CFC0CFEE
:202A8000BFCFBECFBDCFBCCFBBCFBACFB9CFB8CFB7CFB6CFB5CFB4CFB3CFB2CFB1CFB0CFCE
:202AA000AFCFAECFADCFACCFABCFAACFA9CFA8CFA7CFA6CFA5CFA4CFA3CFA2CFA1CFA0CFAE
:202AC0009FCF9ECF9DCF9CCF9BCF9ACF99CF98CF97CF96CF95CF94CF93CF92CF91CF90CF8E
:202AE0008FCF8ECF8DCF8CCF8BCF8ACF89CF88CF87CF86CF85CF84CF83CF82CF81CF80CF6E
:202B00007FCF7ECF7DCF7CCF7BCF7ACF79CF78CF77CF76CF75CF74CF73CF72CF71CF70CF4D
:202B20006FCF6ECF6DCF6CCF6BCF6ACF69CF68CF67CF66CF65CF64CF63CF62CF61CF60CF2D
:202B40005FCF5ECF5DCF5CCF5BCF5ACF59CF58CF57CF56CF55CF54CF53CF52CF51CF50CF0D
:202B60004FCF4ECF4DCF4CCF4BCF4ACF49CF48CF47CF46CF45CF44CF43CF42CF41CF40CFED
:202B80003FCF3ECF3DCF3CCF3BCF3ACF39CF38CF37CF36CF35CF34CF33CF32CF31CF30CFCD
:202BA0002FCF2ECF2DCF2CCF2BCF2ACF29CF28CF27CF26CF25CF24CF23CF22CF21CF20CFAD
:202BC0001FCF1ECF1DCF1CCF1BCF1ACF19CF18CF17CF16CF15CF14CF13CF12CF11CF10CF8D
:202BE0000FCF0ECF0DCF0CCF0BCF0ACF09CF08CF07CF06CF05CF04CF03CF02CF01CF00CF6D
:202C0000FFCFFECFFDCFFCCFFBCFFACFF9CFF8CFF7CFF6CFF5CFF4CFF3CFF2CFF1CFF0CF4C
:202C2000EFCFEECFEDCFECCFEBCFEACFE9CFE8CFE7CFE6CFE5CFE4CFE3CFE2CFE1CFE0CF2C
:202C4000DFCFDECFDDCFDCCFDBCFDACFD9CFD8CFD7CFD6CFD5CFD4CFD3CFD2CFD1CFD0CF0C
:202C6000CFCFCECFCDCFCCCFCBCFCACFC9CFC8CFC7CFC6CFC5CFC4CFC3CFC2CFC1CFC0CFEC
:202C8000BFCFBECFBDCFBCCFBBCFBACFB9CFB8CFB7CFB6CFB5CFB4CFB3CFB2CFB1CFB0CFCC
:202CA000AFCFAECFADCFACCFABCFAACFA9CFA8CFA7CFA6CFA5CFA4CFA3CFA2CFA1CFA0CFAC
:202CC0009FCF9ECF9DCF9CCF9BCF9ACF99CF98CF97CF96CF95CF94CF93CF92CF91CF90CF8C
:202CE0008FCF8ECF8DCF8CCF8BCF8ACF89CF88CF87CF86CF85CF84CF83CF82CF81CF80CF6C
:202D00007FCF7ECF7DCF7CCF7BCF7ACF79CF78CF77CF76CF75CF74CF73CF72CF71CF70CF4B
:202D20006FCF6ECF6DCF6CCF6BCF6ACF69CF68CF67CF66CF65CF64CF63CF62CF61CF60CF2B
:202D40005FCF5ECF5DCF5CCF5BCF5ACF59CF58CF57CF56CF55CF54CF53CF52CF51CF50CF0B
:202D60004FCF4ECF4DCF4CCF4BCF4ACF49CF48CF47CF46CF45CF44CF43CF42CF41CF40CFEB
:202D80003FCF3ECF3DCF3CCF3BCF3ACF39CF38CF37CF36CF35CF34CF33CF32CF31CF30CFCB
:202DA0002FCF2ECF2DCF2CCF2BCF2ACF29CF28CF27CF26CF25CF24CF23CF22CF21CF20CFAB
:202DC0001FCF1ECF1DCF1CCF1BCF1ACF19CF18CF17CF16CF15CF14CF13CF12CF11CF10CF8B
:202DE0000FCF0ECF0DCF0CCF0BCF0ACF09CF08CF07CF06CF05CF04CF03CF02CF01CF00CF6B
:202E0000FFCFFECFFDCFFCCFFBCFFACFF9CFF8CFF7CFF6CFF5CFF4CFF3CFF2CFF1CFF0CF4A
:202E2000EFCFEECFEDCFECCFEBCFEACFE9CFE8CFE7CFE6CFE5CFE4CFE3CFE2CFE1CFE0CF2A
:202E4000DFCFDECFDDCFDCCFDBCFDACFD9CFD8CFD7CFD6CFD5CFD4CFD3CFD2CFD1CFD0CF0A
:202E6000CFCFCECFCDCFCCCFCBCFCACFC9CFC8CFC7CFC6CFC5CFC4CFC3CFC2CFC1CFC0CFEA
:202E8000BFCFBECFBDCFBCCFBBCFBACFB9CFB8CFB7CFB6CFB5CFB4CFB3CFB2CFB1CFB0CFCA
:202EA000AFCFAECFADCFACCFABCFAACFA9CFA8CFA7CFA6CFA5CFA4CFA3CFA2CFA1CFA0CFAA
:202EC0009FCF9ECF9DCF9CCF9BCF9ACF99CF98CF97CF96CF95CF94CF93CF92CF91CF90CF8A
:202EE0008FCF8ECF8DCF8CCF8BCF8ACF89CF88CF87CF86CF85CF84CF83CF82CF81CF80CF6A
:202F00007FCF7ECF7DCF7CCF7BCF7ACF79CF78CF77CF76CF75CF74CF73CF72CF71CF70CF49
:202F20006FCF6ECF6DCF6CCF6BCF6ACF69CF68CF67CF66CF65CF64CF63CF62CF61CF60CF29
:202F40005FCF5ECF5DCF5CCF5BCF5ACF59CF58CF57CF56CF55CF54CF53CF52CF51CF50CF09
:202F60004FCF4ECF4DCF4CCF4BCF4ACF49CF48CF47CF46CF45CF44CF43CF42CF41CF40CFE9
:202F80003FCF3ECF3DCF3CCF3BCF3ACF39CF38CF37CF36CF35CF34CF33CF32CF31CF30CFC9
:202FA0002FCF2ECF2DCF2CCF2BCF2ACF29CF28CF27CF26CF25CF24CF23CF22CF21CF20CFA9
:202FC0001FCF1ECF1DCF1CCF1BCF1ACF19CF18CF17CF16CF15CF14CF13CF12CF11CF10CF89
:202FE0000FCF0ECF0DCF0CCF0BCF0ACF09CF08CF07CF06CF05CF04CF03CF02CF01CF00CF69
:20300000FFCFFECFFDCFFCCFFBCFFACFF9CFF8CFF7CFF6CFF5CFF4CFF3CFF2CFF1CFF0CF48
:20302000EFCFEECFEDCFECCFEBCFEACFE9CFE8CFE7CFE6CFE5CFE4CFE3CFE2CFE1CFE0CF28
:20304000DFCFDECFDDCFDCCFDBCFDACFD9CFD8CFD7CFD6CFD5CFD4CFD3CFD2CFD1CFD0CF08
:20306000CFCFCECFCDCFCCCFCBCFCACFC9CFC8CFC7CFC6CFC5CFC4CFC3CFC2CFC1CFC0CFE8
:20308000BFCFBECFBDCFBCCFBBCFBACFB9CFB8CFB7CFB6CFB5CFB4CFB3CFB2CFB1CFB0CFC8
:2030A000AFCFAECFADCFACCFABCFAACFA9CFA8CFA7CFA6CFA5CFA4CFA3CFA2CFA1CFA0CFA8
:2030C0009FCF9ECF9DCF9CCF9BCF9ACF99CF98CF97CF96CF95CF94CF93CF92CF91CF90CF88
:2030E0008FCF8ECF8DCF8CCF8BCF8ACF89CF88CF87CF86CF85CF84CF83CF82CF81CF80CF68
:203100007FCF7ECF7DCF7CCF7BCF7ACF79CF78CF77CF76CF75CF74CF73CF72CF71CF70CF47
:203120006FCF6ECF6DCF6CCF6BCF6ACF69CF68CF67CF66CF65CF64CF63CF62CF61CF60CF27
:203140005FCF5ECF5DCF5CCF5BCF5ACF59CF58CF57CF56CF55CF54CF53CF52CF51CF50CF07
:203160004FCF4ECF4DCF4CCF4BCF4ACF49CF48CF47CF46CF45CF44CF43CF42CF41CF40CFE7
:203180003FCF3ECF3DCF3CCF3BCF3ACF39CF38CF37CF36CF35CF34CF33CF32CF31CF30CFC7
:2031A0002FCF2ECF2DCF2CCF2BCF2ACF29CF28CF27CF26CF25CF24CF23CF22CF21CF20CFA7
:2031C0001FCF1ECF1DCF1CCF1BCF1ACF19CF18CF17CF16CF15CF14CF13CF12CF11CF10CF87
:2031E0000FCF0ECF0DCF0CCF0BCF0ACF09CF08CF07CF06CF05CF04CF03CF02CF01CF00CF67
:20320000FFCFFECFFDCFFCCFFBCFFACFF9CFF8CFF7CFF6CFF5CFF4CFF3CFF2CFF1CFF0CF46
:20322000EFCFEECFEDCFECCFEBCFEACFE9CFE8CFE7CFE6CFE5CFE4CFE3CFE2CFE1CFE0CF26
:20324000DFCFDECFDDCFDCCFDBCFDACFD9CFD8CFD7CFD6CFD5CFD4CFD3CFD2CFD1CFD0CF06
:20326000CFCFCECFCDCFCCCFCBCFCACFC9CFC8CFC7CFC6CFC5CFC4CFC3CFC2CFC1CFC0CFE6
:20328000BFCFBECFBDCFBCCFBBCFBACFB9CFB8CFB7CFB6CFB5CFB4CFB3CFB2CFB1CFB0CFC6
:2032A000AFCFAECFADCFACCFABCFAACFA9CFA8CFA7CFA6CFA5CFA4CFA3CFA2CFA1CFA0CFA6
:2032C0009FCF9ECF9DCF9CCF9BCF9ACF99CF98CF97CF96CF95CF94CF93CF92CF91CF90CF86
:2032E0008FCF8ECF8DCF8CCF8BCF8ACF89CF88CF87CF86CF85CF84CF83CF82CF81CF80CF66
:203300007FCF7ECF7DCF7CCF7BCF7ACF79CF78CF77CF76CF75CF74CF73CF72CF71CF70CF45
:203320006FCF6ECF6DCF6CCF6BCF6ACF69CF68CF67CF66CF65CF64CF63CF62CF61CF60CF25
:203340005FCF5ECF5DCF5CCF5BCF5ACF59CF58CF57CF56CF55CF54CF53CF52CF51CF50CF05
:203360004FCF4ECF4DCF4CCF4BCF4ACF49CF48CF47CF46CF45CF44CF43CF42CF41CF40CFE5
:203380003FCF3ECF3DCF3CCF3BCF3ACF39CF38CF37CF36CF35CF34CF33CF32CF31CF30CFC5
:2033A0002FCF2ECF2DCF2CCF2BCF2ACF29CF28CF27CF26CF25CF24CF23CF22CF21CF20CFA5
:2033C0001FCF1ECF1DCF1CCF1BCF1ACF19CF18CF17CF16CF15CF14CF13CF12CF11CF10CF85
:2033E0000FCF0ECF0DCF0CCF0BCF0ACF09CF08CF07CF06CF05CF04CF03CF02CF01CF00CF65
:20340000FFCFFECFFDCFFCCFFBCFFACFF9CFF8CFF7CFF6CFF5CFF4CFF3CFF2CFF1CFF0CF44
:20342000EFCFEECFEDCFECCFEBCFEACFE9CFE8CFE7CFE6CFE5CFE4CFE3CFE2CFE1CFE0CF24
:20344000DFCFDECFDDCFDCCFDBCFDACFD9CFD8CFD7CFD6CFD5CFD4CFD3CFD2CFD1CFD0CF04
:20346000CFCFCECFCDCFCCCFCBCFCACFC9CFC8CFC7CFC6CFC5CFC4CFC3CFC2CFC1CFC0CFE4
:20348000BFCFBECFBDCFBCCFBBCFBACFB9CFB8CFB7CFB6CFB5CFB4CFB3CFB2CFB1CFB0CFC4
:2034A000AFCFAECFADCFACCFABCFAACFA9CFA8CFA7CFA6CFA5CFA4CFA3CFA2CFA1CFA0CFA4
:2034C0009FCF9ECF9DCF9CCF9BCF9ACF99CF98CF97CF96CF95CF94CF93CF92CF91CF90CF84
:2034E0008FCF8ECF8DCF8CCF8BCF8ACF89CF88CF87CF86CF85CF84CF83CF82CF81CF80CF64
:203500007FCF7ECF7DCF7CCF7BCF7ACF79CF78CF77CF76CF75CF74CF73CF72CF71CF70CF43
:203520006FCF6ECF6DCF6CCF6BCF6ACF69CF68CF67CF66CF65CF64CF63CF62CF61CF60CF23
:203540005FCF5ECF5DCF5CCF5BCF5ACF59CF58CF57CF56CF55CF54CF53CF52CF51CF50CF03
:203560004FCF4ECF4DCF4CCF4BCF4ACF49CF48CF47CF46CF45CF44CF43CF42CF41CF40CFE3
:203580003FCF3ECF3DCF3CCF3BCF3ACF39CF38CF37CF36CF35CF34CF33CF32CF31CF30CFC3
:2035A0002FCF2ECF2DCF2CCF2BCF2ACF29CF28CF27CF26CF25CF24CF23CF22CF21CF20CFA3
:2035C0001FCF1ECF1DCF1CCF1BCF1ACF19CF18CF17CF16CF15CF14CF13CF12CF11CF10CF83
:2035E0000FCF0ECF0DCF0CCF0BCF0ACF09CF08CF07CF06CF05CF04CF03CF02CF01CF00CF63
:20360000FFCFFECFFDCFFCCFFBCFFACFF9CFF8CFF7CFF6CFF5CFF4CFF3CFF2CFF1CFF0CF42
:20362000EFCFEECFEDCFECCFEBCFEACFE9CFE8CFE7CFE6CFE5CFE4CFE3CFE2CFE1CFE0CF22
:20364000DFCFDECFDDCFDCCFDBCFDACFD9CFD8CFD7CFD6CFD5CFD4CFD3CFD2CFD1CFD0CF02
:20366000CFCFCECFCDCFCCCFCBCFCACFC9CFC8CFC7CFC6CFC5CFC4CFC3CFC2CFC1CFC0CFE2
:20368000BFCFBECFBDCFBCCFBBCFBACFB9CFB8CFB7CFB6CFB5CFB4CFB3CFB2CFB1CFB0CFC2
:2036A000AFCFAECFADCFACCFABCFAACFA9CFA8CFA7CFA6CFA5CFA4CFA3CFA2CFA1CFA0CFA2
:2036C0009FCF9ECF9DCF9CCF9BCF9ACF99CF98CF97CF96CF95CF94CF93CF92CF91CF90CF82
:2036E0008FCF8ECF8DCF8CCF8BCF8ACF89CF88CF87CF86CF85CF84CF83CF82CF81CF80CF62
:203700007FCF7ECF7DCF7CCF7BCF7ACF79CF78CF77CF76CF75CF74CF73CF72CF71CF70CF41
:203720006FCF6ECF6DCF6CCF6BCF6ACF69CF68CF67CF66CF65CF64CF63CF62CF61CF60CF21
:203740005FCF5ECF5DCF5CCF5BCF5ACF59CF58CF57CF56CF55CF54CF53CF52CF51CF50CF01
:203760004FCF4ECF4DCF4CCF4BCF4ACF49CF48CF47CF46CF45CF44CF43CF42CF41CF40CFE1
:203780003FCF3ECF3DCF3CCF3BCF3ACF39CF38CF37CF36CF35CF34CF33CF32CF31CF30CFC1
:2037A0002FCF2ECF2DCF2CCF2BCF2ACF29CF28CF27CF26CF25CF24CF23CF22CF21CF20CFA1
:2037C0001FCF1ECF1DCF1CCF1BCF1ACF19CF18CF17CF16CF15CF14CF13CF12CF11CF10CF81
:2037E0000FCF0ECF0DCF0CCF0BCF0ACF09CF08CF07CF06CF05CF04CF03CF02CF01CF00CF61
:20380000FFCFFECFFDCFFCCFFBCFFACFF9CFF8CFF7CFF6CFF5CFF4CFF3CFF2CFF1CFF0CF40
:20382000EFCFEECFEDCFECCFEBCFEACFE9CFE8CFE7CFE6CFE5CFE4CFE3CFE2CFE1CFE0CF20
:20384000DFCFDECFDDCFDCCFDBCFDACFD9CFD8CFD7CFD6CFD5CFD4CFD3CFD2CFD1CFD0CF00
:20386000CFCFCECFCDCFCCCFCBCFCACFC9CFC8CFC7CFC6CFC5CFC4CFC3CFC2CFC1CFC0CFE0
:20388000BFCFBECFBDCFBCCFBBCFBACFB9CFB8CFB7CFB6CFB5CFB4CFB3CFB2CFB1CFB0CFC0
:2038A000AFCFAECFADCFACCFABCFAACFA9CFA8CFA7CFA6CFA5CFA4CFA3CFA2CFA1CFA0CFA0
:2038C0009FCF9ECF9DCF9CCF9BCF9ACF99CF98CF97CF96CF95CF94CF93CF92CF91CF90CF80
:2038E0008FCF8ECF8DCF8CCF8BCF8ACF89CF88CF87CF86CF85CF84CF83CF82CF81CF80CF60
:203900007FCF7ECF7DCF7CCF7BCF7ACF79CF78CF77CF76CF75CF74CF73CF72CF71CF70CF3F
:203920006FCF6ECF6DCF6CCF6BCF6ACF69CF68CF67CF66CF65CF64CF63CF62CF61CF60CF1F
:203940005FCF5ECF5DCF5CCF5BCF5ACF59CF58CF57CF56CF55CF54CF53CF52CF51CF50CFFF
:203960004FCF4ECF4DCF4CCF4BCF4ACF49CF48CF47CF46CF45CF44CF43CF42CF41CF40CFDF
:203980003FCF3ECF3DCF3CCF3BCF3ACF39CF38CF37CF36CF35CF34CF33CF32CF31CF30CFBF
:2039A0002FCF2ECF2DCF2CCF2BCF2ACF29CF28CF27CF26CF25CF24CF23CF22CF21CF20CF9F
:2039C0001FCF1ECF1DCF1CCF1BCF1ACF19CF18CF17CF16CF15CF14CF13CF12CF11CF10CF7F
:2039E0000FCF0ECF0DCF0CCF0BCF0ACF09CF08CF07CF06CF05CF04CF03CF02CF01CF00CF5F
:203A0000FFCFFECFFDCFFCCFFBCFFACFF9CFF8CFF7CFF6CFF5CFF4CFF3CFF2CFF1CFF0CF3E
:203A2000EFCFEECFEDCFECCFEBCFEACFE9CFE8CFE7CFE6CFE5CFE4CFE3CFE2CFE1CFE0CF1E
:203A4000DFCFDECFDDCFDCCFDBCFDACFD9CFD8CFD7CFD6CFD5CFD4CFD3CFD2CFD1CFD0CFFE
:203A6000CFCFCECFCDCFCCCFCBCFCACFC9CFC8CFC7CFC6CFC5CFC4CFC3CFC2CFC1CFC0CFDE
:203A8000BFCFBECFBDCFBCCFBBCFBACFB9CFB8CFB7CFB6CFB5CFB4CFB3CFB2CFB1CFB0CFBE
:203AA000AFCFAECFADCFACCFABCFAACFA9CFA8CFA7CFA6CFA5CFA4CFA3CFA2CFA1CFA0CF9E
:203AC0009FCF9ECF9DCF9CCF9BCF9ACF99CF98CF97CF96CF95CF94CF93CF92CF91CF90CF7E
:203AE0008FCF8ECF8DCF8CCF8BCF8ACF89CF88CF87CF86CF85CF84CF83CF82CF81CF80CF5E
:203B00007FCF7ECF7DCF7CCF7BCF7ACF79CF78CF77CF76CF75CF74CF73CF72CF71CF70CF3D
:203B20006FCF6ECF6DCF6CCF6BCF6ACF69CF68CF67CF66CF65CF64CF63CF62CF61CF60CF1D
:203B40005FCF5ECF5DCF5CCF5BCF5ACF59CF58CF57CF56CF55CF54CF53CF52CF51CF50CFFD
:203B60004FCF4ECF4DCF4CCF4BCF4ACF49CF48CF47CF46CF45CF44CF43CF42CF41CF40CFDD
:203B80003FCF3ECF3DCF3CCF3BCF3ACF39CF38CF37CF36CF35CF34CF33CF32CF31CF30CFBD
:203BA0002FCF2ECF2DCF2CCF2BCF2ACF29CF28CF27CF26CF25CF24CF23CF22CF21CF20CF9D
:203BC0001FCF1ECF1DCF1CCF1BCF1ACF19CF18CF17CF16CF15CF14CF13CF12CF11CF10CF7D
:203BE0000FCF0ECF0DCF0CCF0BCF0ACF09CF08CF07CF06CF05CF04CF03CF02CF01CF00CF5D
:203C0000FFCFFECFFDCFFCCFFBCFFACFF9CFF8CFF7CFF6CFF5CFF4CFF3CFF2CFF1CFF0CF3C
:203C2000EFCFEECFEDCFECCFEBCFEACFE9CFE8CFE7CFE6CFE5CFE4CFE3CFE2CFE1CFE0CF1C
:203C4000DFCFDECFDDCFDCCFDBCFDACFD9CFD8CFD7CFD6CFD5CFD4CFD3CFD2CFD1CFD0CFFC
:203C6000CFCFCECFCDCFCCCFCBCFCACFC9CFC8CFC7CFC6CFC5CFC4CFC3CFC2CFC1CFC0CFDC
:203C8000BFCFBECFBDCFBCCFBBCFBACFB9CFB8CFB7CFB6CFB5CFB4CFB3CFB2CFB1CFB0CFBC
:203CA000AFCFAECFADCFACCFABCFAACFA9CFA8CFA7CFA6CFA5CFA4CFA3CFA2CFA1CFA0CF9C
:203CC0009FCF9ECF9DCF9CCF9BCF9ACF99CF98CF97CF96CF95CF94CF93CF92CF91CF90CF7C
:203CE0008FCF8ECF8DCF8CCF8BCF8ACF89CF88CF87CF86CF85CF84CF83CF82CF81CF80CF5C
:203D00007FCF7ECF7DCF7CCF7BCF7ACF79CF78CF77CF76CF75CF74CF73CF72CF71CF70CF3B
:203D20006FCF6ECF6DCF6CCF6BCF6ACF69CF68CF67CF66CF65CF64CF63CF62CF61CF60CF1B
:203D40005FCF5ECF5DCF5CCF5BCF5ACF59CF58CF57CF56CF55CF54CF53CF52CF51CF50CFFB
:203D60004FCF4ECF4DCF4CCF4BCF4ACF49CF48CF47CF46CF45CF44CF43CF42CF41CF40CFDB
:203D80003FCF3ECF3DCF3CCF3BCF3ACF39CF38CF37CF36CF35CF34CF33CF32CF31CF30CFBB
:203DA0002FCF2ECF2DCF2CCF2BCF2ACF29CF28CF27CF26CF25CF24CF23CF22CF21CF20CF9B
:203DC0001FCF1ECF1DCF1CCF1BCF1ACF19CF18CF17CF16CF15CF14CF13CF12CF11CF10CF7B
:203DE0000FCF0ECF0DCF0CCF0BCF0ACF09CF08CF07CF06CF05CF04CF03CF02CF01CF00CF5B
:203E0000FFCFFECFFDCFFCCFFBCFFACFF9CFF8CFF7CFF6CFF5CFF4CFF3CFF2CFF1CFF0CF3A
:203E2000EFCFEECFEDCFECCFEBCFEACFE9CFE8CFE7CFE6CFE5CFE4CFE3CFE2CFE1CFE0CF1A
:203E4000DFCFDECFDDCFDCCFDBCFDACFD9CFD8CFD7CFD6CFD5CFD4CFD3CFD2CFD1CFD0CFFA
:203E6000CFCFCECFCDCFCCCFCBCFCACFC9CFC8CFC7CFC6CFC5CFC4CFC3CFC2CFC1CFC0CFDA
:203E8000BFCFBECFBDCFBCCFBBCFBACFB9CFB8CFB7CFB6CFB5CFB4CFB3CFB2CFB1CFB0CFBA
:203EA000AFCFAECFADCFACCFABCFAACFA9CFA8CFA7CFA6CFA5CFA4CFA3CFA2CFA1CFA0CF9A
:203EC0009FCF9ECF9DCF9CCF9BCF9ACF99CF98CF97CF96CF95CF94CF93CF92CF91CF90CF7A
:203EE0008FCF8ECF8DCF8CCF8BCF8ACF89CF88CF87CF86CF85CF84CF83CF82CF81CF80CF5A
:203F00007FCF7ECF7DCF7CCF7BCF7ACF79CF78CF77CF76CF75CF74CF73CF72CF71CF70CF39
:203F20006FCF6ECF6DCF6CCF6BCF6ACF69CF68CF67CF66CF65CF64CF63CF62CF61CF60CF19
:203F40005FCF5ECF5DCF5CCF5BCF5ACF59CF58CF57CF56CF55CF54CF53CF52CF51CF50CFF9
:203F60004FCF4ECF4DCF4CCF4BCF4ACF49CF48CF47CF46CF45CF44CF43CF42CF41CF40CFD9
:203F80003FCF3ECF3DCF3CCF3BCF3ACF39CF38CF37CF36CF35CF34CF33CF32CF31CF30CFB9
:203FA0002FCF2ECF2DCF2CCF2BCF2ACF29CF28CF27CF26CF25CF24CF23CF22CF21CF20CF99
:203FC0001FCF1ECF1DCF1CCF1BCF1ACF19CF18CF17CF16CF15CF14CF13CF12CF11CF10CF79
:203FE0000FCF0ECF0DCF0CCF0BCF0ACF09CF08CF07CF06CF05CF04CF03CF02CF01CF00CF59
:20400000FFCFFECFFDCFFCCFFBCFFACFF9CFF8CFF7CFF6CFF5CFF4CFF3CFF2CFF1CFF0CF38
:20402000EFCFEECFEDCFECCFEBCFEACFE9CFE8CFE7CFE6CFE5CFE4CFE3CFE2CFE1CFE0CF18
:20404000DFCFDECFDDCFDCCFDBCFDACFD9CFD8CFD7CFD6CFD5CFD4CFD3CFD2CFD1CFD0CFF8
:20406000CFCFCECFCDCFCCCFCBCFCACFC9CFC8CFC7CFC6CFC5CFC4CFC3CFC2CFC1CFC0CFD8
:20408000BFCFBECFBDCFBCCFBBCFBACFB9CFB8CFB7CFB6CFB5CFB4CFB3CFB2CFB1CFB0CFB8
:2040A000AFCFAECFADCFACCFABCFAACFA9CFA8CFA7CFA6CFA5CFA4CFA3CFA2CFA1CFA0CF98
:2040C0009FCF9ECF9DCF9CCF9BCF9ACF99CF98CF97CF96CF95CF94CF93CF92CF91CF90CF78
:2040E0008FCF8ECF8DCF8CCF8BCF8ACF89CF88CF87CF86CF85CF84CF83CF82CF81CF80CF58
:204100007FCF7ECF7DCF7CCF7BCF7ACF79CF78CF77CF76CF75CF74CF73CF72CF71CF70CF37
:204120006FCF6ECF6DCF6CCF6BCF6ACF69CF68CF67CF66CF65CF64CF63CF62CF61CF60CF17
:204140005FCF5ECF5DCF5CCF5BCF5ACF59CF58CF57CF56CF55CF54CF53CF52CF51CF50CFF7
:204160004FCF4ECF4DCF4CCF4BCF4ACF49CF48CF47CF46CF45CF44CF43CF42CF41CF40CFD7
:204180003FCF3ECF3DCF3CCF3BCF3ACF39CF38CF37CF36CF35CF34CF33CF32CF31CF30CFB7
:2041A0002FCF2ECF2DCF2CCF2BCF2ACF29CF28CF27CF26CF25CF24CF23CF22CF21CF20CF97
:2041C0001FCF1ECF1DCF1CCF1BCF1ACF19CF18CF17CF16CF15CF14CF13CF12CF11CF10CF77
:2041E0000FCF0ECF0DCF0CCF0BCF0ACF09CF08CF07CF06CF05CF04CF03CF02CF01CF00CF57
:20420000FFCFFECFFDCFFCCFFBCFFACFF9CFF8CFF7CFF6CFF5CFF4CFF3CFF2CFF1CFF0CF36
:20422000EFCFEECFEDCFECCFEBCFEACFE9CFE8CFE7CFE6CFE5CFE4CFE3CFE2CFE1CFE0CF16
:20424000DFCFDECFDDCFDCCFDBCFDACFD9CFD8CFD7CFD6CFD5CFD4CFD3CFD2CFD1CFD0CFF6
:20426000CFCFCECFCDCFCCCFCBCFCACFC9CFC8CFC7CFC6CFC5CFC4CFC3CFC2CFC1CFC0CFD6
:20428000BFCFBECFBDCFBCCFBBCFBACFB9CFB8CFB7CFB6CFB5CFB4CFB3CFB2CFB1CFB0CFB6
:2042A000AFCFAECFADCFACCFABCFAACFA9CFA8CFA7CFA6CFA5CFA4CFA3CFA2CFA1CFA0CF96
:2042C0009FCF9ECF9DCF9CCF9BCF9ACF99CF98CF97CF96CF95CF94CF93CF92CF91CF90CF76
:2042E0008FCF8ECF8DCF8CCF8BCF8ACF89CF88CF87CF86CF85CF84CF83CF82CF81CF80CF56
:204300007FCF7ECF7DCF7CCF7BCF7ACF79CF78CF77CF76CF75CF74CF73CF72CF71CF70CF35
:204320006FCF6ECF6DCF6CCF6BCF6ACF69CF68CF67CF66CF65CF64CF63CF62CF61CF60CF15
:204340005FCF5ECF5DCF5CCF5BCF5ACF59CF58CF57CF56CF55CF54CF53CF52CF51CF50CFF5
:204360004FCF4ECF4DCF4CCF4BCF4ACF49CF48CF47CF46CF45CF44CF43CF42CF41CF40CFD5
:204380003FCF3ECF3DCF3CCF3BCF3ACF39CF38CF37CF36CF35CF34CF33CF32CF31CF30CFB5
:2043A0002FCF2ECF2DCF2CCF2BCF2ACF29CF28CF27CF26CF25CF24CF23CF22CF21CF20CF95
:2043C0001FCF1ECF1DCF1CCF1BCF1ACF19CF18CF17CF16CF15CF14CF13CF12CF11CF10CF75
:2043E0000FCF0ECF0DCF0CCF0BCF0ACF09CF08CF07CF06CF05CF04CF03CF02CF01CF00CF55
:20440000FFCFFECFFDCFFCCFFBCFFACFF9CFF8CFF7CFF6CFF5CFF4CFF3CFF2CFF1CFF0CF34
:20442000EFCFEECFEDCFECCFEBCFEACFE9CFE8CFE7CFE6CFE5CFE4CFE3CFE2CFE1CFE0CF14
:20444000DFCFDECFDDCFDCCFDBCFDACFD9CFD8CFD7CFD6CFD5CFD4CFD3CFD2CFD1CFD0CFF4
:20446000CFCFCECFCDCFCCCFCBCFCACFC9CFC8CFC7CFC6CFC5CFC4CFC3CFC2CFC1CFC0CFD4
:20448000BFCFBECFBDCFBCCFBBCFBACFB9CFB8CFB7CFB6CFB5CFB4CFB3CFB2CFB1CFB0CFB4
:2044A000AFCFAECFADCFACCFABCFAACFA9CFA8CFA7CFA6CFA5CFA4CFA3CFA2CFA1CFA0CF94
:2044C0009FCF9ECF9DCF9CCF9BCF9ACF99CF98CF97CF96CF95CF94CF93CF92CF91CF90CF74
:2044E0008FCF8ECF8DCF8CCF8BCF8ACF89CF88CF87CF86CF85CF84CF83CF82CF81CF80CF54
:204500007FCF7ECF7DCF7CCF7BCF7ACF79CF78CF77CF76CF75CF74CF73CF72CF71CF70CF33
:204520006FCF6ECF6DCF6CCF6BCF6ACF69CF68CF67CF66CF65CF64CF63CF62CF61CF60CF13
:204540005FCF5ECF5DCF5CCF5BCF5ACF59CF58CF57CF56CF55CF54CF53CF52CF51CF50CFF3
:204560004FCF4ECF4DCF4CCF4BCF4ACF49CF48CF47CF46CF45CF44CF43CF42CF41CF40CFD3
:204580003FCF3ECF3DCF3CCF3BCF3ACF39CF38CF37CF36CF35CF34CF33CF32CF31CF30CFB3
:2045A0002FCF2ECF2DCF2CCF2BCF2ACF29CF28CF27CF26CF25CF24CF23CF22CF21CF20CF93
:2045C0001FCF1ECF1DCF1CCF1BCF1ACF19CF18CF17CF16CF15CF14CF13CF12CF11CF10CF73
:2045E0000FCF0ECF0DCF0CCF0BCF0ACF09CF08CF07CF06CF05CF04CF03CF02CF01CF00CF53
:20460000FFCFFECFFDCFFCCFFBCFFACFF9CFF8CFF7CFF6CFF5CFF4CFF3CFF2CFF1CFF0CF32
:20462000EFCFEECFEDCFECCFEBCFEACFE9CFE8CFE7CFE6CFE5CFE4CFE3CFE2CFE1CFE0CF12
:20464000DFCFDECFDDCFDCCFDBCFDACFD9CFD8CFD7CFD6CFD5CFD4CFD3CFD2CFD1CFD0CFF2
:20466000CFCFCECFCDCFCCCFCBCFCACFC9CFC8CFC7CFC6CFC5CFC4CFC3CFC2CFC1CFC0CFD2
:20468000BFCFBECFBDCFBCCFBBCFBACFB9CFB8CFB7CFB6CFB5CFB4CFB3CFB2CFB1CFB0CFB2
:2046A000AFCFAECFADCFACCFABCFAACFA9CFA8CFA7CFA6CFA5CFA4CFA3CFA2CFA1CFA0CF92
:2046C0009FCF9ECF9DCF9CCF9BCF9ACF99CF98CF97CF96CF95CF94CF93CF92CF91CF90CF72
:2046E0008FCF8ECF8DCF8CCF8BCF8ACF89CF88CF87CF86CF85CF84CF83CF82CF81CF80CF52
:204700007FCF7ECF7DCF7CCF7BCF7ACF79CF78CF77CF76CF75CF74CF73CF72CF71CF70CF31
:204720006FCF6ECF6DCF6CCF6BCF6ACF69CF68CF67CF66CF65CF64CF63CF62CF61CF60CF11
:204740005FCF5ECF5DCF5CCF5BCF5ACF59CF58CF57CF56CF55CF54CF53CF52CF51CF50CFF1
:204760004FCF4ECF4DCF4CCF4BCF4ACF49CF48CF47CF46CF45CF44CF43CF42CF41CF40CFD1
:204780003FCF3ECF3DCF3CCF3BCF3ACF39CF38CF37CF36CF35CF34CF33CF32CF31CF30CFB1
:2047A0002FCF2ECF2DCF2CCF2BCF2ACF29CF28CF27CF26CF25CF24CF23CF22CF21CF20CF91
:2047C0001FCF1ECF1DCF1CCF1BCF1ACF19CF18CF17CF16CF15CF14CF13CF12CF11CF10CF71
:2047E0000FCF0ECF0DCF0CCF0BCF0ACF09CF08CF07CF06CF05CF04CF03CF02CF01CF00CF51
:20480000FFCFFECFFDCFFCCFFBCFFACFF9CFF8CFF7CFF6CFF5CFF4CFF3CFF2CFF1CFF0CF30
:20482000EFCFEECFEDCFECCFEBCFEACFE9CFE8CFE7CFE6CFE5CFE4CFE3CFE2CFE1CFE0CF10
:20484000DFCFDECFDDCFDCCFDBCFDACFD9CFD8CFD7CFD6CFD5CFD4CFD3CFD2CFD1CFD0CFF0
:20486000CFCFCECFCDCFCCCFCBCFCACFC9CFC8CFC7CFC6CFC5CFC4CFC3CFC2CFC1CFC0CFD0
:20488000BFCFBECFBDCFBCCFBBCFBACFB9CFB8CFB7CFB6CFB5CFB4CFB3CFB2CFB1CFB0CFB0
:2048A000AFCFAECFADCFACCFABCFAACFA9CFA8CFA7CFA6CFA5CFA4CFA3CFA2CFA1CFA0CF90
:2048C0009FCF9ECF9DCF9CCF9BCF9ACF99CF98CF97CF96CF95CF94CF93CF92CF91CF90CF70
:2048E0008FCF8ECF8DCF8CCF8BCF8ACF89CF88CF87CF86CF85CF84CF83CF82CF81CF80CF50
:204900007FCF7ECF7DCF7CCF7BCF7ACF79CF78CF77CF76CF75CF74CF73CF72CF71CF70CF2F
:204920006FCF6ECF6DCF6CCF6BCF6ACF69CF68CF67CF66CF65CF64CF63CF62CF61CF60CF0F
:204940005FCF5ECF5DCF5CCF5BCF5ACF59CF58CF57CF56CF55CF54CF53CF52CF51CF50CFEF
:204960004FCF4ECF4DCF4CCF4BCF4ACF49CF48CF47CF46CF45CF44CF43CF42CF41CF40CFCF
:204980003FCF3ECF3DCF3CCF3BCF3ACF39CF38CF37CF36CF35CF34CF33CF32CF31CF30CFAF
:2049A0002FCF2ECF2DCF2CCF2BCF2ACF29CF28CF27CF26CF25CF24CF23CF22CF21CF20CF8F
:2049C0001FCF1ECF1DCF1CCF1BCF1ACF19CF18CF17CF16CF15CF14CF13CF12CF11CF10CF6F
:2049E0000FCF0ECF0DCF0CCF0BCF0ACF09CF08CF07CF06CF05CF04CF03CF02CF01CF00CF4F
:204A0000FFCFFECFFDCFFCCFFBCFFACFF9CFF8CFF7CFF6CFF5CFF4CFF3CFF2CFF1CFF0CF2E
:204A2000EFCFEECFEDCFECCFEBCFEACFE9CFE8CFE7CFE6CFE5CFE4CFE3CFE2CFE1CFE0CF0E
:204A4000DFCFDECFDDCFDCCFDBCFDACFD9CFD8CFD7CFD6CFD5CFD4CFD3CFD2CFD1CFD0CFEE
:204A6000CFCFCECFCDCFCCCFCBCFCACFC9CFC8CFC7CFC6CFC5CFC4CFC3CFC2CFC1CFC0CFCE
:204A8000BFCFBECFBDCFBCCFBBCFBACFB9CFB8CFB7CFB6CFB5CFB4CFB3CFB2CFB1CFB0CFAE
:204AA000AFCFAECFADCFACCFABCFAACFA9CFA8CFA7CFA6CFA5CFA4CFA3CFA2CFA1CFA0CF8E
:204AC0009FCF9ECF9DCF9CCF9BCF9ACF99CF98CF97CF96CF95CF94CF93CF92CF91CF90CF6E
:204AE0008FCF8ECF8DCF8CCF8BCF8ACF89CF88CF87CF86CF85CF84CF83CF82CF81CF80CF4E
:204B00007FCF7ECF7DCF7CCF7BCF7ACF79CF78CF77CF76CF75CF74CF73CF72CF71CF70CF2D
:204B20006FCF6ECF6DCF6CCF6BCF6ACF69CF68CF67CF66CF65CF64CF63CF62CF61CF60CF0D
:204B40005FCF5ECF5DCF5CCF5BCF5ACF59CF58CF57CF56CF55CF54CF53CF52CF51CF50CFED
:204B60004FCF4ECF4DCF4CCF4BCF4ACF49CF48CF47CF46CF45CF44CF43CF42CF41CF40CFCD
:204B80003FCF3ECF3DCF3CCF3BCF3ACF39CF38CF37CF36CF35CF34CF33CF32CF31CF30CFAD
:204BA0002FCF2ECF2DCF2CCF2BCF2ACF29CF28CF27CF26CF25CF24CF23CF22CF21CF20CF8D
:204BC0001FCF1ECF1DCF1CCF1BCF1ACF19CF18CF17CF16CF15CF14CF13CF12CF11CF10CF6D
:204BE0000FCF0ECF0DCF0CCF0BCF0ACF09CF08CF07CF06CF05CF04CF03CF02CF01CF00CF4D
:204C0000FFCFFECFFDCFFCCFFBCFFACFF9CFF8CFF7CFF6CFF5CFF4CFF3CFF2CFF1CFF0CF2C
:204C2000EFCFEECFEDCFECCFEBCFEACFE9CFE8CFE7CFE6CFE5CFE4CFE3CFE2CFE1CFE0CF0C
:204C4000DFCFDECFDDCFDCCFDBCFDACFD9CFD8CFD7CFD6CFD5CFD4CFD3CFD2CFD1CFD0CFEC
:204C6000CFCFCECFCDCFCCCFCBCFCACFC9CFC8CFC7CFC6CFC5CFC4CFC3CFC2CFC1CFC0CFCC
:204C8000BFCFBECFBDCFBCCFBBCFBACFB9CFB8CFB7CFB6CFB5CFB4CFB3CFB2CFB1CFB0CFAC
:204CA000AFCFAECFADCFACCFABCFAACFA9CFA8CFA7CFA6CFA5CFA4CFA3CFA2CFA1CFA0CF8C
:204CC0009FCF9ECF9DCF9CCF9BCF9ACF99CF98CF97CF96CF95CF94CF93CF92CF91CF90CF6C
:204CE0008FCF8ECF8DCF8CCF8BCF8ACF89CF88CF87CF86CF85CF84CF83CF82CF81CF80CF4C
:204D00007FCF7ECF7DCF7CCF7BCF7ACF79CF78CF77CF76CF75CF74CF73CF72CF71CF70CF2B
:204D20006FCF6ECF6DCF6CCF6BCF6ACF69CF68CF67CF66CF65CF64CF63CF62CF61CF60CF0B
:204D40005FCF5ECF5DCF5CCF5BCF5ACF59CF58CF57CF56CF55CF54CF53CF52CF51CF50CFEB
:204D60004FCF4ECF4DCF4CCF4BCF4ACF49CF48CF47CF46CF45CF44CF43CF42CF41CF40CFCB
:204D80003FCF3ECF3DCF3CCF3BCF3ACF39CF38CF37CF36CF35CF34CF33CF32CF31CF30CFAB
:204DA0002FCF2ECF2DCF2CCF2BCF2ACF29CF28CF27CF26CF25CF24CF23CF22CF21CF20CF8B
:204DC0001FCF1ECF1DCF1CCF1BCF1ACF19CF18CF17CF16CF15CF14CF13CF12CF11CF10CF6B
:204DE0000FCF0ECF0DCF0CCF0BCF0ACF09CF08CF07CF06CF05CF04CF03CF02CF01CF00CF4B
:204E0000FFCFFECFFDCFFCCFFBCFFACFF9CFF8CFF7CFF6CFF5CFF4CFF3CFF2CFF1CFF0CF2A
:204E2000EFCFEECFEDCFECCFEBCFEACFE9CFE8CFE7CFE6CFE5CFE4CFE3CFE2CFE1CFE0CF0A
:204E4000DFCFDECFDDCFDCCFDBCFDACFD9CFD8CFD7CFD6CFD5CFD4CFD3CFD2CFD1CFD0CFEA
:204E6000CFCFCECFCDCFCCCFCBCFCACFC9CFC8CFC7CFC6CFC5CFC4CFC3CFC2CFC1CFC0CFCA
:204E8000BFCFBECFBDCFBCCFBBCFBACFB9CFB8CFB7CFB6CFB5CFB4CFB3CFB2CFB1CFB0CFAA
:204EA000AFCFAECFADCFACCFABCFAACFA9CFA8CFA7CFA6CFA5CFA4CFA3CFA2CFA1CFA0CF8A
:204EC0009FCF9ECF9DCF9CCF9BCF9ACF99CF98CF97CF96CF95CF94CF93CF92CF91CF90CF6A
:204EE0008FCF8ECF8DCF8CCF8BCF8ACF89CF88CF87CF86CF85CF84CF83CF82CF81CF80CF4A
:204F00007FCF7ECF7DCF7CCF7BCF7ACF79CF78CF77CF76CF75CF74CF73CF72CF71CF70CF29
:204F20006FCF6ECF6DCF6CCF6BCF6ACF69CF68CF67CF66CF65CF64CF63CF62CF61CF60CF09
:204F40005FCF5ECF5DCF5CCF5BCF5ACF59CF58CF57CF56CF55CF54CF53CF52CF51CF50CFE9
:204F60004FCF4ECF4DCF4CCF4BCF4ACF49CF48CF47CF46CF45CF44CF43CF42CF41CF40CFC9
:204F80003FCF3ECF3DCF3CCF3BCF3ACF39CF38CF37CF36CF35CF34CF33CF32CF31CF30CFA9
:204FA0002FCF2ECF2DCF2CCF2BCF2ACF29CF28CF27CF26CF25CF24CF23CF22CF21CF20CF89
:204FC0001FCF1ECF1DCF1CCF1BCF1ACF19CF18CF17CF16CF15CF14CF13CF12CF11CF10CF69
:204FE0000FCF0ECF0DCF0CCF0BCF0ACF09CF08CF07CF06CF05CF04CF03CF02CF01CF00CF49
:20500000FFCFFECFFDCFFCCFFBCFFACFF9CFF8CFF7CFF6CFF5CFF4CFF3CFF2CFF1CFF0CF28
:20502000EFCFEECFEDCFECCFEBCFEACFE9CFE8CFE7CFE6CFE5CFE4CFE3CFE2CFE1CFE0CF08
:20504000DFCFDECFDDCFDCCFDBCFDACFD9CFD8CFD7CFD6CFD5CFD4CFD3CFD2CFD1CFD0CFE8
:20506000CFCFCECFCDCFCCCFCBCFCACFC9CFC8CFC7CFC6CFC5CFC4CFC3CFC2CFC1CFC0CFC8
:20508000BFCFBECFBDCFBCCFBBCFBACFB9CFB8CFB7CFB6CFB5CFB4CFB3CFB2CFB1CFB0CFA8
:2050A000AFCFAECFADCFACCFABCFAACFA9CFA8CFA7CFA6CFA5CFA4CFA3CFA2CFA1CFA0CF88
:2050C0009FCF9ECF9DCF9CCF9BCF9ACF99CF98CF97CF96CF95CF94CF93CF92CF91CF90CF68
:2050E0008FCF8ECF8DCF8CCF8BCF8ACF89CF88CF87CF86CF85CF84CF83CF82CF81CF80CF48
:205100007FCF7ECF7DCF7CCF7BCF7ACF79CF78CF77CF76CF75CF74CF73CF72CF71CF70CF27
:205120006FCF6ECF6DCF6CCF6BCF6ACF69CF68CF67CF66CF65CF64CF63CF62CF61CF60CF07
:205140005FCF5ECF5DCF5CCF5BCF5ACF59CF58CF57CF56CF55CF54CF53CF52CF51CF50CFE7
:205160004FCF4ECF4DCF4CCF4BCF4ACF49CF48CF47CF46CF45CF44CF43CF42CF41CF40CFC7
:205180003FCF3ECF3DCF3CCF3BCF3ACF39CF38CF37CF36CF35CF34CF33CF32CF31CF30CFA7
:2051A0002FCF2ECF2DCF2CCF2BCF2ACF29CF28CF27CF26CF25CF24CF23CF22CF21CF20CF87
:2051C0001FCF1ECF1DCF1CCF1BCF1ACF19CF18CF17CF16CF15CF14CF13CF12CF11CF10CF67
:2051E0000FCF0ECF0DCF0CCF0BCF0ACF09CF08CF07CF06CF05CF04CF03CF02CF01CF00CF47
:20520000FFCFFECFFDCFFCCFFBCFFACFF9CFF8CFF7CFF6CFF5CFF4CFF3CFF2CFF1CFF0CF26
:20522000EFCFEECFEDCFECCFEBCFEACFE9CFE8CFE7CFE6CFE5CFE4CFE3CFE2CFE1CFE0CF06
:20524000DFCFDECFDDCFDCCFDBCFDACFD9CFD8CFD7CFD6CFD5CFD4CFD3CFD2CFD1CFD0CFE6
:20526000CFCFCECFCDCFCCCFCBCFCACFC9CFC8CFC7CFC6CFC5CFC4CFC3CFC2CFC1CFC0CFC6
:20528000BFCFBECFBDCFBCCFBBCFBACFB9CFB8CFB7CFB6CFB5CFB4CFB3CFB2CFB1CFB0CFA6
:2052A000AFCFAECFADCFACCFABCFAACFA9CFA8CFA7CFA6CFA5CFA4CFA3CFA2CFA1CFA0CF86
:2052C0009FCF9ECF9DCF9CCF9BCF9ACF99CF98CF97CF96CF95CF94CF93CF92CF91CF90CF66
:2052E0008FCF8ECF8DCF8CCF8BCF8ACF89CF88CF87CF86CF85CF84CF83CF82CF81CF80CF46
:205300007FCF7ECF7DCF7CCF7BCF7ACF79CF78CF77CF76CF75CF74CF73CF72CF71CF70CF25
:205320006FCF6ECF6DCF6CCF6BCF6ACF69CF68CF67CF66CF65CF64CF63CF62CF61CF60CF05
:205340005FCF5ECF5DCF5CCF5BCF5ACF59CF58CF57CF56CF55CF54CF53CF52CF51CF50CFE5
:205360004FCF4ECF4DCF4CCF4BCF4ACF49CF48CF47CF46CF45CF44CF43CF42CF41CF40CFC5
:205380003FCF3ECF3DCF3CCF3BCF3ACF39CF38CF37CF36CF35CF34CF33CF32CF31CF30CFA5
:2053A0002FCF2ECF2DCF2CCF2BCF2ACF29CF28CF27CF26CF25CF24CF23CF22CF21CF20CF85
:2053C0001FCF1ECF1DCF1CCF1BCF1ACF19CF18CF17CF16CF15CF14CF13CF12CF11CF10CF65
:2053E0000FCF0ECF0DCF0CCF0BCF0ACF09CF08CF07CF06CF05CF04CF03CF02CF01CF00CF45
:20540000FFCFFECFFDCFFCCFFBCFFACFF9CFF8CFF7CFF6CFF5CFF4CFF3CFF2CFF1CFF0CF24
:20542000EFCFEECFEDCFECCFEBCFEACFE9CFE8CFE7CFE6CFE5CFE4CFE3CFE2CFE1CFE0CF04
:20544000DFCFDECFDDCFDCCFDBCFDACFD9CFD8CFD7CFD6CFD5CFD4CFD3CFD2CFD1CFD0CFE4
:20546000CFCFCECFCDCFCCCFCBCFCACFC9CFC8CFC7CFC6CFC5CFC4CFC3CFC2CFC1CFC0CFC4
:20548000BFCFBECFBDCFBCCFBBCFBACFB9CFB8CFB7CFB6CFB5CFB4CFB3CFB2CFB1CFB0CFA4
:2054A000AFCFAECFADCFACCFABCFAACFA9CFA8CFA7CFA6CFA5CFA4CFA3CFA2CFA1CFA0CF84
:2054C0009FCF9ECF9DCF9CCF9BCF9ACF99CF98CF97CF96CF95CF94CF93CF92CF91CF90CF64
:2054E0008FCF8ECF8DCF8CCF8BCF8ACF89CF88CF87CF86CF85CF84CF83CF82CF81CF80CF44
:205500007FCF7ECF7DCF7CCF7BCF7ACF79CF78CF77CF76CF75CF74CF73CF72CF71CF70CF23
:205520006FCF6ECF6DCF6CCF6BCF6ACF69CF68CF67CF66CF65CF64CF63CF62CF61CF60CF03
:155540005FCF5ECF5DCF5CCF5BCF5ACF59CF58CF57CF56CF5562
:020000040002F8
:20AAAB00FFCFFECFFDCFFCCFFBCFFACFF9CFF8CFF7CFF6CFF5CFF4CFF3CFF2CFF1CFF0CF23
:20AACB00EFCFEECFEDCFECCFEBCFEACFE9CFE8CFE7CFE6CFE5CFE4CFE3CFE2CFE1CFE0CF03
:20AAEB00DFCFDECFDDCFDCCFDBCFDACFD9CFD8CFD7CFD6CFD5CFD4CFD3CFD2CFD1CFD0CFE3
:20AB0B00CFCFCECFCDCFCCCFCBCFCACFC9CFC8CFC7CFC6CFC5CFC4CFC3CFC2CFC1CFC0CFC2
:20AB2B00BFCFBECFBDCFBCCFBBCFBACFB9CFB8CFB7CFB6CFB5CFB4CFB3CFB2CFB1CFB0CFA2
:20AB4B00AFCFAECFADCFACCFABCFAACFA9CFA8CFA7CFA6CFA5CFA4CFA3CFA2CFA1CFA0CF82
:20AB6B009FCF9ECF9DCF9CCF9BCF9ACF99CF98CF97CF96CF95CF94CF93CF92CF91CF90CF62
:20AB8B008FCF8ECF8DCF8CCF8BCF8ACF89CF88CF87CF86CF85CF84CF83CF82CF81CF80CF42
:20ABAB007FCF7ECF7DCF7CCF7BCF7ACF79CF78CF77CF76CF75CF74CF73CF72CF71CF70CF22
:20ABCB006FCF6ECF6DCF6CCF6BCF6ACF69CF68CF67CF66CF65CF64CF63CF62CF61CF60CF02
:20ABEB005FCF5ECF5DCF5CCF5BCF5ACF59CF58CF57CF56CF55CF54CF53CF52CF51CF50CFE2
:20AC0B004FCF4ECF4DCF4CCF4BCF4ACF49CF48CF47CF46CF45CF44CF43CF42CF41CF40CFC1
:20AC2B003FCF3ECF3DCF3CCF3BCF3ACF39CF38CF37CF36CF35CF34CF33CF32CF31CF30CFA1
:20AC4B002FCF2ECF2DCF2CCF2BCF2ACF29CF28CF27CF26CF25CF24CF23CF22CF21CF20CF81
:20AC6B001FCF1ECF1DCF1CCF1BCF1ACF19CF18CF17CF16CF15CF14CF13CF12CF11CF10CF61
:20AC8B000FCF0ECF0DCF0CCF0BCF0ACF09CF08CF07CF06CF05CF04CF03CF02CF01CF00CF41
:20ACAB00FFCFFECFFDCFFCCFFBCFFACFF9CFF8CFF7CFF6CFF5CFF4CFF3CFF2CFF1CFF0CF21
:20ACCB00EFCFEECFEDCFECCFEBCFEACFE9CFE8CFE7CFE6CFE5CFE4CFE3CFE2CFE1CFE0CF01
:20ACEB00DFCFDECFDDCFDCCFDBCFDACFD9CFD8CFD7CFD6CFD5CFD4CFD3CFD2CFD1CFD0CFE1
:20AD0B00CFCFCECFCDCFCCCFCBCFCACFC9CFC8CFC7CFC6CFC5CFC4CFC3CFC2CFC1CFC0CFC0
:20AD2B00BFCFBECFBDCFBCCFBBCFBACFB9CFB8CFB7CFB6CFB5CFB4CFB3CFB2CFB1CFB0CFA0
:20AD4B00AFCFAECFADCFACCFABCFAACFA9CFA8CFA7CFA6CFA5CFA4CFA3CFA2CFA1CFA0CF80
:20AD6B009FCF9ECF9DCF9CCF9BCF9ACF99CF98CF97CF96CF95CF94CF93CF92CF91CF90CF60
:20AD8B008FCF8ECF8DCF8CCF8BCF8ACF89CF88CF87CF86CF85CF84CF83CF82CF81CF80CF40
:20ADAB007FCF7ECF7DCF7CCF7BCF7ACF79CF78CF77CF76CF75CF74CF73CF72CF71CF70CF20
:20ADCB006FCF6ECF6DCF6CCF6BCF6ACF69CF68CF67CF66CF65CF64CF63CF62CF61CF60CF00
:15ADEB005FCF5ECF5DCF5CCF5BCF5ACF59CF58CF57CF56CF555F
:20AE0000CF54CF53CF52CF51CF50CF4FCF4ECF4DCF4CCF4BCF4ACF49CF48CF47CF46CF457A
:20AE2000CF44CF43CF42CF41CF40CF3FCF3ECF3DCF3CCF3BCF3ACF39CF38CF37CF36CF355A
:20AE4000CF34CF33CF32CF31CF30CF2FCF2ECF2DCF2CCF2BCF2ACF29CF28CF27CF26CF253A
:20AE6000CF24CF23CF22CF21CF20CF1FCF1ECF1DCF1CCF1BCF1ACF19CF18CF17CF16CF151A
:20AE8000CF14CF13CF12CF11CF10CF0FCF0ECF0DCF0CCF0BCF0ACF09CF08CF07CF06CF05FA
:20AEA000CF04CF03CF02CF01CF00CFFFCFFECFFDCFFCCFFBCFFACFF9CFF8CFF7CFF6CFF5DA
:20AEC000CFF4CFF3CFF2CFF1CFF0CFEFCFEECFEDCFECCFEBCFEACFE9CFE8CFE7CFE6CFE5BA
:20AEE000CFE4CFE3CFE2CFE1CFE0CFDFCFDECFDDCFDCCFDBCFDACFD9CFD8CFD7CFD6CFD59A
:20AF0000CFD4CFD3CFD2CFD1CFD0CFCFCFCECFCDCFCCCFCBCFCACFC9CFC8CFC7CFC6CFC579
:20AF2000CFC4CFC3CFC2CFC1CFC0CFBFCFBECFBDCFBCCFBBCFBACFB9CFB8CFB7CFB6CFB559
:20AF4000CFB4CFB3CFB2CFB1CFB0CFAFCFAECFADCFACCFABCFAACFA9CFA8CFA7CFA6CFA539
:20AF6000CFA4CFA3CFA2CFA1CFA0CF9FCF9ECF9DCF9CCF9BCF9ACF99CF98CF97CF96CF9519
:20AF8000CF94CF93CF92CF91CF90CF8FCF8ECF8DCF8CCF8BCF8ACF89CF88CF87CF86CF85F9
:20AFA000CF84CF83CF82CF81CF80CF7FCF7ECF7DCF7CCF7BCF7ACF79CF78CF77CF76CF75D9
:20AFC000CF74CF73CF72CF71CF70CF6FCF6ECF6DCF6CCF6BCF6ACF69CF68CF67CF66CF65B9
:20AFE000CF64CF63CF62CF61CF60CF5FCF5ECF5DCF5CCF5BCF5ACF59CF58CF57CF56CF5599
:20B00000CF54CF53CF52CF51CF50CF4FCF4ECF4DCF4CCF4BCF4ACF49CF48CF47CF46CF4578
:20B02000CF44CF43CF42CF41CF40CF3FCF3ECF3DCF3CCF3BCF3ACF39CF38CF37CF36CF3558
:20B04000CF34CF33CF32CF31CF30CF2FCF2ECF2DCF2CCF2BCF2ACF29CF28CF27CF26CF2538
:20B06000CF24CF23CF22CF21CF20CF1FCF1ECF1DCF1CCF1BCF1ACF19CF18CF17CF16CF1518
:20B08000CF14CF13CF12CF11CF10CF0FCF0ECF0DCF0CCF0BCF0ACF09CF08CF07CF06CF05F8
:20B0A000CF04CF03CF02CF01CF00CFFFCFFECFFDCFFCCFFBCFFACFF9CFF8CFF7CFF6CFF5D8
:20B0C000CFF4CFF3CFF2CFF1CFF0CFEFCFEECFEDCFECCFEBCFEACFE9CFE8CFE7CFE6CFE5B8
:20B0E000CFE4CFE3CFE2CFE1CFE0CFDFCFDECFDDCFDCCFDBCFDACFD9CFD8CFD7CFD6CFD598
:20B10000CFD4CFD3CFD2CFD1CFD0CFCFCFCECFCDCFCCCFCBCFCACFC9CFC8CFC7CFC6CFC577
:20B12000CFC4CFC3CFC2CFC1CFC0CFBFCFBECFBDCFBCCFBBCFBACFB9CFB8CFB7CFB6CFB557
:20B14000CFB4CFB3CFB2CFB1CFB0CFAFCFAECFADCFACCFABCFAACFA9CFA8CFA7CFA6CFA537
:20B16000CFA4CFA3CFA2CFA1CFA0CF9FCF9ECF9DCF9CCF9BCF9ACF99CF98CF97CF96CF9517
:20B18000CF94CF93CF92CF91CF90CF8FCF8ECF8DCF8CCF8BCF8ACF89CF88CF87CF86CF85F7
:20B1A000CF84CF83CF82CF81CF80CF7FCF7ECF7DCF7CCF7BCF7ACF79CF78CF77CF76CF75D7
:20B1C000CF74CF73CF72CF71CF70CF6FCF6ECF6DCF6CCF6BCF6ACF69CF68CF67CF66CF65B7
:20B1E000CF64CF63CF62CF61CF60CF5FCF5ECF5DCF5CCF5BCF5ACF59CF58CF57CF56CF5597
:20B20000CF54CF53CF52CF51CF50CF4FCF4ECF4DCF4CCF4BCF4ACF49CF48CF47CF46CF4576
:20B22000CF44CF43CF42CF41CF40CF3FCF3ECF3DCF3CCF3BCF3ACF39CF38CF37CF36CF3556
:20B24000CF34CF33CF32CF31CF30CF2FCF2ECF2DCF2CCF2BCF2ACF29CF28CF27CF26CF2536
:20B26000CF24CF23CF22CF21CF20CF1FCF1ECF1DCF1CCF1BCF1ACF19CF18CF17CF16CF1516
:20B28000CF14CF13CF12CF11CF10CF0FCF0ECF0DCF0CCF0BCF0ACF09CF08CF07CF06CF05F6
:20B2A000CF04CF03CF02CF01CF00CFFFCFFECFFDCFFCCFFBCFFACFF9CFF8CFF7CFF6CFF5D6
:20B2C000CFF4CFF3CFF2CFF1CFF0CFEFCFEECFEDCFECCFEBCFEACFE9CFE8CFE7CFE6CFE5B6
:20B2E000CFE4CFE3CFE2CFE1CFE0CFDFCFDECFDDCFDCCFDBCFDACFD9CFD8CFD7CFD6CFD596
:20B30000CFD4CFD3CFD2CFD1CFD0CFCFCFCECFCDCFCCCFCBCFCACFC9CFC8CFC7CFC6CFC575
:20B32000CFC4CFC3CFC2CFC1CFC0CFBFCFBECFBDCFBCCFBBCFBACFB9CFB8CFB7CFB6CFB555
:20B34000CFB4CFB3CFB2CFB1CFB0CFAFCFAECFADCFACCFABCFAACFA9CFA8CFA7CFA6CFA535
:20B36000CFA4CFA3CFA2CFA1CFA0CF9FCF9ECF9DCF9CCF9BCF9ACF99CF98CF97CF96CF9515
:20B38000CF94CF93CF92CF91CF90CF8FCF8ECF8DCF8CCF8BCF8ACF89CF88CF87CF86CF85F5
:20B3A000CF84CF83CF82CF81CF80CF7FCF7ECF7DCF7CCF7BCF7ACF79CF78CF77CF76CF75D5
:20B3C000CF74CF73CF72CF71CF70CF6FCF6ECF6DCF6CCF6BCF6ACF69CF68CF67CF66CF65B5
:20B3E000CF64CF63CF62CF61CF60CF5FCF5ECF5DCF5CCF5BCF5ACF59CF58CF57CF56CF5595
:20B40000CF54CF53CF52CF51CF50CF4FCF4ECF4DCF4CCF4BCF4ACF49CF48CF47CF46CF4574
:20B42000CF44CF43CF42CF41CF40CF3FCF3ECF3DCF3CCF3BCF3ACF39CF38CF37CF36CF3554
:20B44000CF34CF33CF32CF31CF30CF2FCF2ECF2DCF2CCF2BCF2ACF29CF28CF27CF26CF2534
:20B46000CF24CF23CF22CF21CF20CF1FCF1ECF1DCF1CCF1BCF1ACF19CF18CF17CF16CF1514
:20B48000CF14CF13CF12CF11CF10CF0FCF0ECF0DCF0CCF0BCF0ACF09CF08CF07CF06CF05F4
:20B4A000CF04CF03CF02CF01CF00CFFFCFFECFFDCFFCCFFBCFFACFF9CFF8CFF7CFF6CFF5D4
:20B4C000CFF4CFF3CFF2CFF1CFF0CFEFCFEECFEDCFECCFEBCFEACFE9CFE8CFE7CFE6CFE5B4
:20B4E000CFE4CFE3CFE2CFE1CFE0CFDFCFDECFDDCFDCCFDBCFDACFD9CFD8CFD7CFD6CFD594
:20B50000CFD4CFD3CFD2CFD1CFD0CFCFCFCECFCDCFCCCFCBCFCACFC9CFC8CFC7CFC6CFC573
:20B52000CFC4CFC3CFC2CFC1CFC0CFBFCFBECFBDCFBCCFBBCFBACFB9CFB8CFB7CFB6CFB553
:20B54000CFB4CFB3CFB2CFB1CFB0CFAFCFAECFADCFACCFABCFAACFA9CFA8CFA7CFA6CFA533
:20B56000CFA4CFA3CFA2CFA1CFA0CF9FCF9ECF9DCF9CCF9BCF9ACF99CF98CF97CF96CF9513
:20B58000CF94CF93CF92CF91CF90CF8FCF8ECF8DCF8CCF8BCF8ACF89CF88CF87CF86CF85F3
:20B5A000CF84CF83CF82CF81CF80CF7FCF7ECF7DCF7CCF7BCF7ACF79CF78CF77CF76CF75D3
:20B5C000CF74CF73CF72CF71CF70CF6FCF6ECF6DCF6CCF6BCF6ACF69CF68CF67CF66CF65B3
:20B5E000CF64CF63CF62CF61CF60CF5FCF5ECF5DCF5CCF5BCF5ACF59CF58CF57CF56CF5593
:20B60000CF54CF53CF52CF51CF50CF4FCF4ECF4DCF4CCF4BCF4ACF49CF48CF47CF46CF4572
:20B62000CF44CF43CF42CF41CF40CF3FCF3ECF3DCF3CCF3BCF3ACF39CF38CF37CF36CF3552
:20B64000CF34CF33CF32CF31CF30CF2FCF2ECF2DCF2CCF2BCF2ACF29CF28CF27CF26CF2532
:20B66000CF24CF23CF22CF21CF20CF1FCF1ECF1DCF1CCF1BCF1ACF19CF18CF17CF16CF1512
:20B68000CF14CF13CF12CF11CF10CF0FCF0ECF0DCF0CCF0BCF0ACF09CF08CF07CF06CF05F2
:20B6A000CF04CF03CF02CF01CF00CFFFCFFECFFDCFFCCFFBCFFACFF9CFF8CFF7CFF6CFF5D2
:20B6C000CFF4CFF3CFF2CFF1CFF0CFEFCFEECFEDCFECCFEBCFEACFE9CFE8CFE7CFE6CFE5B2
:20B6E000CFE4CFE3CFE2CFE1CFE0CFDFCFDECFDDCFDCCFDBCFDACFD9CFD8CFD7CFD6CFD592
:20B70000CFD4CFD3CFD2CFD1CFD0CFCFCFCECFCDCFCCCFCBCFCACFC9CFC8CFC7CFC6CFC571
:20B72000CFC4CFC3CFC2CFC1CFC0CFBFCFBECFBDCFBCCFBBCFBACFB9CFB8CFB7CFB6CFB551
:20B74000CFB4CFB3CFB2CFB1CFB0CFAFCFAECFADCFACCFABCFAACFA9CFA8CFA7CFA6CFA531
:20B76000CFA4CFA3CFA2CFA1CFA0CF9FCF9ECF9DCF9CCF9BCF9ACF99CF98CF97CF96CF9511
:20B78000CF94CF93CF92CF91CF90CF8FCF8ECF8DCF8CCF8BCF8ACF89CF88CF87CF86CF85F1
:20B7A000CF84CF83CF82CF81CF80CF7FCF7ECF7DCF7CCF7BCF7ACF79CF78CF77CF76CF75D1
:20B7C000CF74CF73CF72CF71CF70CF6FCF6ECF6DCF6CCF6BCF6ACF69CF68CF67CF66CF65B1
:20B7E000CF64CF63CF62CF61CF60CF5FCF5ECF5DCF5CCF5BCF5ACF59CF58CF57CF56CF5591
:20B80000CF54CF53CF52CF51CF50CF4FCF4ECF4DCF4CCF4BCF4ACF49CF48CF47CF46CF4570
:20B82000CF44CF43CF42CF41CF40CF3FCF3ECF3DCF3CCF3BCF3ACF39CF38CF37CF36CF3550
:20B84000CF34CF33CF32CF31CF30CF2FCF2ECF2DCF2CCF2BCF2ACF29CF28CF27CF26CF2530
:20B86000CF24CF23CF22CF21CF20CF1FCF1ECF1DCF1CCF1BCF1ACF19CF18CF17CF16CF1510
:20B88000CF14CF13CF12CF11CF10CF0FCF0ECF0DCF0CCF0BCF0ACF09CF08CF07CF06CF05F0
:20B8A000CF04CF03CF02CF01CF00CFFFCFFECFFDCFFCCFFBCFFACFF9CFF8CFF7CFF6CFF5D0
:20B8C000CFF4CFF3CFF2CFF1CFF0CFEFCFEECFEDCFECCFEBCFEACFE9CFE8CFE7CFE6CFE5B0
:20B8E000CFE4CFE3CFE2CFE1CFE0CFDFCFDECFDDCFDCCFDBCFDACFD9CFD8CFD7CFD6CFD590
:20B90000CFD4CFD3CFD2CFD1CFD0CFCFCFCECFCDCFCCCFCBCFCACFC9CFC8CFC7CFC6CFC56F
:20B92000CFC4CFC3CFC2CFC1CFC0CFBFCFBECFBDCFBCCFBBCFBACFB9CFB8CFB7CFB6CFB54F
:20B94000CFB4CFB3CFB2CFB1CFB0CFAFCFAECFADCFACCFABCFAACFA9CFA8CFA7CFA6CFA52F
:20B96000CFA4CFA3CFA2CFA1CFA0CF9FCF9ECF9DCF9CCF9BCF9ACF99CF98CF97CF96CF950F
:20B98000CF94CF93CF92CF91CF90CF8FCF8ECF8DCF8CCF8BCF8ACF89CF88CF87CF86CF85EF
:20B9A000CF84CF83CF82CF81CF80CF7FCF7ECF7DCF7CCF7BCF7ACF79CF78CF77CF76CF75CF
:20B9C000CF74CF73CF72CF71CF70CF6FCF6ECF6DCF6CCF6BCF6ACF69CF68CF67CF66CF65AF
:20B9E000CF64CF63CF62CF61CF60CF5FCF5ECF5DCF5CCF5BCF5ACF59CF58CF57CF56CF558F
:20BA0000CF54CF53CF52CF51CF50CF4FCF4ECF4DCF4CCF4BCF4ACF49CF48CF47CF46CF456E
:20BA2000CF44CF43CF42CF41CF40CF3FCF3ECF3DCF3CCF3BCF3ACF39CF38CF37CF36CF354E
:20BA4000CF34CF33CF32CF31CF30CF2FCF2ECF2DCF2CCF2BCF2ACF29CF28CF27CF26CF252E
:20BA6000CF24CF23CF22CF21CF20CF1FCF1ECF1DCF1CCF1BCF1ACF19CF18CF17CF16CF150E
:20BA8000CF14CF13CF12CF11CF10CF0FCF0ECF0DCF0CCF0BCF0ACF09CF08CF07CF06CF05EE
:20BAA000CF04CF03CF02CF01CF00CFFFCFFECFFDCFFCCFFBCFFACFF9CFF8CFF7CFF6CFF5CE
:20BAC000CFF4CFF3CFF2CFF1CFF0CFEFCFEECFEDCFECCFEBCFEACFE9CFE8CFE7CFE6CFE5AE
:20BAE000CFE4CFE3CFE2CFE1CFE0CFDFCFDECFDDCFDCCFDBCFDACFD9CFD8CFD7CFD6CFD58E
:20BB0000CFD4CFD3CFD2CFD1CFD0CFCFCFCECFCDCFCCCFCBCFCACFC9CFC8CFC7CFC6CFC56D
:20BB2000CFC4CFC3CFC2CFC1CFC0CFBFCFBECFBDCFBCCFBBCFBACFB9CFB8CFB7CFB6CFB54D
:20BB4000CFB4CFB3CFB2CFB1CFB0CFAFCFAECFADCFACCFABCFAACFA9CFA8CFA7CFA6CFA52D
:20BB6000CFA4CFA3CFA2CFA1CFA0CF9FCF9ECF9DCF9CCF9BCF9ACF99CF98CF97CF96CF950D
:20BB8000CF94CF93CF92CF91CF90CF8FCF8ECF8DCF8CCF8BCF8ACF89CF88CF87CF86CF85ED
:20BBA000CF84CF83CF82CF81CF80CF7FCF7ECF7DCF7CCF7BCF7ACF79CF78CF77CF76CF75CD
:20BBC000CF74CF73CF72CF71CF70CF6FCF6ECF6DCF6CCF6BCF6ACF69CF68CF67CF66CF65AD
:20BBE000CF64CF63CF62CF61CF60CF5FCF5ECF5DCF5CCF5BCF5ACF59CF58CF57CF56CF558D
:20BC0000CF54CF53CF52CF51CF50CF4FCF4ECF4DCF4CCF4BCF4ACF49CF48CF47CF46CF456C
:20BC2000CF44CF43CF42CF41CF40CF3FCF3ECF3DCF3CCF3BCF3ACF39CF38CF37CF36CF354C
:20BC4000CF34CF33CF32CF31CF30CF2FCF2ECF2DCF2CCF2BCF2ACF29CF28CF27CF26CF252C
:20BC6000CF24CF23CF22CF21CF20CF1FCF1ECF1DCF1CCF1BCF1ACF19CF18CF17CF16CF150C
:20BC8000CF14CF13CF12CF11CF10CF0FCF0ECF0DCF0CCF0BCF0ACF09CF08CF07CF06CF05EC
:20BCA000CF04CF03CF02CF01CF00CFFFCFFECFFDCFFCCFFBCFFACFF9CFF8CFF7CFF6CFF5CC
:20BCC000CFF4CFF3CFF2CFF1CFF0CFEFCFEECFEDCFECCFEBCFEACFE9CFE8CFE7CFE6CFE5AC
:20BCE000CFE4CFE3CFE2CFE1CFE0CFDFCFDECFDDCFDCCFDBCFDACFD9CFD8CFD7CFD6CFD58C
:20BD0000CFD4CFD3CFD2CFD1CFD0CFCFCFCECFCDCFCCCFCBCFCACFC9CFC8CFC7CFC6CFC56B
:20BD2000CFC4CFC3CFC2CFC1CFC0CFBFCFBECFBDCFBCCFBBCFBACFB9CFB8CFB7CFB6CFB54B
:20BD4000CFB4CFB3CFB2CFB1CFB0CFAFCFAECFADCFACCFABCFAACFA9CFA8CFA7CFA6CFA52B
:20BD6000CFA4CFA3CFA2CFA1CFA0CF9FCF9ECF9DCF9CCF9BCF9ACF99CF98CF97CF96CF950B
:20BD8000CF94CF93CF92CF91CF90CF8FCF8ECF8DCF8CCF8BCF8ACF89CF88CF87CF86CF85EB
:20BDA000CF84CF83CF82CF81CF80CF7FCF7ECF7DCF7CCF7BCF7ACF79CF78CF77CF76CF75CB
:20BDC000CF74CF73CF72CF71CF70CF6FCF6ECF6DCF6CCF6BCF6ACF69CF68CF67CF66CF65AB
:20BDE000CF64CF63CF62CF61CF60CF5FCF5ECF5DCF5CCF5BCF5ACF59CF58CF57CF56CF558B
:20BE0000CF54CF53CF52CF51CF50CF4FCF4ECF4DCF4CCF4BCF4ACF49CF48CF47CF46CF456A
:20BE2000CF44CF43CF42CF41CF40CF3FCF3ECF3DCF3CCF3BCF3ACF39CF38CF37CF36CF354A
:20BE4000CF34CF33CF32CF31CF30CF2FCF2ECF2DCF2CCF2BCF2ACF29CF28CF27CF26CF252A
:20BE6000CF24CF23CF22CF21CF20CF1FCF1ECF1DCF1CCF1BCF1ACF19CF18CF17CF16CF150A
:20BE8000CF14CF13CF12CF11CF10CF0FCF0ECF0DCF0CCF0BCF0ACF09CF08CF07CF06CF05EA
:20BEA000CF04CF03CF02CF01CF00CFFFCFFECFFDCFFCCFFBCFFACFF9CFF8CFF7CFF6CFF5CA
:20BEC000CFF4CFF3CFF2CFF1CFF0CFEFCFEECFEDCFECCFEBCFEACFE9CFE8CFE7CFE6CFE5AA
:20BEE000CFE4CFE3CFE2CFE1CFE0CFDFCFDECFDDCFDCCFDBCFDACFD9CFD8CFD7CFD6CFD58A
:20BF0000CFD4CFD3CFD2CFD1CFD0CFCFCFCECFCDCFCCCFCBCFCACFC9CFC8CFC7CFC6CFC569
:20BF2000CFC4CFC3CFC2CFC1CFC0CFBFCFBECFBDCFBCCFBBCFBACFB9CFB8CFB7CFB6CFB549
:20BF4000CFB4CFB3CFB2CFB1CFB0CFAFCFAECFADCFACCFABCFAACFA9CFA8CFA7CFA6CFA529
:20BF6000CFA4CFA3CFA2CFA1CFA0CF9FCF9ECF9DCF9CCF9BCF9ACF99CF98CF97CF96CF9509
:20BF8000CF94CF93CF92CF91CF90CF8FCF8ECF8DCF8CCF8BCF8ACF89CF88CF87CF86CF85E9
:20BFA000CF84CF83CF82CF81CF80CF7FCF7ECF7DCF7CCF7BCF7ACF79CF78CF77CF76CF75C9
:20BFC000CF74CF73CF72CF71CF70CF6FCF6ECF6DCF6CCF6BCF6ACF69CF68CF67CF66CF65A9
:20BFE000CF64CF63CF62CF61CF60CF5FCF5ECF5DCF5CCF5BCF5ACF59CF58CF57CF56CF5589
:20C00000CF54CF53CF52CF51CF50CF4FCF4ECF4DCF4CCF4BCF4ACF49CF48CF47CF46CF4568
:20C02000CF44CF43CF42CF41CF40CF3FCF3ECF3DCF3CCF3BCF3ACF39CF38CF37CF36CF3548
:20C04000CF34CF33CF32CF31CF30CF2FCF2ECF2DCF2CCF2BCF2ACF29CF28CF27CF26CF2528
:20C06000CF24CF23CF22CF21CF20CF1FCF1ECF1DCF1CCF1BCF1ACF19CF18CF17CF16CF1508
:20C08000CF14CF13CF12CF11CF10CF0FCF0ECF0DCF0CCF0BCF0ACF09CF08CF07CF06CF05E8
:20C0A000CF04CF03CF02CF01CF00CFFFCFFECFFDCFFCCFFBCFFACFF9CFF8CFF7CFF6CFF5C8
:20C0C000CFF4CFF3CFF2CFF1CFF0CFEFCFEECFEDCFECCFEBCFEACFE9CFE8CFE7CFE6CFE5A8
:20C0E000CFE4CFE3CFE2CFE1CFE0CFDFCFDECFDDCFDCCFDBCFDACFD9CFD8CFD7CFD6CFD588
:20C10000CFD4CFD3CFD2CFD1CFD0CFCFCFCECFCDCFCCCFCBCFCACFC9CFC8CFC7CFC6CFC567
:20C12000CFC4CFC3CFC2CFC1CFC0CFBFCFBECFBDCFBCCFBBCFBACFB9CFB8CFB7CFB6CFB547
:20C14000CFB4CFB3CFB2CFB1CFB0CFAFCFAECFADCFACCFABCFAACFA9CFA8CFA7CFA6CFA527
:20C16000CFA4CFA3CFA2CFA1CFA0CF9FCF9ECF9DCF9CCF9BCF9ACF99CF98CF97CF96CF9507
:20C18000CF94CF93CF92CF91CF90CF8FCF8ECF8DCF8CCF8BCF8ACF89CF88CF87CF86CF85E7
:20C1A000CF84CF83CF82CF81CF80CF7FCF7ECF7DCF7CCF7BCF7ACF79CF78CF77CF76CF75C7
:20C1C000CF74CF73CF72CF71CF70CF6FCF6ECF6DCF6CCF6BCF6ACF69CF68CF67CF66CF65A7
:20C1E000CF64CF63CF62CF61CF60CF5FCF5ECF5DCF5CCF5BCF5ACF59CF58CF57CF56CF5587
:20C20000CF54CF53CF52CF51CF50CF4FCF4ECF4DCF4CCF4BCF4ACF49CF48CF47CF46CF4566
:20C22000CF44CF43CF42CF41CF40CF3FCF3ECF3DCF3CCF3BCF3ACF39CF38CF37CF36CF3546
:20C24000CF34CF33CF32CF31CF30CF2FCF2ECF2DCF2CCF2BCF2ACF29CF28CF27CF26CF2526
:20C26000CF24CF23CF22CF21CF20CF1FCF1ECF1DCF1CCF1BCF1ACF19CF18CF17CF16CF1506
:20C28000CF14CF13CF12CF11CF10CF0FCF0ECF0DCF0CCF0BCF0ACF09CF08CF07CF06CF05E6
:20C2A000CF04CF03CF02CF01CF00CFFFCFFECFFDCFFCCFFBCFFACFF9CFF8CFF7CFF6CFF5C6
:20C2C000CFF4CFF3CFF2CFF1CFF0CFEFCFEECFEDCFECCFEBCFEACFE9CFE8CFE7CFE6CFE5A6
:20C2E000CFE4CFE3CFE2CFE1CFE0CFDFCFDECFDDCFDCCFDBCFDACFD9CFD8CFD7CFD6CFD586
:20C30000CFD4CFD3CFD2CFD1CFD0CFCFCFCECFCDCFCCCFCBCFCACFC9CFC8CFC7CFC6CFC565
:20C32000CFC4CFC3CFC2CFC1CFC0CFBFCFBECFBDCFBCCFBBCFBACFB9CFB8CFB7CFB6CFB545
:20C34000CFB4CFB3CFB2CFB1CFB0CFAFCFAECFADCFACCFABCFAACFA9CFA8CFA7CFA6CFA525
:20C36000CFA4CFA3CFA2CFA1CFA0CF9FCF9ECF9DCF9CCF9BCF9ACF99CF98CF97CF96CF9505
:20C38000CF94CF93CF92CF91CF90CF8FCF8ECF8DCF8CCF8BCF8ACF89CF88CF87CF86CF85E5
:20C3A000CF84CF83CF82CF81CF80CF7FCF7ECF7DCF7CCF7BCF7ACF79CF78CF77CF76CF75C5
:20C3C000CF74CF73CF72CF71CF70CF6FCF6ECF6DCF6CCF6BCF6ACF69CF68CF67CF66CF65A5
:20C3E000CF64CF63CF62CF61CF60CF5FCF5ECF5DCF5CCF5BCF5ACF59CF58CF57CF56CF5585
:20C40000CF54CF53CF52CF51CF50CF4FCF4ECF4DCF4CCF4BCF4ACF49CF48CF47CF46CF4564
:20C42000CF44CF43CF42CF41CF40CF3FCF3ECF3DCF3CCF3BCF3ACF39CF38CF37CF36CF3544
:20C44000CF34CF33CF32CF31CF30CF2FCF2ECF2DCF2CCF2BCF2ACF29CF28CF27CF26CF2524
:20C46000CF24CF23CF22CF21CF20CF1FCF1ECF1DCF1CCF1BCF1ACF19CF18CF17CF16CF1504
:20C48000CF14CF13CF12CF11CF10CF0FCF0ECF0DCF0CCF0BCF0ACF09CF08CF07CF06CF05E4
:20C4A000CF04CF03CF02CF01CF00CFFFCFFECFFDCFFCCFFBCFFACFF9CFF8CFF7CFF6CFF5C4
:20C4C000CFF4CFF3CFF2CFF1CFF0CFEFCFEECFEDCFECCFEBCFEACFE9CFE8CFE7CFE6CFE5A4
:20C4E000CFE4CFE3CFE2CFE1CFE0CFDFCFDECFDDCFDCCFDBCFDACFD9CFD8CFD7CFD6CFD584
:20C50000CFD4CFD3CFD2CFD1CFD0CFCFCFCECFCDCFCCCFCBCFCACFC9CFC8CFC7CFC6CFC563
:20C52000CFC4CFC3CFC2CFC1CFC0CFBFCFBECFBDCFBCCFBBCFBACFB9CFB8CFB7CFB6CFB543
:20C54000CFB4CFB3CFB2CFB1CFB0CFAFCFAECFADCFACCFABCFAACFA9CFA8CFA7CFA6CFA523
:20C56000CFA4CFA3CFA2CFA1CFA0CF9FCF9ECF9DCF9CCF9BCF9ACF99CF98CF97CF96CF9503
:20C58000CF94CF93CF92CF91CF90CF8FCF8ECF8DCF8CCF8BCF8ACF89CF88CF87CF86CF85E3
:20C5A000CF84CF83CF82CF81CF80CF7FCF7ECF7DCF7CCF7BCF7ACF79CF78CF77CF76CF75C3
:20C5C000CF74CF73CF72CF71CF70CF6FCF6ECF6DCF6CCF6BCF6ACF69CF68CF67CF66CF65A3
:20C5E000CF64CF63CF62CF61CF60CF5FCF5ECF5DCF5CCF5BCF5ACF59CF58CF57CF56CF5583
:20C60000CF54CF53CF52CF51CF50CF4FCF4ECF4DCF4CCF4BCF4ACF49CF48CF47CF46CF4562
:20C62000CF44CF43CF42CF41CF40CF3FCF3ECF3DCF3CCF3BCF3ACF39CF38CF37CF36CF3542
:20C64000CF34CF33CF32CF31CF30CF2FCF2ECF2DCF2CCF2BCF2ACF29CF28CF27CF26CF2522
:20C66000CF24CF23CF22CF21CF20CF1FCF1ECF1DCF1CCF1BCF1ACF19CF18CF17CF16CF1502
:20C68000CF14CF13CF12CF11CF10CF0FCF0ECF0DCF0CCF0BCF0ACF09CF08CF07CF06CF05E2
:20C6A000CF04CF03CF02CF01CF00CFFFCFFECFFDCFFCCFFBCFFACFF9CFF8CFF7CFF6CFF5C2
:20C6C000CFF4CFF3CFF2CFF1CFF0CFEFCFEECFEDCFECCFEBCFEACFE9CFE8CFE7CFE6CFE5A2
:20C6E000CFE4CFE3CFE2CFE1CFE0CFDFCFDECFDDCFDCCFDBCFDACFD9CFD8CFD7CFD6CFD582
:20C70000CFD4CFD3CFD2CFD1CFD0CFCFCFCECFCDCFCCCFCBCFCACFC9CFC8CFC7CFC6CFC561
:20C72000CFC4CFC3CFC2CFC1CFC0CFBFCFBECFBDCFBCCFBBCFBACFB9CFB8CFB7CFB6CFB541
:20C74000CFB4CFB3CFB2CFB1CFB0CFAFCFAECFADCFACCFABCFAACFA9CFA8CFA7CFA6CFA521
:20C76000CFA4CFA3CFA2CFA1CFA0CF9FCF9ECF9DCF9CCF9BCF9ACF99CF98CF97CF96CF9501
:20C78000CF94CF93CF92CF91CF90CF8FCF8ECF8DCF8CCF8BCF8ACF89CF88CF87CF86CF85E1
:20C7A000CF84CF83CF82CF81CF80CF7FCF7ECF7DCF7CCF7BCF7ACF79CF78CF77CF76CF75C1
:20C7C000CF74CF73CF72CF71CF70CF6FCF6ECF6DCF6CCF6BCF6ACF69CF68CF67CF66CF65A1
:20C7E000CF64CF63CF62CF61CF60CF5FCF5ECF5DCF5CCF5BCF5ACF59CF58CF57CF56CF5581
:20C80000CF54CF53CF52CF51CF50CF4FCF4ECF4DCF4CCF4BCF4ACF49CF48CF47CF46CF4560
:20C82000CF44CF43CF42CF41CF40CF3FCF3ECF3DCF3CCF3BCF3ACF39CF38CF37CF36CF3540
:20C84000CF34CF33CF32CF31CF30CF2FCF2ECF2DCF2CCF2BCF2ACF29CF28CF27CF26CF2520
:20C86000CF24CF23CF22CF21CF20CF1FCF1ECF1DCF1CCF1BCF1ACF19CF18CF17CF16CF1500
:20C88000CF14CF13CF12CF11CF10CF0FCF0ECF0DCF0CCF0BCF0ACF09CF08CF07CF06CF05E0
:20C8A000CF04CF03CF02CF01CF00CFFFCFFECFFDCFFCCFFBCFFACFF9CFF8CFF7CFF6CFF5C0
:20C8C000CFF4CFF3CFF2CFF1CFF0CFEFCFEECFEDCFECCFEBCFEACFE9CFE8CFE7CFE6CFE5A0
:20C8E000CFE4CFE3CFE2CFE1CFE0CFDFCFDECFDDCFDCCFDBCFDACFD9CFD8CFD7CFD6CFD580
:20C90000CFD4CFD3CFD2CFD1CFD0CFCFCFCECFCDCFCCCFCBCFCACFC9CFC8CFC7CFC6CFC55F
:20C92000CFC4CFC3CFC2CFC1CFC0CFBFCFBECFBDCFBCCFBBCFBACFB9CFB8CFB7CFB6CFB53F
:20C94000CFB4CFB3CFB2CFB1CFB0CFAFCFAECFADCFACCFABCFAACFA9CFA8CFA7CFA6CFA51F
:20C96000CFA4CFA3CFA2CFA1CFA0CF9FCF9ECF9DCF9CCF9BCF9ACF99CF98CF97CF96CF95FF
:20C98000CF94CF93CF92CF91CF90CF8FCF8ECF8DCF8CCF8BCF8ACF89CF88CF87CF86CF85DF
:20C9A000CF84CF83CF82CF81CF80CF7FCF7ECF7DCF7CCF7BCF7ACF79CF78CF77CF76CF75BF
:20C9C000CF74CF73CF72CF71CF70CF6FCF6ECF6DCF6CCF6BCF6ACF69CF68CF67CF66CF659F
:20C9E000CF64CF63CF62CF61CF60CF5FCF5ECF5DCF5CCF5BCF5ACF59CF58CF57CF56CF557F
:20CA0000CF54CF53CF52CF51CF50CF4FCF4ECF4DCF4CCF4BCF4ACF49CF48CF47CF46CF455E
:20CA2000CF44CF43CF42CF41CF40CF3FCF3ECF3DCF3CCF3BCF3ACF39CF38CF37CF36CF353E
:20CA4000CF34CF33CF32CF31CF30CF2FCF2ECF2DCF2CCF2BCF2ACF29CF28CF27CF26CF251E
:20CA6000CF24CF23CF22CF21CF20CF1FCF1ECF1DCF1CCF1BCF1ACF19CF18CF17CF16CF15FE
:20CA8000CF14CF13CF12CF11CF10CF0FCF0ECF0DCF0CCF0BCF0ACF09CF08CF07CF06CF05DE
:20CAA000CF04CF03CF02CF01CF00CFFFCFFECFFDCFFCCFFBCFFACFF9CFF8CFF7CFF6CFF5BE
:20CAC000CFF4CFF3CFF2CFF1CFF0CFEFCFEECFEDCFECCFEBCFEACFE9CFE8CFE7CFE6CFE59E
:20CAE000CFE4CFE3CFE2CFE1CFE0CFDFCFDECFDDCFDCCFDBCFDACFD9CFD8CFD7CFD6CFD57E
:20CB0000CFD4CFD3CFD2CFD1CFD0CFCFCFCECFCDCFCCCFCBCFCACFC9CFC8CFC7CFC6CFC55D
:20CB2000CFC4CFC3CFC2CFC1CFC0CFBFCFBECFBDCFBCCFBBCFBACFB9CFB8CFB7CFB6CFB53D
:20CB4000CFB4CFB3CFB2CFB1CFB0CFAFCFAECFADCFACCFABCFAACFA9CFA8CFA7CFA6CFA51D
:20CB6000CFA4CFA3CFA2CFA1CFA0CF9FCF9ECF9DCF9CCF9BCF9ACF99CF98CF97CF96CF95FD
:20CB8000CF94CF93CF92CF91CF90CF8FCF8ECF8DCF8CCF8BCF8ACF89CF88CF87CF86CF85DD
:20CBA000CF84CF83CF82CF81CF80CF7FCF7ECF7DCF7CCF7BCF7ACF79CF78CF77CF76CF75BD
:20CBC000CF74CF73CF72CF71CF70CF6FCF6ECF6DCF6CCF6BCF6ACF69CF68CF67CF66CF659D
:20CBE000CF64CF63CF62CF61CF60CF5FCF5ECF5DCF5CCF5BCF5ACF59CF58CF57CF56CF557D
:20CC0000CF54CF53CF52CF51CF50CF4FCF4ECF4DCF4CCF4BCF4ACF49CF48CF47CF46CF455C
:20CC2000CF44CF43CF42CF41CF40CF3FCF3ECF3DCF3CCF3BCF3ACF39CF38CF37CF36CF353C
:20CC4000CF34CF33CF32CF31CF30CF2FCF2ECF2DCF2CCF2BCF2ACF29CF28CF27CF26CF251C
:20CC6000CF24CF23CF22CF21CF20CF1FCF1ECF1DCF1CCF1BCF1ACF19CF18CF17CF16CF15FC
:20CC8000CF14CF13CF12CF11CF10CF0FCF0ECF0DCF0CCF0BCF0ACF09CF08CF07CF06CF05DC
:20CCA000CF04CF03CF02CF01CF00CFFFCFFECFFDCFFCCFFBCFFACFF9CFF8CFF7CFF6CFF5BC
:20CCC000CFF4CFF3CFF2CFF1CFF0CFEFCFEECFEDCFECCFEBCFEACFE9CFE8CFE7CFE6CFE59C
:20CCE000CFE4CFE3CFE2CFE1CFE0CFDFCFDECFDDCFDCCFDBCFDACFD9CFD8CFD7CFD6CFD57C
:20CD0000CFD4CFD3CFD2CFD1CFD0CFCFCFCECFCDCFCCCFCBCFCACFC9CFC8CFC7CFC6CFC55B
:20CD2000CFC4CFC3CFC2CFC1CFC0CFBFCFBECFBDCFBCCFBBCFBACFB9CFB8CFB7CFB6CFB53B
:20CD4000CFB4CFB3CFB2CFB1CFB0CFAFCFAECFADCFACCFABCFAACFA9CFA8CFA7CFA6CFA51B
:20CD6000CFA4CFA3CFA2CFA1CFA0CF9FCF9ECF9DCF9CCF9BCF9ACF99CF98CF97CF96CF95FB
:20CD8000CF94CF93CF92CF91CF90CF8FCF8ECF8DCF8CCF8BCF8ACF89CF88CF87CF86CF85DB
:20CDA000CF84CF83CF82CF81CF80CF7FCF7ECF7DCF7CCF7BCF7ACF79CF78CF77CF76CF75BB
:20CDC000CF74CF73CF72CF71CF70CF6FCF6ECF6DCF6CCF6BCF6ACF69CF68CF67CF66CF659B
:20CDE000CF64CF63CF62CF61CF60CF5FCF5ECF5DCF5CCF5BCF5ACF59CF58CF57CF56CF557B
:20CE0000CF54CF53CF52CF51CF50CF4FCF4ECF4DCF4CCF4BCF4ACF49CF48CF47CF46CF455A
:20CE2000CF44CF43CF42CF41CF40CF3FCF3ECF3DCF3CCF3BCF3ACF39CF38CF37CF36CF353A
:20CE4000CF34CF33CF32CF31CF30CF2FCF2ECF2DCF2CCF2BCF2ACF29CF28CF27CF26CF251A
:20CE6000CF24CF23CF22CF21CF20CF1FCF1ECF1DCF1CCF1BCF1ACF19CF18CF17CF16CF15FA
:20CE8000CF14CF13CF12CF11CF10CF0FCF0ECF0DCF0CCF0BCF0ACF09CF08CF07CF06CF05DA
:20CEA000CF04CF03CF02CF01CF00CFFFCFFECFFDCFFCCFFBCFFACFF9CFF8CFF7CFF6CFF5BA
:20CEC000CFF4CFF3CFF2CFF1CFF0CFEFCFEECFEDCFECCFEBCFEACFE9CFE8CFE7CFE6CFE59A
:20CEE000CFE4CFE3CFE2CFE1CFE0CFDFCFDECFDDCFDCCFDBCFDACFD9CFD8CFD7CFD6CFD57A
:20CF0000CFD4CFD3CFD2CFD1CFD0CFCFCFCECFCDCFCCCFCBCFCACFC9CFC8CFC7CFC6CFC559
:20CF2000CFC4CFC3CFC2CFC1CFC0CFBFCFBECFBDCFBCCFBBCFBACFB9CFB8CFB7CFB6CFB539
:20CF4000CFB4CFB3CFB2CFB1CFB0CFAFCFAECFADCFACCFABCFAACFA9CFA8CFA7CFA6CFA519
:20CF6000CFA4CFA3CFA2CFA1CFA0CF9FCF9ECF9DCF9CCF9BCF9ACF99CF98CF97CF96CF95F9
:20CF8000CF94CF93CF92CF91CF90CF8FCF8ECF8DCF8CCF8BCF8ACF89CF88CF87CF86CF85D9
:20CFA000CF84CF83CF82CF81CF80CF7FCF7ECF7DCF7CCF7BCF7ACF79CF78CF77CF76CF75B9
:20CFC000CF74CF73CF72CF71CF70CF6FCF6ECF6DCF6CCF6BCF6ACF69CF68CF67CF66CF6599
:20CFE000CF64CF63CF62CF61CF60CF5FCF5ECF5DCF5CCF5BCF5ACF59CF58CF57CF56CF5579
:20D00000CF54CF53CF52CF51CF50CF4FCF4ECF4DCF4CCF4BCF4ACF49CF48CF47CF46CF4558
:20D02000CF44CF43CF42CF41CF40CF3FCF3ECF3DCF3CCF3BCF3ACF39CF38CF37CF36CF3538
:20D04000CF34CF33CF32CF31CF30CF2FCF2ECF2DCF2CCF2BCF2ACF29CF28CF27CF26CF2518
:20D06000CF24CF23CF22CF21CF20CF1FCF1ECF1DCF1CCF1BCF1ACF19CF18CF17CF16CF15F8
:20D08000CF14CF13CF12CF11CF10CF0FCF0ECF0DCF0CCF0BCF0ACF09CF08CF07CF06CF05D8
:20D0A000CF04CF03CF02CF01CF00CFFFCFFECFFDCFFCCFFBCFFACFF9CFF8CFF7CFF6CFF5B8
:20D0C000CFF4CFF3CFF2CFF1CFF0CFEFCFEECFEDCFECCFEBCFEACFE9CFE8CFE7CFE6CFE598
:20D0E000CFE4CFE3CFE2CFE1CFE0CFDFCFDECFDDCFDCCFDBCFDACFD9CFD8CFD7CFD6CFD578
:20D10000CFD4CFD3CFD2CFD1CFD0CFCFCFCECFCDCFCCCFCBCFCACFC9CFC8CFC7CFC6CFC557
:20D12000CFC4CFC3CFC2CFC1CFC0CFBFCFBECFBDCFBCCFBBCFBACFB9CFB8CFB7CFB6CFB537
:20D14000CFB4CFB3CFB2CFB1CFB0CFAFCFAECFADCFACCFABCFAACFA9CFA8CFA7CFA6CFA517
:20D16000CFA4CFA3CFA2CFA1CFA0CF9FCF9ECF9DCF9CCF9BCF9ACF99CF98CF97CF96CF95F7
:20D18000CF94CF93CF92CF91CF90CF8FCF8ECF8DCF8CCF8BCF8ACF89CF88CF87CF86CF85D7
:20D1A000CF84CF83CF82CF81CF80CF7FCF7ECF7DCF7CCF7BCF7ACF79CF78CF77CF76CF75B7
:20D1C000CF74CF73CF72CF71CF70CF6FCF6ECF6DCF6CCF6BCF6ACF69CF68CF67CF66CF6597
:20D1E000CF64CF63CF62CF61CF60CF5FCF5ECF5DCF5CCF5BCF5ACF59CF58CF57CF56CF5577
:20D20000CF54CF53CF52CF51CF50CF4FCF4ECF4DCF4CCF4BCF4ACF49CF48CF47CF46CF4556
:20D22000CF44CF43CF42CF41CF40CF3FCF3ECF3DCF3CCF3BCF3ACF39CF38CF37CF36CF3536
:20D24000CF34CF33CF32CF31CF30CF2FCF2ECF2DCF2CCF2BCF2ACF29CF28CF27CF26CF2516
:20D26000CF24CF23CF22CF21CF20CF1FCF1ECF1DCF1CCF1BCF1ACF19CF18CF17CF16CF15F6
:20D28000CF14CF13CF12CF11CF10CF0FCF0ECF0DCF0CCF0BCF0ACF09CF08CF07CF06CF05D6
:20D2A000CF04CF03CF02CF01CF00CFFFCFFECFFDCFFCCFFBCFFACFF9CFF8CFF7CFF6CFF5B6
:20D2C000CFF4CFF3CFF2CFF1CFF0CFEFCFEECFEDCFECCFEBCFEACFE9CFE8CFE7CFE6CFE596
:20D2E000CFE4CFE3CFE2CFE1CFE0CFDFCFDECFDDCFDCCFDBCFDACFD9CFD8CFD7CFD6CFD576
:20D30000CFD4CFD3CFD2CFD1CFD0CFCFCFCECFCDCFCCCFCBCFCACFC9CFC8CFC7CFC6CFC555
:20D32000CFC4CFC3CFC2CFC1CFC0CFBFCFBECFBDCFBCCFBBCFBACFB9CFB8CFB7CFB6CFB535
:20D34000CFB4CFB3CFB2CFB1CFB0CFAFCFAECFADCFACCFABCFAACFA9CFA8CFA7CFA6CFA515
:20D36000CFA4CFA3CFA2CFA1CFA0CF9FCF9ECF9DCF9CCF9BCF9ACF99CF98CF97CF96CF95F5
:20D38000CF94CF93CF92CF91CF90CF8FCF8ECF8DCF8CCF8BCF8ACF89CF88CF87CF86CF85D5
:20D3A000CF84CF83CF82CF81CF80CF7FCF7ECF7DCF7CCF7BCF7ACF79CF78CF77CF76CF75B5
:20D3C000CF74CF73CF72CF71CF70CF6FCF6ECF6DCF6CCF6BCF6ACF69CF68CF67CF66CF6595
:20D3E000CF64CF63CF62CF61CF60CF5FCF5ECF5DCF5CCF5BCF5ACF59CF58CF57CF56CF5575
:20D40000CF54CF53CF52CF51CF50CF4FCF4ECF4DCF4CCF4BCF4ACF49CF48CF47CF46CF4554
:20D42000CF44CF43CF42CF41CF40CF3FCF3ECF3DCF3CCF3BCF3ACF39CF38CF37CF36CF3534
:20D44000CF34CF33CF32CF31CF30CF2FCF2ECF2DCF2CCF2BCF2ACF29CF28CF27CF26CF2514
:20D46000CF24CF23CF22CF21CF20CF1FCF1ECF1DCF1CCF1BCF1ACF19CF18CF17CF16CF15F4
:20D48000CF14CF13CF12CF11CF10CF0FCF0ECF0DCF0CCF0BCF0ACF09CF08CF07CF06CF05D4
:20D4A000CF04CF03CF02CF01CF00CFFFCFFECFFDCFFCCFFBCFFACFF9CFF8CFF7CFF6CFF5B4
:20D4C000CFF4CFF3CFF2CFF1CFF0CFEFCFEECFEDCFECCFEBCFEACFE9CFE8CFE7CFE6CFE594
:20D4E000CFE4CFE3CFE2CFE1CFE0CFDFCFDECFDDCFDCCFDBCFDACFD9CFD8CFD7CFD6CFD574
:20D50000CFD4CFD3CFD2CFD1CFD0CFCFCFCECFCDCFCCCFCBCFCACFC9CFC8CFC7CFC6CFC553
:20D52000CFC4CFC3CFC2CFC1CFC0CFBFCFBECFBDCFBCCFBBCFBACFB9CFB8CFB7CFB6CFB533
:20D54000CFB4CFB3CFB2CFB1CFB0CFAFCFAECFADCFACCFABCFAACFA9CFA8CFA7CFA6CFA513
:20D56000CFA4CFA3CFA2CFA1CFA0CF9FCF9ECF9DCF9CCF9BCF9ACF99CF98CF97CF96CF95F3
:20D58000CF94CF93CF92CF91CF90CF8FCF8ECF8DCF8CCF8BCF8ACF89CF88CF87CF86CF85D3
:20D5A000CF84CF83CF82CF81CF80CF7FCF7ECF7DCF7CCF7BCF7ACF79CF78CF77CF76CF75B3
:20D5C000CF74CF73CF72CF71CF70CF6FCF6ECF6DCF6CCF6BCF6ACF69CF68CF67CF66CF6593
:20D5E000CF64CF63CF62CF61CF60CF5FCF5ECF5DCF5CCF5BCF5ACF59CF58CF57CF56CF5573
:20D60000CF54CF53CF52CF51CF50CF4FCF4ECF4DCF4CCF4BCF4ACF49CF48CF47CF46CF4552
:20D62000CF44CF43CF42CF41CF40CF3FCF3ECF3DCF3CCF3BCF3ACF39CF38CF37CF36CF3532
:20D64000CF34CF33CF32CF31CF30CF2FCF2ECF2DCF2CCF2BCF2ACF29CF28CF27CF26CF2512
:20D66000CF24CF23CF22CF21CF20CF1FCF1ECF1DCF1CCF1BCF1ACF19CF18CF17CF16CF15F2
:20D68000CF14CF13CF12CF11CF10CF0FCF0ECF0DCF0CCF0BCF0ACF09CF08CF07CF06CF05D2
:20D6A000CF04CF03CF02CF01CF00CFFFCFFECFFDCFFCCFFBCFFACFF9CFF8CFF7CFF6CFF5B2
:20D6C000CFF4CFF3CFF2CFF1CFF0CFEFCFEECFEDCFECCFEBCFEACFE9CFE8CFE7CFE6CFE592
:20D6E000CFE4CFE3CFE2CFE1CFE0CFDFCFDECFDDCFDCCFDBCFDACFD9CFD8CFD7CFD6CFD572
:20D70000CFD4CFD3CFD2CFD1CFD0CFCFCFCECFCDCFCCCFCBCFCACFC9CFC8CFC7CFC6CFC551
:20D72000CFC4CFC3CFC2CFC1CFC0CFBFCFBECFBDCFBCCFBBCFBACFB9CFB8CFB7CFB6CFB531
:20D74000CFB4CFB3CFB2CFB1CFB0CFAFCFAECFADCFACCFABCFAACFA9CFA8CFA7CFA6CFA511
:20D76000CFA4CFA3CFA2CFA1CFA0CF9FCF9ECF9DCF9CCF9BCF9ACF99CF98CF97CF96CF95F1
:20D78000CF94CF93CF92CF91CF90CF8FCF8ECF8DCF8CCF8BCF8ACF89CF88CF87CF86CF85D1
:20D7A000CF84CF83CF82CF81CF80CF7FCF7ECF7DCF7CCF7BCF7ACF79CF78CF77CF76CF75B1
:20D7C000CF74CF73CF72CF71CF70CF6FCF6ECF6DCF6CCF6BCF6ACF69CF68CF67CF66CF6591
:20D7E000CF64CF63CF62CF61CF60CF5FCF5ECF5DCF5CCF5BCF5ACF59CF58CF57CF56CF5571
:20D80000CF54CF53CF52CF51CF50CF4FCF4ECF4DCF4CCF4BCF4ACF49CF48CF47CF46CF4550
:20D82000CF44CF43CF42CF41CF40CF3FCF3ECF3DCF3CCF3BCF3ACF39CF38CF37CF36CF3530
:20D84000CF34CF33CF32CF31CF30CF2FCF2ECF2DCF2CCF2BCF2ACF29CF28CF27CF26CF2510
:20D86000CF24CF23CF22CF21CF20CF1FCF1ECF1DCF1CCF1BCF1ACF19CF18CF17CF16CF15F0
:20D88000CF14CF13CF12CF11CF10CF0FCF0ECF0DCF0CCF0BCF0ACF09CF08CF07CF06CF05D0
:20D8A000CF04CF03CF02CF01CF00CFFFCFFECFFDCFFCCFFBCFFACFF9CFF8CFF7CFF6CFF5B0
:20D8C000CFF4CFF3CFF2CFF1CFF0CFEFCFEECFEDCFECCFEBCFEACFE9CFE8CFE7CFE6CFE590
:20D8E000CFE4CFE3CFE2CFE1CFE0CFDFCFDECFDDCFDCCFDBCFDACFD9CFD8CFD7CFD6CFD570
:20D90000CFD4CFD3CFD2CFD1CFD0CFCFCFCECFCDCFCCCFCBCFCACFC9CFC8CFC7CFC6CFC54F
:20D92000CFC4CFC3CFC2CFC1CFC0CFBFCFBECFBDCFBCCFBBCFBACFB9CFB8CFB7CFB6CFB52F
:20D94000CFB4CFB3CFB2CFB1CFB0CFAFCFAECFADCFACCFABCFAACFA9CFA8CFA7CFA6CFA50F
:20D96000CFA4CFA3CFA2CFA1CFA0CF9FCF9ECF9DCF9CCF9BCF9ACF99CF98CF97CF96CF95EF
:20D98000CF94CF93CF92CF91CF90CF8FCF8ECF8DCF8CCF8BCF8ACF89CF88CF87CF86CF85CF
:20D9A000CF84CF83CF82CF81CF80CF7FCF7ECF7DCF7CCF7BCF7ACF79CF78CF77CF76CF75AF
:20D9C000CF74CF73CF72CF71CF70CF6FCF6ECF6DCF6CCF6BCF6ACF69CF68CF67CF66CF658F
:20D9E000CF64CF63CF62CF61CF60CF5FCF5ECF5DCF5CCF5BCF5ACF59CF58CF57CF56CF556F
:20DA0000CF54CF53CF52CF51CF50CF4FCF4ECF4DCF4CCF4BCF4ACF49CF48CF47CF46CF454E
:20DA2000CF44CF43CF42CF41CF40CF3FCF3ECF3DCF3CCF3BCF3ACF39CF38CF37CF36CF352E
:20DA4000CF34CF33CF32CF31CF30CF2FCF2ECF2DCF2CCF2BCF2ACF29CF28CF27CF26CF250E
:20DA6000CF24CF23CF22CF21CF20CF1FCF1ECF1DCF1CCF1BCF1ACF19CF18CF17CF16CF15EE
:20DA8000CF14CF13CF12CF11CF10CF0FCF0ECF0DCF0CCF0BCF0ACF09CF08CF07CF06CF05CE
:20DAA000CF04CF03CF02CF01CF00CFFFCFFECFFDCFFCCFFBCFFACFF9CFF8CFF7CFF6CFF5AE
:20DAC000CFF4CFF3CFF2CFF1CFF0CFEFCFEECFEDCFECCFEBCFEACFE9CFE8CFE7CFE6CFE58E
:20DAE000CFE4CFE3CFE2CFE1CFE0CFDFCFDECFDDCFDCCFDBCFDACFD9CFD8CFD7CFD6CFD56E
:20DB0000CFD4CFD3CFD2CFD1CFD0CFCFCFCECFCDCFCCCFCBCFCACFC9CFC8CFC7CFC6CFC54D
:20DB2000CFC4CFC3CFC2CFC1CFC0CFBFCFBECFBDCFBCCFBBCFBACFB9CFB8CFB7CFB6CFB52D
:20DB4000CFB4CFB3CFB2CFB1CFB0CFAFCFAECFADCFACCFABCFAACFA9CFA8CFA7CFA6CFA50D
:20DB6000CFA4CFA3CFA2CFA1CFA0CF9FCF9ECF9DCF9CCF9BCF9ACF99CF98CF97CF96CF95ED
:20DB8000CF94CF93CF92CF91CF90CF8FCF8ECF8DCF8CCF8BCF8ACF89CF88CF87CF86CF85CD
:20DBA000CF84CF83CF82CF81CF80CF7FCF7ECF7DCF7CCF7BCF7ACF79CF78CF77CF76CF75AD
:20DBC000CF74CF73CF72CF71CF70CF6FCF6ECF6DCF6CCF6BCF6ACF69CF68CF67CF66CF658D
:20DBE000CF64CF63CF62CF61CF60CF5FCF5ECF5DCF5CCF5BCF5ACF59CF58CF57CF56CF556D
:20DC0000CF54CF53CF52CF51CF50CF4FCF4ECF4DCF4CCF4BCF4ACF49CF48CF47CF46CF454C
:20DC2000CF44CF43CF42CF41CF40CF3FCF3ECF3DCF3CCF3BCF3ACF39CF38CF37CF36CF352C
:20DC4000CF34CF33CF32CF31CF30CF2FCF2ECF2DCF2CCF2BCF2ACF29CF28CF27CF26CF250C
:20DC6000CF24CF23CF22CF21CF20CF1FCF1ECF1DCF1CCF1BCF1ACF19CF18CF17CF16CF15EC
:20DC8000CF14CF13CF12CF11CF10CF0FCF0ECF0DCF0CCF0BCF0ACF09CF08CF07CF06CF05CC
:20DCA000CF04CF03CF02CF01CF00CFFFCFFECFFDCFFCCFFBCFFACFF9CFF8CFF7CFF6CFF5AC
:20DCC000CFF4CFF3CFF2CFF1CFF0CFEFCFEECFEDCFECCFEBCFEACFE9CFE8CFE7CFE6CFE58C
:20DCE000CFE4CFE3CFE2CFE1CFE0CFDFCFDECFDDCFDCCFDBCFDACFD9CFD8CFD7CFD6CFD56C
:20DD0000CFD4CFD3CFD2CFD1CFD0CFCFCFCECFCDCFCCCFCBCFCACFC9CFC8CFC7CFC6CFC54B
:20DD2000CFC4CFC3CFC2CFC1CFC0CFBFCFBECFBDCFBCCFBBCFBACFB9CFB8CFB7CFB6CFB52B
:20DD4000CFB4CFB3CFB2CFB1CFB0CFAFCFAECFADCFACCFABCFAACFA9CFA8CFA7CFA6CFA50B
:20DD6000CFA4CFA3CFA2CFA1CFA0CF9FCF9ECF9DCF9CCF9BCF9ACF99CF98CF97CF96CF95EB
:20DD8000CF94CF93CF92CF91CF90CF8FCF8ECF8DCF8CCF8BCF8ACF89CF88CF87CF86CF85CB
:20DDA000CF84CF83CF82CF81CF80CF7FCF7ECF7DCF7CCF7BCF7ACF79CF78CF77CF76CF75AB
:20DDC000CF74CF73CF72CF71CF70CF6FCF6ECF6DCF6CCF6BCF6ACF69CF68CF67CF66CF658B
:20DDE000CF64CF63CF62CF61CF60CF5FCF5ECF5DCF5CCF5BCF5ACF59CF58CF57CF56CF556B
:20DE0000CF54CF53CF52CF51CF50CF4FCF4ECF4DCF4CCF4BCF4ACF49CF48CF47CF46CF454A
:20DE2000CF44CF43CF42CF41CF40CF3FCF3ECF3DCF3CCF3BCF3ACF39CF38CF37CF36CF352A
:20DE4000CF34CF33CF32CF31CF30CF2FCF2ECF2DCF2CCF2BCF2ACF29CF28CF27CF26CF250A
:20DE6000CF24CF23CF22CF21CF20CF1FCF1ECF1DCF1CCF1BCF1ACF19CF18CF17CF16CF15EA
:20DE8000CF14CF13CF12CF11CF10CF0FCF0ECF0DCF0CCF0BCF0ACF09CF08CF07CF06CF05CA
:20DEA000CF04CF03CF02CF01CF00CFFFCFFECFFDCFFCCFFBCFFACFF9CFF8CFF7CFF6CFF5AA
:20DEC000CFF4CFF3CFF2CFF1CFF0CFEFCFEECFEDCFECCFEBCFEACFE9CFE8CFE7CFE6CFE58A
:20DEE000CFE4CFE3CFE2CFE1CFE0CFDFCFDECFDDCFDCCFDBCFDACFD9CFD8CFD7CFD6CFD56A
:20DF0000CFD4CFD3CFD2CFD1CFD0CFCFCFCECFCDCFCCCFCBCFCACFC9CFC8CFC7CFC6CFC549
:20DF2000CFC4CFC3CFC2CFC1CFC0CFBFCFBECFBDCFBCCFBBCFBACFB9CFB8CFB7CFB6CFB529
:20DF4000CFB4CFB3CFB2CFB1CFB0CFAFCFAECFADCFACCFABCFAACFA9CFA8CFA7CFA6CFA509
:20DF6000CFA4CFA3CFA2CFA1CFA0CF9FCF9ECF9DCF9CCF9BCF9ACF99CF98CF97CF96CF95E9
:20DF8000CF94CF93CF92CF91CF90CF8FCF8ECF8DCF8CCF8BCF8ACF89CF88CF87CF86CF85C9
:20DFA000CF84CF83CF82CF81CF80CF7FCF7ECF7DCF7CCF7BCF7ACF79CF78CF77CF76CF75A9
:20DFC000CF74CF73CF72CF71CF70CF6FCF6ECF6DCF6CCF6BCF6ACF69CF68CF67CF66CF6589
:20DFE000CF64CF63CF62CF61CF60CF5FCF5ECF5DCF5CCF5BCF5ACF59CF58CF57CF56CF5569
:20E00000CF54CF53CF52CF51CF50CF4FCF4ECF4DCF4CCF4BCF4ACF49CF48CF47CF46CF4548
:20E02000CF44CF43CF42CF41CF40CF3FCF3ECF3DCF3CCF3BCF3ACF39CF38CF37CF36CF3528
:20E04000CF34CF33CF32CF31CF30CF2FCF2ECF2DCF2CCF2BCF2ACF29CF28CF27CF26CF2508
:20E06000CF24CF23CF22CF21CF20CF1FCF1ECF1DCF1CCF1BCF1ACF19CF18CF17CF16CF15E8
:20E08000CF14CF13CF12CF11CF10CF0FCF0ECF0DCF0CCF0BCF0ACF09CF08CF07CF06CF05C8
:20E0A000CF04CF03CF02CF01CF00CFFFCFFECFFDCFFCCFFBCFFACFF9CFF8CFF7CFF6CFF5A8
:20E0C000CFF4CFF3CFF2CFF1CFF0CFEFCFEECFEDCFECCFEBCFEACFE9CFE8CFE7CFE6CFE588
:20E0E000CFE4CFE3CFE2CFE1CFE0CFDFCFDECFDDCFDCCFDBCFDACFD9CFD8CFD7CFD6CFD568
:20E10000CFD4CFD3CFD2CFD1CFD0CFCFCFCECFCDCFCCCFCBCFCACFC9CFC8CFC7CFC6CFC547
:20E12000CFC4CFC3CFC2CFC1CFC0CFBFCFBECFBDCFBCCFBBCFBACFB9CFB8CFB7CFB6CFB527
:20E14000CFB4CFB3CFB2CFB1CFB0CFAFCFAECFADCFACCFABCFAACFA9CFA8CFA7CFA6CFA507
:20E16000CFA4CFA3CFA2CFA1CFA0CF9FCF9ECF9DCF9CCF9BCF9ACF99CF98CF97CF96CF95E7
:20E18000CF94CF93CF92CF91CF90CF8FCF8ECF8DCF8CCF8BCF8ACF89CF88CF87CF86CF85C7
:20E1A000CF84CF83CF82CF81CF80CF7FCF7ECF7DCF7CCF7BCF7ACF79CF78CF77CF76CF75A7
:20E1C000CF74CF73CF72CF71CF70CF6FCF6ECF6DCF6CCF6BCF6ACF69CF68CF67CF66CF6587
:20E1E000CF64CF63CF62CF61CF60CF5FCF5ECF5DCF5CCF5BCF5ACF59CF58CF57CF56CF5567
:20E20000CF54CF53CF52CF51CF50CF4FCF4ECF4DCF4CCF4BCF4ACF49CF48CF47CF46CF4546
:20E22000CF44CF43CF42CF41CF40CF3FCF3ECF3DCF3CCF3BCF3ACF39CF38CF37CF36CF3526
:20E24000CF34CF33CF32CF31CF30CF2FCF2ECF2DCF2CCF2BCF2ACF29CF28CF27CF26CF2506
:20E26000CF24CF23CF22CF21CF20CF1FCF1ECF1DCF1CCF1BCF1ACF19CF18CF17CF16CF15E6
:20E28000CF14CF13CF12CF11CF10CF0FCF0ECF0DCF0CCF0BCF0ACF09CF08CF07CF06CF05C6
:20E2A000CF04CF03CF02CF01CF00CFFFCFFECFFDCFFCCFFBCFFACFF9CFF8CFF7CFF6CFF5A6
:20E2C000CFF4CFF3CFF2CFF1CFF0CFEFCFEECFEDCFECCFEBCFEACFE9CFE8CFE7CFE6CFE586
:20E2E000CFE4CFE3CFE2CFE1CFE0CFDFCFDECFDDCFDCCFDBCFDACFD9CFD8CFD7CFD6CFD566
:20E30000CFD4CFD3CFD2CFD1CFD0CFCFCFCECFCDCFCCCFCBCFCACFC9CFC8CFC7CFC6CFC545
:20E32000CFC4CFC3CFC2CFC1CFC0CFBFCFBECFBDCFBCCFBBCFBACFB9CFB8CFB7CFB6CFB525
:20E34000CFB4CFB3CFB2CFB1CFB0CFAFCFAECFADCFACCFABCFAACFA9CFA8CFA7CFA6CFA505
:20E36000CFA4CFA3CFA2CFA1CFA0CF9FCF9ECF9DCF9CCF9BCF9ACF99CF98CF97CF96CF95E5
:20E38000CF94CF93CF92CF91CF90CF8FCF8ECF8DCF8CCF8BCF8ACF89CF88CF87CF86CF85C5
:20E3A000CF84CF83CF82CF81CF80CF7FCF7ECF7DCF7CCF7BCF7ACF79CF78CF77CF76CF75A5
:20E3C000CF74CF73CF72CF71CF70CF6FCF6ECF6DCF6CCF6BCF6ACF69CF68CF67CF66CF6585
:20E3E000CF64CF63CF62CF61CF60CF5FCF5ECF5DCF5CCF5BCF5ACF59CF58CF57CF56CF5565
:20E40000CF54CF53CF52CF51CF50CF4FCF4ECF4DCF4CCF4BCF4ACF49CF48CF47CF46CF4544
:20E42000CF44CF43CF42CF41CF40CF3FCF3ECF3DCF3CCF3BCF3ACF39CF38CF37CF36CF3524
:20E44000CF34CF33CF32CF31CF30CF2FCF2ECF2DCF2CCF2BCF2ACF29CF28CF27CF26CF2504
:20E46000CF24CF23CF22CF21CF20CF1FCF1ECF1DCF1CCF1BCF1ACF19CF18CF17CF16CF15E4
:20E48000CF14CF13CF12CF11CF10CF0FCF0ECF0DCF0CCF0BCF0ACF09CF08CF07CF06CF05C4
:20E4A000CF04CF03CF02CF01CF00CFFFCFFECFFDCFFCCFFBCFFACFF9CFF8CFF7CFF6CFF5A4
:20E4C000CFF4CFF3CFF2CFF1CFF0CFEFCFEECFEDCFECCFEBCFEACFE9CFE8CFE7CFE6CFE584
:20E4E000CFE4CFE3CFE2CFE1CFE0CFDFCFDECFDDCFDCCFDBCFDACFD9CFD8CFD7CFD6CFD564
:20E50000CFD4CFD3CFD2CFD1CFD0CFCFCFCECFCDCFCCCFCBCFCACFC9CFC8CFC7CFC6CFC543
:20E52000CFC4CFC3CFC2CFC1CFC0CFBFCFBECFBDCFBCCFBBCFBACFB9CFB8CFB7CFB6CFB523
:20E54000CFB4CFB3CFB2CFB1CFB0CFAFCFAECFADCFACCFABCFAACFA9CFA8CFA7CFA6CFA503
:20E56000CFA4CFA3CFA2CFA1CFA0CF9FCF9ECF9DCF9CCF9BCF9ACF99CF98CF97CF96CF95E3
:20E58000CF94CF93CF92CF91CF90CF8FCF8ECF8DCF8CCF8BCF8ACF89CF88CF87CF86CF85C3
:20E5A000CF84CF83CF82CF81CF80CF7FCF7ECF7DCF7CCF7BCF7ACF79CF78CF77CF76CF75A3
:20E5C000CF74CF73CF72CF71CF70CF6FCF6ECF6DCF6CCF6BCF6ACF69CF68CF67CF66CF6583
:20E5E000CF64CF63CF62CF61CF60CF5FCF5ECF5DCF5CCF5BCF5ACF59CF58CF57CF56CF5563
:20E60000CF54CF53CF52CF51CF50CF4FCF4ECF4DCF4CCF4BCF4ACF49CF48CF47CF46CF4542
:20E62000CF44CF43CF42CF41CF40CF3FCF3ECF3DCF3CCF3BCF3ACF39CF38CF37CF36CF3522
:20E64000CF34CF33CF32CF31CF30CF2FCF2ECF2DCF2CCF2BCF2ACF29CF28CF27CF26CF2502
:20E66000CF24CF23CF22CF21CF20CF1FCF1ECF1DCF1CCF1BCF1ACF19CF18CF17CF16CF15E2
:20E68000CF14CF13CF12CF11CF10CF0FCF0ECF0DCF0CCF0BCF0ACF09CF08CF07CF06CF05C2
:20E6A000CF04CF03CF02CF01CF00CFFFCFFECFFDCFFCCFFBCFFACFF9CFF8CFF7CFF6CFF5A2
:20E6C000CFF4CFF3CFF2CFF1CFF0CFEFCFEECFEDCFECCFEBCFEACFE9CFE8CFE7CFE6CFE582
:20E6E000CFE4CFE3CFE2CFE1CFE0CFDFCFDECFDDCFDCCFDBCFDACFD9CFD8CFD7CFD6CFD562
:20E70000CFD4CFD3CFD2CFD1CFD0CFCFCFCECFCDCFCCCFCBCFCACFC9CFC8CFC7CFC6CFC541
:20E72000CFC4CFC3CFC2CFC1CFC0CFBFCFBECFBDCFBCCFBBCFBACFB9CFB8CFB7CFB6CFB521
:20E74000CFB4CFB3CFB2CFB1CFB0CFAFCFAECFADCFACCFABCFAACFA9CFA8CFA7CFA6CFA501
:20E76000CFA4CFA3CFA2CFA1CFA0CF9FCF9ECF9DCF9CCF9BCF9ACF99CF98CF97CF96CF95E1
:20E78000CF94CF93CF92CF91CF90CF8FCF8ECF8DCF8CCF8BCF8ACF89CF88CF87CF86CF85C1
:20E7A000CF84CF83CF82CF81CF80CF7FCF7ECF7DCF7CCF7BCF7ACF79CF78CF77CF76CF75A1
:20E7C000CF74CF73CF72CF71CF70CF6FCF6ECF6DCF6CCF6BCF6ACF69CF68CF67CF66CF6581
:20E7E000CF64CF63CF62CF61CF60CF5FCF5ECF5DCF5CCF5BCF5ACF59CF58CF57CF56CF5561
:20E80000CF54CF53CF52CF51CF50CF4FCF4ECF4DCF4CCF4BCF4ACF49CF48CF47CF46CF4540
:20E82000CF44CF43CF42CF41CF40CF3FCF3ECF3DCF3CCF3BCF3ACF39CF38CF37CF36CF3520
:20E84000CF34CF33CF32CF31CF30CF2FCF2ECF2DCF2CCF2BCF2ACF29CF28CF27CF26CF2500
:20E86000CF24CF23CF22CF21CF20CF1FCF1ECF1DCF1CCF1BCF1ACF19CF18CF17CF16CF15E0
:20E88000CF14CF13CF12CF11CF10CF0FCF0ECF0DCF0CCF0BCF0ACF09CF08CF07CF06CF05C0
:20E8A000CF04CF03CF02CF01CF00CFFFCFFECFFDCFFCCFFBCFFACFF9CFF8CFF7CFF6CFF5A0
:20E8C000CFF4CFF3CFF2CFF1CFF0CFEFCFEECFEDCFECCFEBCFEACFE9CFE8CFE7CFE6CFE580
:20E8E000CFE4CFE3CFE2CFE1CFE0CFDFCFDECFDDCFDCCFDBCFDACFD9CFD8CFD7CFD6CFD560
:20E90000CFD4CFD3CFD2CFD1CFD0CFCFCFCECFCDCFCCCFCBCFCACFC9CFC8CFC7CFC6CFC53F
:20E92000CFC4CFC3CFC2CFC1CFC0CFBFCFBECFBDCFBCCFBBCFBACFB9CFB8CFB7CFB6CFB51F
:20E94000CFB4CFB3CFB2CFB1CFB0CFAFCFAECFADCFACCFABCFAACFA9CFA8CFA7CFA6CFA5FF
:20E96000CFA4CFA3CFA2CFA1CFA0CF9FCF9ECF9DCF9CCF9BCF9ACF99CF98CF97CF96CF95DF
:20E98000CF94CF93CF92CF91CF90CF8FCF8ECF8DCF8CCF8BCF8ACF89CF88CF87CF86CF85BF
:20E9A000CF84CF83CF82CF81CF80CF7FCF7ECF7DCF7CCF7BCF7ACF79CF78CF77CF76CF759F
:20E9C000CF74CF73CF72CF71CF70CF6FCF6ECF6DCF6CCF6BCF6ACF69CF68CF67CF66CF657F
:20E9E000CF64CF63CF62CF61CF60CF5FCF5ECF5DCF5CCF5BCF5ACF59CF58CF57CF56CF555F
:20EA0000CF54CF53CF52CF51CF50CF4FCF4ECF4DCF4CCF4BCF4ACF49CF48CF47CF46CF453E
:20EA2000CF44CF43CF42CF41CF40CF3FCF3ECF3DCF3CCF3BCF3ACF39CF38CF37CF36CF351E
:20EA4000CF34CF33CF32CF31CF30CF2FCF2ECF2DCF2CCF2BCF2ACF29CF28CF27CF26CF25FE
:20EA6000CF24CF23CF22CF21CF20CF1FCF1ECF1DCF1CCF1BCF1ACF19CF18CF17CF16CF15DE
:20EA8000CF14CF13CF12CF11CF10CF0FCF0ECF0DCF0CCF0BCF0ACF09CF08CF07CF06CF05BE
:20EAA000CF04CF03CF02CF01CF00CFFFCFFECFFDCFFCCFFBCFFACFF9CFF8CFF7CFF6CFF59E
:20EAC000CFF4CFF3CFF2CFF1CFF0CFEFCFEECFEDCFECCFEBCFEACFE9CFE8CFE7CFE6CFE57E
:20EAE000CFE4CFE3CFE2CFE1CFE0CFDFCFDECFDDCFDCCFDBCFDACFD9CFD8CFD7CFD6CFD55E
:20EB0000CFD4CFD3CFD2CFD1CFD0CFCFCFCECFCDCFCCCFCBCFCACFC9CFC8CFC7CFC6CFC53D
:20EB2000CFC4CFC3CFC2CFC1CFC0CFBFCFBECFBDCFBCCFBBCFBACFB9CFB8CFB7CFB6CFB51D
:20EB4000CFB4CFB3CFB2CFB1CFB0CFAFCFAECFADCFACCFABCFAACFA9CFA8CFA7CFA6CFA5FD
:20EB6000CFA4CFA3CFA2CFA1CFA0CF9FCF9ECF9DCF9CCF9BCF9ACF99CF98CF97CF96CF95DD
:20EB8000CF94CF93CF92CF91CF90CF8FCF8ECF8DCF8CCF8BCF8ACF89CF88CF87CF86CF85BD
:20EBA000CF84CF83CF82CF81CF80CF7FCF7ECF7DCF7CCF7BCF7ACF79CF78CF77CF76CF759D
:20EBC000CF74CF73CF72CF71CF70CF6FCF6ECF6DCF6CCF6BCF6ACF69CF68CF67CF66CF657D
:20EBE000CF64CF63CF62CF61CF60CF5FCF5ECF5DCF5CCF5BCF5ACF59CF58CF57CF56CF555D
:20EC0000CF54CF53CF52CF51CF50CF4FCF4ECF4DCF4CCF4BCF4ACF49CF48CF47CF46CF453C
:20EC2000CF44CF43CF42CF41CF40CF3FCF3ECF3DCF3CCF3BCF3ACF39CF38CF37CF36CF351C
:20EC4000CF34CF33CF32CF31CF30CF2FCF2ECF2DCF2CCF2BCF2ACF29CF28CF27CF26CF25FC
:20EC6000CF24CF23CF22CF21CF20CF1FCF1ECF1DCF1CCF1BCF1ACF19CF18CF17CF16CF15DC
:20EC8000CF14CF13CF12CF11CF10CF0FCF0ECF0DCF0CCF0BCF0ACF09CF08CF07CF06CF05BC
:20ECA000CF04CF03CF02CF01CF00CFFFCFFECFFDCFFCCFFBCFFACFF9CFF8CFF7CFF6CFF59C
:20ECC000CFF4CFF3CFF2CFF1CFF0CFEFCFEECFEDCFECCFEBCFEACFE9CFE8CFE7CFE6CFE57C
:20ECE000CFE4CFE3CFE2CFE1CFE0CFDFCFDECFDDCFDCCFDBCFDACFD9CFD8CFD7CFD6CFD55C
:20ED0000CFD4CFD3CFD2CFD1CFD0CFCFCFCECFCDCFCCCFCBCFCACFC9CFC8CFC7CFC6CFC53B
:20ED2000CFC4CFC3CFC2CFC1CFC0CFBFCFBECFBDCFBCCFBBCFBACFB9CFB8CFB7CFB6CFB51B
:20ED4000CFB4CFB3CFB2CFB1CFB0CFAFCFAECFADCFACCFABCFAACFA9CFA8CFA7CFA6CFA5FB
:20ED6000CFA4CFA3CFA2CFA1CFA0CF9FCF9ECF9DCF9CCF9BCF9ACF99CF98CF97CF96CF95DB
:20ED8000CF94CF93CF92CF91CF90CF8FCF8ECF8DCF8CCF8BCF8ACF89CF88CF87CF86CF85BB
:20EDA000CF84CF83CF82CF81CF80CF7FCF7ECF7DCF7CCF7BCF7ACF79CF78CF77CF76CF759B
:20EDC000CF74CF73CF72CF71CF70CF6FCF6ECF6DCF6CCF6BCF6ACF69CF68CF67CF66CF657B
:20EDE000CF64CF63CF62CF61CF60CF5FCF5ECF5DCF5CCF5BCF5ACF59CF58CF57CF56CF555B
:20EE0000CF54CF53CF52CF51CF50CF4FCF4ECF4DCF4CCF4BCF4ACF49CF48CF47CF46CF453A
:20EE2000CF44CF43CF42CF41CF40CF3FCF3ECF3DCF3CCF3BCF3ACF39CF38CF37CF36CF351A
:20EE4000CF34CF33CF32CF31CF30CF2FCF2ECF2DCF2CCF2BCF2ACF29CF28CF27CF26CF25FA
:20EE6000CF24CF23CF22CF21CF20CF1FCF1ECF1DCF1CCF1BCF1ACF19CF18CF17CF16CF15DA
:20EE8000CF14CF13CF12CF11CF10CF0FCF0ECF0DCF0CCF0BCF0ACF09CF08CF07CF06CF05BA
:20EEA000CF04CF03CF02CF01CF00CFFFCFFECFFDCFFCCFFBCFFACFF9CFF8CFF7CFF6CFF59A
:20EEC000CFF4CFF3CFF2CFF1CFF0CFEFCFEECFEDCFECCFEBCFEACFE9CFE8CFE7CFE6CFE57A
:20EEE000CFE4CFE3CFE2CFE1CFE0CFDFCFDECFDDCFDCCFDBCFDACFD9CFD8CFD7CFD6CFD55A
:20EF0000CFD4CFD3CFD2CFD1CFD0CFCFCFCECFCDCFCCCFCBCFCACFC9CFC8CFC7CFC6CFC539
:20EF2000CFC4CFC3CFC2CFC1CFC0CFBFCFBECFBDCFBCCFBBCFBACFB9CFB8CFB7CFB6CFB519
:20EF4000CFB4CFB3CFB2CFB1CFB0CFAFCFAECFADCFACCFABCFAACFA9CFA8CFA7CFA6CFA5F9
:20EF6000CFA4CFA3CFA2CFA1CFA0CF9FCF9ECF9DCF9CCF9BCF9ACF99CF98CF97CF96CF95D9
:20EF8000CF94CF93CF92CF91CF90CF8FCF8ECF8DCF8CCF8BCF8ACF89CF88CF87CF86CF85B9
:20EFA000CF84CF83CF82CF81CF80CF7FCF7ECF7DCF7CCF7BCF7ACF79CF78CF77CF76CF7599
:20EFC000CF74CF73CF72CF71CF70CF6FCF6ECF6DCF6CCF6BCF6ACF69CF68CF67CF66CF6579
:20EFE000CF64CF63CF62CF61CF60CF5FCF5ECF5DCF5CCF5BCF5ACF59CF58CF57CF56CF5559
:20F00000CF54CF53CF52CF51CF50CF4FCF4ECF4DCF4CCF4BCF4ACF49CF48CF47CF46CF4538
:20F02000CF44CF43CF42CF41CF40CF3FCF3ECF3DCF3CCF3BCF3ACF39CF38CF37CF36CF3518
:20F04000CF34CF33CF32CF31CF30CF2FCF2ECF2DCF2CCF2BCF2ACF29CF28CF27CF26CF25F8
:20F06000CF24CF23CF22CF21CF20CF1FCF1ECF1DCF1CCF1BCF1ACF19CF18CF17CF16CF15D8
:20F08000CF14CF13CF12CF11CF10CF0FCF0ECF0DCF0CCF0BCF0ACF09CF08CF07CF06CF05B8
:20F0A000CF04CF03CF02CF01CF00CFFFCFFECFFDCFFCCFFBCFFACFF9CFF8CFF7CFF6CFF598
:20F0C000CFF4CFF3CFF2CFF1CFF0CFEFCFEECFEDCFECCFEBCFEACFE9CFE8CFE7CFE6CFE578
:20F0E000CFE4CFE3CFE2CFE1CFE0CFDFCFDECFDDCFDCCFDBCFDACFD9CFD8CFD7CFD6CFD558
:20F10000CFD4CFD3CFD2CFD1CFD0CFCFCFCECFCDCFCCCFCBCFCACFC9CFC8CFC7CFC6CFC537
:20F12000CFC4CFC3CFC2CFC1CFC0CFBFCFBECFBDCFBCCFBBCFBACFB9CFB8CFB7CFB6CFB517
:20F14000CFB4CFB3CFB2CFB1CFB0CFAFCFAECFADCFACCFABCFAACFA9CFA8CFA7CFA6CFA5F7
:20F16000CFA4CFA3CFA2CFA1CFA0CF9FCF9ECF9DCF9CCF9BCF9ACF99CF98CF97CF96CF95D7
:20F18000CF94CF93CF92CF91CF90CF8FCF8ECF8DCF8CCF8BCF8ACF89CF88CF87CF86CF85B7
:20F1A000CF84CF83CF82CF81CF80CF7FCF7ECF7DCF7CCF7BCF7ACF79CF78CF77CF76CF7597
:20F1C000CF74CF73CF72CF71CF70CF6FCF6ECF6DCF6CCF6BCF6ACF69CF68CF67CF66CF6577
:20F1E000CF64CF63CF62CF61CF60CF5FCF5ECF5DCF5CCF5BCF5ACF59CF58CF57CF56CF5557
:20F20000CF54CF53CF52CF51CF50CF4FCF4ECF4DCF4CCF4BCF4ACF49CF48CF47CF46CF4536
:20F22000CF44CF43CF42CF41CF40CF3FCF3ECF3DCF3CCF3BCF3ACF39CF38CF37CF36CF3516
:20F24000CF34CF33CF32CF31CF30CF2FCF2ECF2DCF2CCF2BCF2ACF29CF28CF27CF26CF25F6
:20F26000CF24CF23CF22CF21CF20CF1FCF1ECF1DCF1CCF1BCF1ACF19CF18CF17CF16CF15D6
:20F28000CF14CF13CF12CF11CF10CF0FCF0ECF0DCF0CCF0BCF0ACF09CF08CF07CF06CF05B6
:20F2A000CF04CF03CF02CF01CF00CFFFCFFECFFDCFFCCFFBCFFACFF9CFF8CFF7CFF6CFF596
:20F2C000CFF4CFF3CFF2CFF1CFF0CFEFCFEECFEDCFECCFEBCFEACFE9CFE8CFE7CFE6CFE576
:20F2E000CFE4CFE3CFE2CFE1CFE0CFDFCFDECFDDCFDCCFDBCFDACFD9CFD8CFD7CFD6CFD556
:20F30000CFD4CFD3CFD2CFD1CFD0CFCFCFCECFCDCFCCCFCBCFCACFC9CFC8CFC7CFC6CFC535
:20F32000CFC4CFC3CFC2CFC1CFC0CFBFCFBECFBDCFBCCFBBCFBACFB9CFB8CFB7CFB6CFB515
:20F34000CFB4CFB3CFB2CFB1CFB0CFAFCFAECFADCFACCFABCFAACFA9CFA8CFA7CFA6CFA5F5
:20F36000CFA4CFA3CFA2CFA1CFA0CF9FCF9ECF9DCF9CCF9BCF9ACF99CF98CF97CF96CF95D5
:20F38000CF94CF93CF92CF91CF90CF8FCF8ECF8DCF8CCF8BCF8ACF89CF88CF87CF86CF85B5
:20F3A000CF84CF83CF82CF81CF80CF7FCF7ECF7DCF7CCF7BCF7ACF79CF78CF77CF76CF7595
:20F3C000CF74CF73CF72CF71CF70CF6FCF6ECF6DCF6CCF6BCF6ACF69CF68CF67CF66CF6575
:20F3E000CF64CF63CF62CF61CF60CF5FCF5ECF5DCF5CCF5BCF5ACF59CF58CF57CF56CF5555
:20F40000CF54CF53CF52CF51CF50CF4FCF4ECF4DCF4CCF4BCF4ACF49CF48CF47CF46CF4534
:20F42000CF44CF43CF42CF41CF40CF3FCF3ECF3DCF3CCF3BCF3ACF39CF38CF37CF36CF3514
:20F44000CF34CF33CF32CF31CF30CF2FCF2ECF2DCF2CCF2BCF2ACF29CF28CF27CF26CF25F4
:20F46000CF24CF23CF22CF21CF20CF1FCF1ECF1DCF1CCF1BCF1ACF19CF18CF17CF16CF15D4
:20F48000CF14CF13CF12CF11CF10CF0FCF0ECF0DCF0CCF0BCF0ACF09CF08CF07CF06CF05B4
:20F4A000CF04CF03CF02CF01CF00CFFFCFFECFFDCFFCCFFBCFFACFF9CFF8CFF7CFF6CFF594
:20F4C000CFF4CFF3CFF2CFF1CFF0CFEFCFEECFEDCFECCFEBCFEACFE9CFE8CFE7CFE6CFE574
:20F4E000CFE4CFE3CFE2CFE1CFE0CFDFCFDECFDDCFDCCFDBCFDACFD9CFD8CFD7CFD6CFD554
:20F50000CFD4CFD3CFD2CFD1CFD0CFCFCFCECFCDCFCCCFCBCFCACFC9CFC8CFC7CFC6CFC533
:20F52000CFC4CFC3CFC2CFC1CFC0CFBFCFBECFBDCFBCCFBBCFBACFB9CFB8CFB7CFB6CFB513
:20F54000CFB4CFB3CFB2CFB1CFB0CFAFCFAECFADCFACCFABCFAACFA9CFA8CFA7CFA6CFA5F3
:20F56000CFA4CFA3CFA2CFA1CFA0CF9FCF9ECF9DCF9CCF9BCF9ACF99CF98CF97CF96CF95D3
:20F58000CF94CF93CF92CF91CF90CF8FCF8ECF8DCF8CCF8BCF8ACF89CF88CF87CF86CF85B3
:20F5A000CF84CF83CF82CF81CF80CF7FCF7ECF7DCF7CCF7BCF7ACF79CF78CF77CF76CF7593
:20F5C000CF74CF73CF72CF71CF70CF6FCF6ECF6DCF6CCF6BCF6ACF69CF68CF67CF66CF6573
:20F5E000CF64CF63CF62CF61CF60CF5FCF5ECF5DCF5CCF5BCF5ACF59CF58CF57CF56CF5553
:20F60000CF54CF53CF52CF51CF50CF4FCF4ECF4DCF4CCF4BCF4ACF49CF48CF47CF46CF4532
:20F62000CF44CF43CF42CF41CF40CF3FCF3ECF3DCF3CCF3BCF3ACF39CF38CF37CF36CF3512
:20F64000CF34CF33CF32CF31CF30CF2FCF2ECF2DCF2CCF2BCF2ACF29CF28CF27CF26CF25F2
:20F66000CF24CF23CF22CF21CF20CF1FCF1ECF1DCF1CCF1BCF1ACF19CF18CF17CF16CF15D2
:20F68000CF14CF13CF12CF11CF10CF0FCF0ECF0DCF0CCF0BCF0ACF09CF08CF07CF06CF05B2
:20F6A000CF04CF03CF02CF01CF00CFFFCFFECFFDCFFCCFFBCFFACFF9CFF8CFF7CFF6CFF592
:20F6C000CFF4CFF3CFF2CFF1CFF0CFEFCFEECFEDCFECCFEBCFEACFE9CFE8CFE7CFE6CFE572
:20F6E000CFE4CFE3CFE2CFE1CFE0CFDFCFDECFDDCFDCCFDBCFDACFD9CFD8CFD7CFD6CFD552
:20F70000CFD4CFD3CFD2CFD1CFD0CFCFCFCECFCDCFCCCFCBCFCACFC9CFC8CFC7CFC6CFC531
:20F72000CFC4CFC3CFC2CFC1CFC0CFBFCFBECFBDCFBCCFBBCFBACFB9CFB8CFB7CFB6CFB511
:20F74000CFB4CFB3CFB2CFB1CFB0CFAFCFAECFADCFACCFABCFAACFA9CFA8CFA7CFA6CFA5F1
:20F76000CFA4CFA3CFA2CFA1CFA0CF9FCF9ECF9DCF9CCF9BCF9ACF99CF98CF97CF96CF95D1
:20F78000CF94CF93CF92CF91CF90CF8FCF8ECF8DCF8CCF8BCF8ACF89CF88CF87CF86CF85B1
:20F7A000CF84CF83CF82CF81CF80CF7FCF7ECF7DCF7CCF7BCF7ACF79CF78CF77CF76CF7591
:20F7C000CF74CF73CF72CF71CF70CF6FCF6ECF6DCF6CCF6BCF6ACF69CF68CF67CF66CF6571
:20F7E000CF64CF63CF62CF61CF60CF5FCF5ECF5DCF5CCF5BCF5ACF59CF58CF57CF56CF5551
:20F80000CF54CF53CF52CF51CF50CF4FCF4ECF4DCF4CCF4BCF4ACF49CF48CF47CF46CF4530
:20F82000CF44CF43CF42CF41CF40CF3FCF3ECF3DCF3CCF3BCF3ACF39CF38CF37CF36CF3510
:20F84000CF34CF33CF32CF31CF30CF2FCF2ECF2DCF2CCF2BCF2ACF29CF28CF27CF26CF25F0
:20F86000CF24CF23CF22CF21CF20CF1FCF1ECF1DCF1CCF1BCF1ACF19CF18CF17CF16CF15D0
:20F88000CF14CF13CF12CF11CF10CF0FCF0ECF0DCF0CCF0BCF0ACF09CF08CF07CF06CF05B0
:20F8A000CF04CF03CF02CF01CF00CFFFCFFECFFDCFFCCFFBCFFACFF9CFF8CFF7CFF6CFF590
:20F8C000CFF4CFF3CFF2CFF1CFF0CFEFCFEECFEDCFECCFEBCFEACFE9CFE8CFE7CFE6CFE570
:20F8E000CFE4CFE3CFE2CFE1CFE0CFDFCFDECFDDCFDCCFDBCFDACFD9CFD8CFD7CFD6CFD550
:20F90000CFD4CFD3CFD2CFD1CFD0CFCFCFCECFCDCFCCCFCBCFCACFC9CFC8CFC7CFC6CFC52F
:20F92000CFC4CFC3CFC2CFC1CFC0CFBFCFBECFBDCFBCCFBBCFBACFB9CFB8CFB7CFB6CFB50F
:20F94000CFB4CFB3CFB2CFB1CFB0CFAFCFAECFADCFACCFABCFAACFA9CFA8CFA7CFA6CFA5EF
:20F96000CFA4CFA3CFA2CFA1CFA0CF9FCF9ECF9DCF9CCF9BCF9ACF99CF98CF97CF96CF95CF
:20F98000CF94CF93CF92CF91CF90CF8FCF8ECF8DCF8CCF8BCF8ACF89CF88CF87CF86CF85AF
:20F9A000CF84CF83CF82CF81CF80CF7FCF7ECF7DCF7CCF7BCF7ACF79CF78CF77CF76CF758F
:20F9C000CF74CF73CF72CF71CF70CF6FCF6ECF6DCF6CCF6BCF6ACF69CF68CF67CF66CF656F
:20F9E000CF64CF63CF62CF61CF60CF5FCF5ECF5DCF5CCF5BCF5ACF59CF58CF57CF56CF554F
:20FA0000CF54CF53CF52CF51CF50CF4FCF4ECF4DCF4CCF4BCF4ACF49CF48CF47CF46CF452E
:20FA2000CF44CF43CF42CF41CF40CF3FCF3ECF3DCF3CCF3BCF3ACF39CF38CF37CF36CF350E
:20FA4000CF34CF33CF32CF31CF30CF2FCF2ECF2DCF2CCF2BCF2ACF29CF28CF27CF26CF25EE
:20FA6000CF24CF23CF22CF21CF20CF1FCF1ECF1DCF1CCF1BCF1ACF19CF18CF17CF16CF15CE
:20FA8000CF14CF13CF12CF11CF10CF0FCF0ECF0DCF0CCF0BCF0ACF09CF08CF07CF06CF05AE
:20FAA000CF04CF03CF02CF01CF00CFFFCFFECFFDCFFCCFFBCFFACFF9CFF8CFF7CFF6CFF58E
:20FAC000CFF4CFF3CFF2CFF1CFF0CFEFCFEECFEDCFECCFEBCFEACFE9CFE8CFE7CFE6CFE56E
:20FAE000CFE4CFE3CFE2CFE1CFE0CFDFCFDECFDDCFDCCFDBCFDACFD9CFD8CFD7CFD6CFD54E
:20FB0000CFD4CFD3CFD2CFD1CFD0CFCFCFCECFCDCFCCCFCBCFCACFC9CFC8CFC7CFC6CFC52D
:20FB2000CFC4CFC3CFC2CFC1CFC0CFBFCFBECFBDCFBCCFBBCFBACFB9CFB8CFB7CFB6CFB50D
:20FB4000CFB4CFB3CFB2CFB1CFB0CFAFCFAECFADCFACCFABCFAACFA9CFA8CFA7CFA6CFA5ED
:20FB6000CFA4CFA3CFA2CFA1CFA0CF9FCF9ECF9DCF9CCF9BCF9ACF99CF98CF97CF96CF95CD
:20FB8000CF94CF93CF92CF91CF90CF8FCF8ECF8DCF8CCF8BCF8ACF89CF88CF87CF86CF85AD
:20FBA000CF84CF83CF82CF81CF80CF7FCF7ECF7DCF7CCF7BCF7ACF79CF78CF77CF76CF758D
:20FBC000CF74CF73CF72CF71CF70CF6FCF6ECF6DCF6CCF6BCF6ACF69CF68CF67CF66CF656D
:20FBE000CF64CF63CF62CF61CF60CF5FCF5ECF5DCF5CCF5BCF5ACF59CF58CF57CF56CF554D
:20FC0000CF54CF53CF52CF51CF50CF4FCF4ECF4DCF4CCF4BCF4ACF49CF48CF47CF46CF452C
:20FC2000CF44CF43CF42CF41CF40CF3FCF3ECF3DCF3CCF3BCF3ACF39CF38CF37CF36CF350C
:20FC4000CF34CF33CF32CF31CF30CF2FCF2ECF2DCF2CCF2BCF2ACF29CF28CF27CF26CF25EC
:20FC6000CF24CF23CF22CF21CF20CF1FCF1ECF1DCF1CCF1BCF1ACF19CF18CF17CF16CF15CC
:20FC8000CF14CF13CF12CF11CF10CF0FCF0ECF0DCF0CCF0BCF0ACF09CF08CF07CF06CF05AC
:20FCA000CF04CF03CF02CF01CF00CFFFCFFECFFDCFFCCFFBCFFACFF9CFF8CFF7CFF6CFF58C
:20FCC000CFF4CFF3CFF2CFF1CFF0CFEFCFEECFEDCFECCFEBCFEACFE9CFE8CFE7CFE6CFE56C
:20FCE000CFE4CFE3CFE2CFE1CFE0CFDFCFDECFDDCFDCCFDBCFDACFD9CFD8CFD7CFD6CFD54C
:20FD0000CFD4CFD3CFD2CFD1CFD0CFCFCFCECFCDCFCCCFCBCFCACFC9CFC8CFC7CFC6CFC52B
:20FD2000CFC4CFC3CFC2CFC1CFC0CFBFCFBECFBDCFBCCFBBCFBACFB9CFB8CFB7CFB6CFB50B
:20FD4000CFB4CFB3CFB2CFB1CFB0CFAFCFAECFADCFACCFABCFAACFA9CFA8CFA7CFA6CFA5EB
:20FD6000CFA4CFA3CFA2CFA1CFA0CF9FCF9ECF9DCF9CCF9BCF9ACF99CF98CF97CF96CF95CB
:20FD8000CF94CF93CF92CF91CF90CF8FCF8ECF8DCF8CCF8BCF8ACF89CF88CF87CF86CF85AB
:20FDA000CF84CF83CF82CF81CF80CF7FCF7ECF7DCF7CCF7BCF7ACF79CF78CF77CF76CF758B
:20FDC000CF74CF73CF72CF71CF70CF6FCF6ECF6DCF6CCF6BCF6ACF69CF68CF67CF66CF656B
:20FDE000CF64CF63CF62CF61CF60CF5FCF5ECF5DCF5CCF5BCF5ACF59CF58CF57CF56CF554B
:20FE0000CF54CF53CF52CF51CF50CF4FCF4ECF4DCF4CCF4BCF4ACF49CF48CF47CF46CF452A
:20FE2000CF44CF43CF42CF41CF40CF3FCF3ECF3DCF3CCF3BCF3ACF39CF38CF37CF36CF350A
:20FE4000CF34CF33CF32CF31CF30CF2FCF2ECF2DCF2CCF2BCF2ACF29CF28CF27CF26CF25EA
:20FE6000CF24CF23CF22CF21CF20CF1FCF1ECF1DCF1CCF1BCF1ACF19CF18CF17CF16CF15CA
:20FE8000CF14CF13CF12CF11CF10CF0FCF0ECF0DCF0CCF0BCF0ACF09CF08CF07CF06CF05AA
:20FEA000CF04CF03CF02CF01CF00CFFFCFFECFFDCFFCCFFBCFFACFF9CFF8CFF7CFF6CFF58A
:20FEC000CFF4CFF3CFF2CFF1CFF0CFEFCFEECFEDCFECCFEBCFEACFE9CFE8CFE7CFE6CFE56A
:20FEE000CFE4CFE3CFE2CFE1CFE0CFDFCFDECFDDCFDCCFDBCFDACFD9CFD8CFD7CFD6CFD54A
:20FF0000CFD4CFD3CFD2CFD1CFD0CFCFCFCECFCDCFCCCFCBCFCACFC9CFC8CFC7CFC6CFC529
:20FF2000CFC4CFC3CFC2CFC1CFC0CFBFCFBECFBDCFBCCFBBCFBACFB9CFB8CFB7CFB6CFB509
:20FF4000CFB4CFB3CFB2CFB1CFB0CFAFCFAECFADCFACCFABCFAACFA9CFA8CFA7CFA6CFA5E9
:20FF6000CFA4CFA3CFA2CFA1CFA0CF9FCF9ECF9DCF9CCF9BCF9ACF99CF98CF97CF96CF95C9
:20FF8000CF94CF93CF92CF91CF90CF8FCF8ECF8DCF8CCF8BCF8ACF89CF88CF87CF86CF85A9
:20FFA000CF84CF83CF82CF81CF80CF7FCF7ECF7DCF7CCF7BCF7ACF79CF78CF77CF76CF7589
:20FFC000CF74CF73CF72CF71CF70CF6FCF6ECF6DCF6CCF6BCF6ACF69CF68CF67CF66CF6569
:1EFFE000CF64CF63CF62CF61CF60CF5FCF5ECF5DCF5CCF5BCF5ACF59CF58CF57CF566F
:01FFFF00CF32
:00000001FF
